:020000040800F2
:1000000000000120C1460008B92C0008BB2C0008E4
:10001000BD2C0008BF2C0008C12C00080000000007
:10002000000000000000000000000000C32C0008D9
:10003000C52C000800000000C72C0008C92C0008CF
:100040001147000811470008CD2C0008114700088F
:100050001147000811470008D92C0008DF2C0008C0
:100060001147000811470008072D00081147000834
:10007000E52C0008E72C0008E92C0008F52C000806
:10008000012D0008032D0008114700081147000842
:100090000000000011470008092D00081147000862
:1000A00011470008114700081147000811470008D0
:1000B00011470008114700081147000811470008C0
:1000C00011470008114700081147000811470008B0
:1000D00011470008112D00081147000811470008BA
:1000E000114700080F2D00081D2D000811470008BA
:1000F0001147000800000000000000001147000840
:100100001147000811470008292D00081147000871
:10011000114700081147000811470008114700085F
:10012000114700081147000811470008114700084F
:08013000114700081147000807
:1001400010B5054C237833B9044B13B10448AFF311
:1001500000800123237010BD840A002000000000ED
:10016000F86E010808B5034B1BB103490348AFF310
:10017000008008BD00000000880A0020F86E010819
:1001800014214160704714207047406A7047000096
:1001900081010008870100088B010008A101000807
:1001A00010B5044604F1100000F05CFCC4F8F8003F
:1001B0000148C4F87C0110BD90010008F8B5E6B014
:1001C00004460D4616461F460A4906A800F0CAFE18
:1001D00070996F9A05910492009733466E996D9AC3
:1001E000039102922A466C990191214600F060F831
:1001F00067B0F0BD9C010008F8B5E6B004460D46B6
:1002000016461F46094906A800F0ACFE6F996E9A83
:100210000491039200976D996C9A02910192334672
:100220002A46214600F087F867B0F0BD9C0100081F
:1002300038B500281CBF01680029184A23D1184B83
:100240001C684FF6F0710C404CF24025AC421FBFC9
:100250001B6819404CF27024A14212D1114D29683B
:1002600079B911490B68C3F30B03B3F58A6F1FBF4C
:100270000968C1F30B0140F28343994204BF012195
:10028000117028B905E0094B994204BF0121117092
:100290004068BDE8324002F01BB900BFA00A002050
:1002A00000ED00E0002004E00010005C0000374892
:1002B0002DE9F04104460D46216816464A681F465E
:1002C00090478046B8F5403F2ED122680A9993683E
:1002D000204698478046B8F5403F25D12368089AC4
:1002E0000799D3F80CC02046E0478046B8F5403F58
:1002F0001AD12368069A39461F692046B8478046B6
:10030000B8F5403F10D1236829465D693246204642
:10031000A8478046B8F5403F06D123680B9A099953
:100320009D692046A847804621680A682046904774
:100330004046BDE8F0812DE9F04104460D462168B4
:1003400016464A681F4690478046B8F5403F2ED172
:1003500022680A999368204698478046B8F5403F3E
:1003600025D12368089A0799D3F80CC02046E047A6
:100370008046B8F5403F1AD12368069A39461F696E
:100380002046B8478046B8F5403F10D1236829463B
:100390005D6932462046A8478046B8F5403F06D101
:1003A00023680999DD6900222046A8478046216814
:1003B0000A68204690474046BDE8F0814FF440303F
:1003C00070470000F0B50C4685B0114600281A466B
:1003D0001CBF0568002D0B4B11D082B104B971B957
:1003E0000D9860B10F9E0E9F0A9B02900496039792
:1003F0000B980C9E009001962046A847034618468D
:1004000005B0F0BD020003002DE9F04F0646D0B064
:100410000868F56DD6F860E0726EB76EF36E00BADC
:1004200000906C46486800BA60600DF1400888682A
:1004300000BAA060C86800BAE060086900BA20612C
:10044000486900BA6061886900BAA061C86900BAE9
:10045000E061086A00BA2062486A00BA6062886A8D
:1004600000BAA062C86A00BAE062086B00BA2063F2
:10047000486B00BA6063886B00BAA063C86B00BAAF
:10048000E063402058F80C1C58F820CC58F838ACE1
:100490008CEA010158F840CC8AEA01018CEA010992
:1004A0004FEAF979401E48F8049BEBD187EA020035
:1004B00000EA0E00784010EBF5610098DFF824C4E4
:1004C00041186144C81882EABE032B404FEAF0612C
:1004D00053405918636859186144CF194FEAB5035E
:1004E00083EABE01014081EABE0111EBF765A16814
:1004F0004D196544A91883EAB0023A404FEAF16504
:100500005A405519E26855194FEAB70282EAB00716
:1005100065440F4005EBBE0E97EAB00717EBFE658A
:1005200027697D194FEAB10782EA0701654401EAAC
:100530000E01EB18514011EBF36561694D194FEA5B
:10054000BE0187EA010E65440EEA030E15EBB0000A
:100550008EEA070E0EEBF065D4F818E0754465449A
:10056000AA1881EAB30505404FEAF26E4D40AE4449
:10057000E569AE44E64477444FEAB00080EAB30E42
:100580000EEA020E8EEAB30E0EEBF765D4F820E009
:1005900075446544691880EAB2053D404FEAF16E42
:1005A0004540AE44656AAE44E6440EEBB3034FEA01
:1005B000B70787EAB20E0EEA010E8EEAB20E0EEB14
:1005C000F365D4F828E075446544281887EAB10536
:1005D0001D404FEAF06E7D40AE44E56AAE44E6440D
:1005E0000EEBB2024FEAB30383EAB10E0EEA000E3D
:1005F0008EEAB10E0EEBF265D4F830E07544654436
:10060000EF1983EAB00515404FEAF76E5D40AE443E
:10061000656BAE44E6440EEBB1014FEAB20282EAEA
:10062000B00E0EEA070E8EEAB00E0EEBF165D4F8AE
:1006300038E075446544EB1882EAB7050D404FEA8F
:10064000F36E5540AE44E56BAE44E6440EEBB000AD
:100650004FEAB10181EAB70E0EEA030E8EEAB70E39
:100660000EEBF065D4F840E07544654481EAB30EC2
:10067000AA180EEA000E4FEAF2658EEA010E7544E2
:10068000DDF844E04FEAB000754480EAB30E6544FB
:100690000EEA020E15EBB7078EEAB30E0EEBF76506
:1006A000DDF848E04FEAB202754480EA020E654484
:1006B0000EEA070E69188EEA000E0EEBF165DDF802
:1006C0004CE07544654405EBB3034FEAB70E1427BD
:1006D0000DF1500CDFF810528EEA010B82EA0B0B81
:1006E0000BEBF36A5CF804BBDA44AA44504483EA97
:1006F000B10B4FEAF06A8EEA0B0BDA445CF804BBEC
:10070000DA44AA44524480EAB30B4FEAF26A8BEA15
:10071000B10BDA445CF804BBDA444FEAB000AA44F7
:1007200080EA020BD6448BEAB30B0BEBFE6A5CF853
:1007300004BBDA444FEAB202AA4482EA0E0B0AEB87
:10074000B10180EA0B0B0BEBF16A5CF804BBDA44F5
:100750007F1DAA44282F0AEBB3034FEABE0EBBD37A
:100760003C2F61D3502F4DD204EB870CC7F15407B7
:100770005E4CA7FB04A504465D4FA8088EEA010A5B
:1007800082EA0A0A5CF804BB0AEBF3655D447D1952
:100790002C1983EAB10A4FEAF4658EEA0A0A554435
:1007A0005CF804AB5CF804BB55447D19AA1884EAD4
:1007B000B30A4FEAF2658AEAB10A55445D444FEA4A
:1007C000B4047D1984EA020AAE448AEAB30A0AEB49
:1007D000FE655CF804AB55444FEAB2027D1982EA2B
:1007E0000E0A15EBB10184EA0A0A5CF804BB0AEBB5
:1007F000F1655D447D1915EBB303401E4FEABE0E53
:10080000BCD12046F46D1B19F365336EC9183166EF
:10081000716E71447166B36ED218B266F16E401893
:10082000F06650B0BDE8F08F4EEA010B0EEA010A07
:100830000BEA020B4BEA0A0A0AEBF36554F827A00D
:10084000DFF8B0C0554443EAB10B654403EAB10A8E
:100850000BEA0E0B28184BEA0A0A7F1C0AEBF0651C
:1008600054F827A0554440EAB30B654400EAB30AA4
:100870000BEAB10BAA184BEA0A0A7F1C0AEBF265D5
:1008800054F827A055444FEAB00040EA020B6544F3
:1008900000EA020A0BEAB30BAE444BEA0A0A7F1CD9
:1008A0000AEBFE6554F827A055444FEAB20242EA2B
:1008B0000E0B654402EA0E0A0BEA000B15EBB101C0
:1008C0004BEA0A0A7F1C0AEBF16554F827A055444D
:1008D0007F1C65443C2F05EBB3034FEABE0EA3D348
:1008E00040E700BF9979825AA1EBD96ECDCCCCCC30
:1008F000D6C162CADCBC1B8F00B581B00168074A53
:10090000914200D110B9064801B000BD7C2114F01D
:10091000BAFB4FF4003001B000BD00BF040A00086C
:10092000030002002DE9F0410B4A92E8F85188B02B
:10093000694681E8F8510268084B9A4200D118B91B
:10094000074808B0BDE8F0811422083000F04FFBE2
:1009500008B0BDE8F08100BFE4090008040A0008FF
:1009600003000200152904D20268044B9A4200D108
:1009700008B903487047083000F048BB040A000873
:100980000300020010B481B013460268074CA24273
:1009900000D118B901B010BC0548704701B000F192
:1009A000240210BC083000F035BB00BF040A000868
:1009B0000300020010B481B013460268074CA24243
:1009C00000D118B901B010BC054870470A4601B003
:1009D00000F1240110BC083000F070BB040A0008CC
:1009E000030002000123456789ABCDEFFEDCBA9816
:1009F00076543210F0E1D2C3000000000000000085
:100A000000000000F9080008250900086509000831
:100A100085090008B509000809040008810F0008CD
:100A2000CD0F0008890F0008F0B5A3B004460B48AD
:100A300002900D4616461F46094B0822402104A885
:100A400000F0D1FA28980190009733462A462146B3
:100A500002A800F01BF823B0F0BD00BF040A000894
:100A6000180A000810B5040008BF002408D0054883
:100A7000054B20600822402104F1080000F0B3FA81
:100A8000204610BD040A0008180A00082DE9F041AC
:100A900004460E46216817464A681D469047804620
:100AA000B8F5003F19D12268069993682046984707
:100AB0008046B8F5003F10D123683146DE683A46DB
:100AC0002046B0478046B8F5003F06D12368079A14
:100AD00029461D692046A847804621680A682046A5
:100AE00090474046BDE8F08110B500F033FA4FF46E
:100AF000403400280EBF034C4FF4C07114F0C3FA09
:100B0000204610BD0200030010B5044600F022FA92
:100B100008B9054810BD0021A160D0F87C211168FA
:100B200088474FF4403010BD0200030070B5044602
:100B30000D4600F00FFA064E40B1D0F87C01416836
:100B40008847A84224BF65604FF44036304670BDE8
:100B5000020003002DE9FF4715000C4600D02CB120
:100B6000064600F0F7F95FEA000801D16448C3E0E7
:100B7000D8F8F80001684A689047B0F5003F17D1EF
:100B8000D8F87C118A68404690478146B9F1810FB8
:100B900080F09E80A94508F1FC0A17D2D8F8F80029
:100BA0000368D3F80CC02A462146E047B0F5003F61
:100BB00040F08E80D8F8F8000368D3F810C06A4679
:100BC0005146E047B0F5003F76D10AE0002004E04E
:100BD000215C0AF800100098401C00900098A84280
:100BE000F6D34FF0000C4749474A484B01AC0098F8
:100BF000844558D2D3E9007001ADC5E90070107882
:100C000000281ABF042086464FF0000E085854F8FA
:100C10000E5028443E4D05600127D0F800E0876063
:100C2000019D4F681AF80C007D408EEA050585F09D
:100C3000040E65680F687D4085F0FC05754485F0FD
:100C4000A30568400AF80C000CF1010CCFE7D3E9CA
:100C5000004501A8C0E9004510782E4D002814BFBA
:100C60004FF0040E4FF0000E01A8744651F80EE04C
:100C70000459A6440127CEF80050DEF80040CEF813
:100C800008704D68019F40687D406C400D68684069
:100C900084F0040480F0FC00041984F057040AF87E
:100CA0000C400CF1010CCC45D1D3D8F8F800016808
:100CB0004A689047B0F5003F0AD1D8F8F8000368B9
:100CC000D3F80C804A465146C047B0F5003F01D0EA
:100CD000114811E0002006E05AF8201081F06A3136
:100CE0004AF82010401CB0EB990FF5D3B06840F0E3
:100CF0000100B0604FF4403004B0BDE8F08700BFA1
:100D000002000300906F0108A00A00202C0F0008C9
:100D1000ADBE4ED70DBE75A10100030038B50C461F
:100D2000017A1546CA0702D500F014F908B9084837
:100D300032BDD0F8F80003682146DC682A46A04797
:100D4000B0F5003F01D0034832BD4FF4403032BD12
:100D500002000300010003002DE9F84191B00546AF
:100D60000E461746402101A814F08DF9297AC807CC
:100D700004D5284600F0EEF8040002D1DFF8A48084
:100D80004BE0D4F8F800DFF8A0800368D3F810C077
:100D90006A4601A9E047B0F5003F3ED1D4F8F8001B
:100DA00001684A689047B0F5003F36D1D4F87C110D
:100DB0008A6820469047D4F8F830024618461B68E7
:100DC000D3F80CC004F1FC01E047B0F5003F24D19A
:100DD000D4F87C0141688847D4F8F83002461846B8
:100DE0001B68D3F80CC001A9E047B0F5003F14D14F
:100DF000D4F8F8000268696893689847B0F5003F36
:100E00000BD1D4F8F80003681C693A463146A04774
:100E1000B0F5003F08BF4FF44038404612B0BDE87F
:100E2000F08100BF02000300010003002DE9F8413A
:100E3000A5B0074688461646402115A814F023F9A8
:100E400000220492402105A814F01DF9387AC10748
:100E50005ED5384600F07EF8050059D0D5F8F80088
:100E60002D4C0368D3F810C06A4605A9E047B0F5D9
:100E7000003F3CD1D5F8F80001684A689047B0F5CA
:100E8000003F34D1D5F87C118A6828469047D5F8C0
:100E9000F830024618461B68D3F80CC005F1FC0177
:100EA000E047B0F5003F22D1D5F87C014168884782
:100EB000D5F8F830024618461B68D3F80CC005A9CF
:100EC000E047B0F5003F12D1D5F8F8000268796824
:100ED00093689847B0F5003F09D1D5F8F80003684A
:100EE0001D6904AA15A9A847B0F5003F01D0204606
:100EF0000FE00A4B0A490B4A0396029101924046C1
:100F00001C68049B009415AA796800F0E5F900E0DC
:100F1000054826B0BDE8F08101000300986F010884
:100F2000936E030026C703000200030004B0010112
:100F300000170145E90A0008090B00082D0B0008FD
:100F4000BD030008550B00081D0D0008590D0008D1
:100F50002D0E00080168024A914218BF0020704718
:100F6000340F000810B5040008BF002404D0034863
:100F70002060204609688847204610BD340F0008CD
:100F800020225C3014F07DB8F0B58468A3080022FC
:100F900004F0030407E000F15C0555F8226035BA5F
:100FA00041F82250521C9A42F5D300220BE000F186
:100FB0005C0502EB830755F82360D500C5F11805E1
:100FC000EE40CE55521CA242F1D3F0BD30B5C468FC
:100FD00003690022E31AD5188C5C0544521C082AC8
:100FE0002C77F8D330BD0360C1600261704738B51B
:100FF000044615460022626023685A689047002024
:101000006061A061A5604FF4003032BD81604FF493
:10101000003070472DE9F84304462079D4F80C805D
:10102000450748BF244845D466691D46A8F101001C
:1010300000EAD60306EBC506B6EBC50F666102D221
:10104000A669761CA6611746A66906EB5576A661C9
:101050000E46E918884225D2A8EB03094A463146D4
:10106000F81814F00EF82268136839460FE042466B
:10107000384614F006F823681A6839462046904727
:1010800007E0311811F00300F1D1226813682046FF
:101090009847484600EB0809A9F10101A942F0D39D
:1010A000002300E000202A1A3118F81813F0E9FF95
:1010B0004FF40030BDE8F283040002002DE9FC4F3C
:1010C000024685B0D0681369DFF86CC1DFF86C8127
:1010D000A0EB030A506840F004005060002703A80A
:1010E00002900DF10C0ED8E9003403A8544DC0E96C
:1010F00000342878534D00280CBF00230423994660
:101100005CF803305EF80940234401261D601C682A
:101110009E60DCF80430039DDCF80090DEF804608B
:101120005D406540484C654089EA0606474C66408C
:101130007519474C6540D8E9006B03AC0028C4E939
:10114000006B0EBF002404200424029E5CF8000003
:10115000345920183F4C04600126046886600398C7
:10116000029E43406340384C7068634089EA000047
:10117000364C6040034438484340280018BF0120E3
:101180005B1E9B41042F2CBFC0B2D80F02F1140389
:1011900053F8200007F00303C3F10303DB00D8403A
:1011A0000DF807007F1C082F9DD315460C466A6971
:1011B000AB69E868D20842EA4372401E00EA0207BF
:1011C000002302409B420AD8524508D28020E055B5
:1011D0007F1C574516D2AAEB0701E01910E08020CA
:1011E000E05500E0E355E8687F1C8742FAD32A689F
:1011F000136828469847BAF1000F03D0514620469D
:1012000013F041FF2A68069E059F936869462846A9
:1012100098472A68D2F8009021462846C8472B688C
:10122000DA683946284690470EB1A86830604FF416
:10123000003007B0BDE8F08F906F01085C12000825
:10124000A00A00205FC5109304850012FC68017A93
:10125000C0F524FF24AF33D426AF698B04B001015D
:1012600000170145F8B501240094002300240DE087
:10127000009D065D0F5D7E40F643761CF60F86F0FE
:10128000010635400095641C009DEB189442EFD395
:101290001846F2BDF8B5002301240094002A11E09D
:1012A000009C85188F1815F8016C17F8015C6E40CA
:1012B000F643761CF60F86F0010634400094009C3D
:1012C000E318521EECD11846F2BD0000651200086A
:1012D00095120008010000002DE9F84F1D46DDF8C9
:1012E00028900B9F0D9C4FF0FF3300930E469246C3
:1012F000D9F800B0804632465146D847834664B399
:10130000D9F8043032465146404698476FEA0B02FE
:10131000521C42EA0B0200996FEAD2735B1C19401F
:10132000C2430091521C024300996FEAD2735B1CC6
:101330001940009186F05531484087EA000181F05C
:101340005531216080F05531C943491C0843009A4A
:101350006FEAD070401C82430092D9F8080001283F
:1013600009D17540E943491C0D4300986FEAD572D5
:10137000521C90430AE0F11C85EA9102D243521CB0
:10138000154300986FEAD5735B1C984386F0AA3624
:10139000009086EA0B0686F0AA33F243DB430C98F2
:1013A000C2F3C0725B1C42EAD3720099D243521C52
:1013B00091430091774000998843009987F0AA37BC
:1013C0000F403843BDE8F28F00000000000000002D
:1013D00001F0FF01102A2BDB10F0070F08D010F8E6
:1013E000013B013A8B422DD010F0070F42B3F6D1EA
:1013F000F0B441EA012141EA014122F007047FF003
:1014000000070023F0E80256083C85EA010586EA59
:10141000010685FA47F5A3FA87F586FA47F6A5FA95
:1014200087F68EB9EED1F0BC01F0FF0102F00702A1
:1014300032B110F8013B013A83EA010313B1F8D14C
:101440000020704701387047002D06BF354603382D
:10145000073815F0010F07D1013015F4807F02BF66
:10146000013015F4C03F0130F0BC0138704700BFB7
:10147000034613F8012B002AFBD1181A01387047D4
:1014800081F0004102E000BF83F0004330B54FEA35
:1014900041044FEA430594EA050F08BF90EA020FA2
:1014A0001FBF54EA000C55EA020C7FEA645C7FEA35
:1014B000655C00F0E2804FEA5454D4EB5555B8BF58
:1014C0006D420CDD2C4480EA020281EA030382EAC9
:1014D000000083EA010180EA020281EA0303362D5B
:1014E00088BF30BD11F0004F4FEA01314FF4801C2E
:1014F0004CEA113102D0404261EB410113F0004F40
:101500004FEA03334CEA133302D0524263EB4303F6
:1015100094EA050F00F0A780A4F10104D5F1200E94
:101520000DDB02FA0EFC22FA05F2801841F10001EF
:1015300003FA0EF2801843FA05F359410EE0A5F1C3
:1015400020050EF1200E012A03FA0EFC28BF4CF0F4
:10155000020C43FA05F3C01851EBE37101F00045AA
:1015600007D54FF0000EDCF1000C7EEB00006EEBB7
:101570000101B1F5801F1BD3B1F5001F0CD3490841
:101580005FEA30004FEA3C0C04F101044FEA445298
:1015900012F5800F80F09A80BCF1004F08BF5FEA1F
:1015A000500C50F1000041EB045141EA050130BDFF
:1015B0005FEA4C0C404141EB0101013C28BFB1F511
:1015C000801FE9D291F0000F04BF01460020B1FA5C
:1015D00081F308BF2033A3F10B03B3F120020CDA2F
:1015E0000C3208DD02F1140CC2F10C0201FA0CF00D
:1015F00021FA02F10CE002F11402D8BFC2F1200C72
:1016000001FA02F120FA0CFCDCBF41EA0C01904027
:10161000E41AA2BF01EB0451294330BD6FEA040470
:101620001F3C1CDA0C340EDC04F11404C4F120025B
:1016300020FA04F001FA02F340EA030021FA04F36D
:1016400045EA030130BDC4F10C04C4F1200220FAC4
:1016500002F001FA04F340EA0300294630BD21FA02
:1016600004F0294630BD94F0000F83F4801306BFC8
:1016700081F480110134013D4EE77FEA645C18BFBC
:101680007FEA655C29D094EA050F08BF90EA020F53
:1016900005D054EA000C04BF1946104630BD91EA4B
:1016A000030F1EBF0021002030BD5FEA545C05D14E
:1016B0004000494128BF41F0004130BD14F580048D
:1016C0003CBF01F5801130BD01F0004545F0FE4101
:1016D00041F470014FF0000030BD7FEA645C1ABF36
:1016E000194610467FEA655C1CBF0B46024650EA6D
:1016F000013406BF52EA033591EA030F41F4002199
:1017000030BD00BF90F0000F04BF0021704730B51E
:101710004FF4806404F132044FF000054FF00001F3
:1017200050E700BF90F0000F04BF0021704730B5B4
:101730004FF4806404F1320410F0004548BF404289
:101740004FF000013EE700BF42004FEAE2014FEADE
:1017500031014FEA02701FBF12F07F4393F07F4FB9
:1017600081F06051704732F07F4208BF704793F0BC
:101770007F4F04BF41F40021704730B54FF46074CF
:1017800001F0004521F000411CE700BF50EA0102D2
:1017900008BF704730B54FF000050AE050EA01027B
:1017A00008BF704730B511F0004502D5404261EBEB
:1017B00041014FF4806404F132045FEA915C3FF42C
:1017C000D8AE4FF003025FEADC0C18BF03325FEAC9
:1017D000DC0C18BF033202EBDC02C2F1200300FA7A
:1017E00003FC20FA02F001FA03FE40EA0E0021FA9F
:1017F00002F11444BDE600BF70B54FF0FF0C4CF48D
:10180000E06C1CEA11541DBF1CEA135594EA0C0F3E
:1018100095EA0C0F00F0DEF82C4481EA030621EA79
:101820004C5123EA4C5350EA013518BF52EA0335B4
:1018300041F4801143F4801338D0A0FB02CE4FF066
:101840000005E1FB02E506F00042E0FB03E54FF096
:101850000006E1FB03569CF0000F18BF4EF0010E8E
:10186000A4F1FF04B6F5007F64F5407404D25FEA8A
:101870004E0E6D4146EB060642EAC62141EA55513D
:101880004FEAC52040EA5E504FEACE2EB4F1FD0C7F
:1018900088BFBCF5E06F1ED8BEF1004F08BF5FEAFD
:1018A000500E50F1000041EB045170BD06F00046AF
:1018B00046EA010140EA020081EA0301B4EB5C045C
:1018C000C2BFD4EB0C0541EA045170BD41F4801154
:1018D0004FF0000E013C00F3AB8014F1360FDEBF79
:1018E000002001F0004170BDC4F10004203C35DA55
:1018F0000C341BDC04F11404C4F1200500FA05F3D8
:1019000020FA04F001FA05F240EA020001F0004278
:1019100021F0004110EBD37021FA04F642EB0601EE
:101920005EEA430E08BF20EAD37070BDC4F10C0418
:10193000C4F1200500FA04F320FA05F001FA04F2DC
:1019400040EA020001F0004110EBD37041F10001C8
:101950005EEA430E08BF20EAD37070BDC4F12005D3
:1019600000FA05F24EEA020E20FA04F301FA05F23B
:1019700043EA020321FA04F001F0004121FA04F2E3
:1019800020EA020000EBD3705EEA430E08BF20EAB3
:10199000D37070BD94F0000F0FD101F000464000ED
:1019A00041EB010111F4801F08BF013CF7D041EA6F
:1019B000060195F0000F18BF704703F00046520073
:1019C00043EB030313F4801F08BF013DF7D043EA44
:1019D0000603704794EA0C0F0CEA135518BF95EAFA
:1019E0000C0F0CD050EA410618BF52EA4306D1D181
:1019F00081EA030101F000414FF0000070BD50EAA0
:101A0000410606BF1046194652EA430619D094EA29
:101A10000C0F02D150EA013613D195EA0C0F05D113
:101A200052EA03361CBF104619460AD181EA030167
:101A300001F0004141F0FE4141F470014FF000001F
:101A400070BD41F0FE4141F4780170BD70B54FF0BA
:101A5000FF0C4CF4E06C1CEA11541DBF1CEA13553A
:101A600094EA0C0F95EA0C0F00F0A7F8A4EB05041C
:101A700081EA030E52EA03354FEA013100F0888013
:101A80004FEA03334FF0805545EA131343EA1263DC
:101A90004FEA022245EA111545EA10654FEA002691
:101AA0000EF000419D4208BF964244F1FD0404F54A
:101AB000407402D25B084FEA3202B61A65EB0305A6
:101AC0005B084FEA32024FF480104FF4002CB6EB63
:101AD000020E75EB030E22BFB61A754640EA0C00E3
:101AE0005B084FEA3202B6EB020E75EB030E22BF23
:101AF000B61A754640EA5C005B084FEA3202B6EB64
:101B0000020E75EB030E22BFB61A754640EA9C0022
:101B10005B084FEA3202B6EB020E75EB030E22BFF2
:101B2000B61A754640EADC0055EA060E18D04FEAB0
:101B3000051545EA16754FEA06164FEAC30343EA50
:101B400052734FEAC2025FEA1C1CC0D111F4801F1D
:101B50000BD141EA00014FF000004FF0004CB6E716
:101B600011F4801F04BF01430020B4F1FD0C88BFB5
:101B7000BCF5E06F3FF6AFAEB5EB030C04BFB6EBC0
:101B8000020C5FEA500C50F1000041EB045170BDB3
:101B90000EF0004E4EEA113114EB5C04C2BFD4EBE0
:101BA0000C0541EA045170BD41F480114FF0000E64
:101BB000013C90E645EA060E8DE60CEA135594EAE0
:101BC0000C0F08BF95EA0C0F3FF43BAF94EA0C0FE3
:101BD0000AD150EA01347FF434AF95EA0C0F7FF458
:101BE00025AF104619462CE795EA0C0F06D152EAAC
:101BF00003353FF4FDAE1046194622E750EA410690
:101C000018BF52EA43067FF4C5AE50EA41047FF4A0
:101C10000DAF52EA43057FF4EBAE12E74FF0FF3C05
:101C200006E000BF4FF0010C02E000BF4FF0010CD6
:101C30004DF804CD4FEA410C7FEA6C5C4FEA430C4F
:101C400018BF7FEA6C5C1BD001B050EA410C0CBF9E
:101C500052EA430C91EA030F02BF90EA020F002000
:101C6000704710F1000F91EA030F58BF994208BF67
:101C700090422CBFD8176FEAE37040F00100704724
:101C80004FEA410C7FEA6C5C02D150EA013C07D17B
:101C90004FEA430C7FEA6C5CD6D152EA033CD3D0C6
:101CA0005DF8040B704700BF8446104662468C46C0
:101CB0001946634600E000BF01B5FFF7B7FF0028F3
:101CC00048BF10F1000F01BD4DF808EDFFF7F4FF1C
:101CD0000CBF012000205DF808FB00BF4DF808EDA7
:101CE000FFF7EAFF34BF012000205DF808FB00BFCA
:101CF0004DF808EDFFF7E0FF94BF012000205DF8EC
:101D000008FB00BF4DF808EDFFF7CEFF94BF0120A0
:101D100000205DF808FB00BF4DF808EDFFF7C4FF99
:101D200034BF012000205DF808FB00BF4FEA410CE2
:101D30007FEA6C5C02D150EA013C0AD14FEA430CC5
:101D40007FEA6C5C02D152EA033C02D14FF0000002
:101D500070474FF0010070474FEA410212F5001240
:101D600015D211D56FF47873B3EB625212D94FEAE2
:101D7000C12343F0004343EA505311F0004F23FACC
:101D800002F018BF404270474FF00000704750EA21
:101D9000013005D111F0004008BF6FF000407047DE
:101DA0004FF00000704700BF80F0004002E000BF2D
:101DB00081F0004142001FBF5FEA410392EA030F36
:101DC0007FEA226C7FEA236C6AD04FEA1262D2EB80
:101DD0001363C1BFD218414048404140B8BF5B4285
:101DE000192B88BF704710F0004F40F4000020F01E
:101DF0007F4018BF404211F0004F41F4000121F034
:101E00007F4118BF494292EA030F3FD0A2F101027D
:101E100041FA03FC10EB0C00C3F1200301FA03F1BB
:101E200000F0004302D5494260EB4000B0F5000FDE
:101E300013D3B0F1807F06D340084FEA310102F19D
:101E40000102FE2A51D2B1F1004F40EBC25008BF4F
:101E500020F0010040EA03007047490040EB000019
:101E6000013A28BFB0F5000FEDD2B0FA80FCACF11A
:101E7000080CB2EB0C0200FA0CF0AABF00EBC25047
:101E800052421843BCBFD0401843704792F0000F35
:101E900081F4000106BF80F400000132013BB5E788
:101EA0004FEA41037FEA226C18BF7FEA236C21D0FE
:101EB00092EA030F04D092F0000F08BF0846704763
:101EC00090EA010F1CBF0020704712F07F4F04D131
:101ED000400028BF40F00040704712F100723CBF44
:101EE00000F50000704700F0004343F0FE4040F46E
:101EF000000070477FEA226216BF08467FEA23632C
:101F00000146420206BF5FEA412390EA010F40F416
:101F1000800070474FF0000304E000BF10F0004362
:101F200048BF40425FEA000C08BF704743F0964349
:101F300001464FF000001CE050EA010208BF704764
:101F40004FF000030AE000BF50EA010208BF7047EB
:101F500011F0004302D5404261EB41015FEA010C00
:101F600002BF84460146002043F0B64308BFA3F1F8
:101F70008053A3F50003BCFA8CF2083AA3EBC253DA
:101F800010DB01FA02FC634400FA02FCC2F12002F9
:101F9000BCF1004F20FA02F243EB020008BF20F030
:101FA0000100704702F1200201FA02FCC2F1200296
:101FB00050EA4C0021FA02F243EB020008BF20EA8B
:101FC000DC7070474FEA4002B2F1FE4F0FD34FF082
:101FD0009E03B3EB12620DD94FEA002343F0004396
:101FE00010F0004F23FA02F018BF404270474FF044
:101FF0000000704712F1610F01D1420205D110F0CB
:10200000004008BF6FF0004070474FF0000070477D
:1020100053B94AB9002908BF00281CBF4FF0FF314F
:102020004FF0FF3000F070B9ADF1080C6DE904CE4F
:1020300000F006F8DDF804E0DDE9022304B07047A3
:102040002DE9F047089E0D4604460F46002B4AD165
:102050008A42944665D9B2FA82F343B102FA03FC8C
:10206000C3F120029F4020FA02F217439C404FEA3E
:102070001C4E1FFA8CF5B7FBFEF1220C0EFB1177FC
:1020800042EA074201FB05F090420AD91CEB02022A
:1020900001F1FF3780F01B81904240F21881023934
:1020A0006244121AA4B2B2FBFEF00EFB102244EA04
:1020B000024400FB05F5A5420AD91CEB040400F11B
:1020C000FF3280F00681A54240F203816444023869
:1020D00040EA0140641B00211EB1DC400023C6E938
:1020E0000043BDE8F0878B4208D9002E00F0EC8059
:1020F0000021C6E900050846BDE8F087B3FA83F180
:10210000002949D1AB4202D3824200F2F780841AFF
:1021100065EB030201201746002EE2D0C6E9004716
:10212000DFE702B9FFDEB2FA82F3002B40F08F80C6
:102130008A1A4FEA1C471FFA8CFE0121B2FBF7F501
:1021400007FB1520220C42EA00420EFB05F09042EC
:1021500008D91CEB020205F1FF3802D2904200F2CE
:10216000CA804546121AA4B2B2FBF7F007FB102250
:1021700044EA02440EFB00FEA64508D91CEB040409
:1021800000F1FF3202D2A64500F2BA801046A4EB5D
:102190000E0440EA05409FE7C1F120078B4022FA78
:1021A00007FC4CEA030C05FA01F420FA07F3FD40A2
:1021B000234300FA01F94FEA1C401FFA8CFEB5FBDD
:1021C000F0F81C0C00FB185544EA054408FB0EF51A
:1021D000A54202FA01F20BD91CEB040408F1FF3A04
:1021E00080F08780A54240F28480A8F10208644410
:1021F000641B9DB2B4FBF0F300FB134445EA0444B6
:1022000003FB0EFEA64508D91CEB040403F1FF30C6
:102210006BD2A64569D9023B644443EA0840A0FB5F
:102220000283A4EB0E049C42C6461D4655D352D0F1
:1022300056B1B9EB0E0364EB050404FA07F7CB4083
:10224000CC401F43C6E900740021BDE8F087C3F10C
:10225000200102FA03FC20FA01F225FA01F19D4067
:102260002A434FEA1C471FFA8CFEB1FBF7F007FB2D
:102270001015110C41EA054100FB0EF58D4204FAE0
:1022800003F408D91CEB010100F1FF382FD28D4275
:102290002DD902386144491B92B2B1FBF7F507FB17
:1022A000151142EA014205FB0EF1914208D91CEBDF
:1022B000020205F1FF3816D2914214D9023D624460
:1022C000521A45EA004139E73146304609E73946B6
:1022D000E7E61046FCE6C145AAD2B8EB020E63EB76
:1022E0000C050138A4E74546EAE7034695E7404672
:1022F000D1E7D0467CE7023D624433E708460BE76E
:102300006444023843E700BF704700BF1348144AD3
:1023100008B54FF00043C0E90023042200234261C6
:102320000122C2614FF4805107220383C0E90233C6
:10233000C0E90933C0E90C120361837680F82030CC
:1023400080F82C30826380F83C30C36404F0E8FFEE
:1023500018B1BDE8084000F00BBC08BDA40A00207D
:10236000002401400268084B9A4282B00AD14FF023
:10237000B0431A6E42F400721A661B6E03F40073C7
:102380000193019B02B07047002401400268054B95
:102390009A4201BF4FF0B042136E23F400731366EC
:1023A000704700BF0024014030B585B000240546C9
:1023B000CDE901440394FFF7A9FF144805F048FB59
:1023C00008B100F0D5FB1148039401A9CDE90154EF
:1023D00005F004F908B100F0CBFB0C4805F062FAF7
:1023E00008B100F0C5FB4FF0FF31084805F098F840
:1023F000064805F00FFB054805F0ECF804460348D5
:1024000005F0B2FA204605B030BD00BFA40A002096
:10241000014B024A1A607047A40A002000240140C0
:1024200008B50948FFF7C0FF68B1084BB3F8AA30F8
:102430004FF6FF72934216BF40F6E442044B5343FB
:10244000B3FBF0F398B208BD002000B40075FF1F85
:10245000D8084C0013B50023ADF80630FFF7E0FFB5
:1024600004461948FFF7A0FF184BB3F8C820B3F88B
:10247000A8108A4204FB00F018D040F6E443B0FBF9
:10248000F3F364205B1A4343521A93FBF2F31E33B7
:102490001BB2ADF80630BDF806305BB21B02ADF8DA
:1024A0000630BDF8060000B202B010BD4FF47A72DB
:1024B00040F6FF73B0FBF3F35343A3F53923A3F5C1
:1024C0000C6340F6C412E0E7001000B00075FF1F77
:1024D0004FF0B04382B09A6A22F480529A629A6CAA
:1024E00042F480529A649B6C03F480530193019BE5
:1024F000002002B070474FF0B04382B09A6C0243A4
:102500009A649B6C03400193019B02B0704708B52D
:102510000420FFF7F0FF0120FFF7EDFF0220FFF797
:10252000EAFF002211460B2005F030FB0B2005F0DE
:102530005FFB002211460C2005F028FB0C2005F063
:1025400057FB002211460D2005F020FB0D2005F061
:102550004FFB002211460E2005F018FB0E2005F05F
:1025600047FB002211460F2005F010FB0F2005F05D
:102570003FFB00221146112005F008FB112005F059
:1025800037FB00223620114605F000FBBDE808406D
:10259000362005F02DBB000008B505F071FD10B127
:1025A0006FF0040008BD064B9A6942F040429A6100
:1025B0004CF2FA321A6105F075FD0028F2D0EFE70F
:1025C00000400058F0B585B000230C460093064645
:1025D000A8B3FFF7E1FF054670BB05F051FD88BBCE
:1025E0001A481B4A02230193D0F8E01506F17843FC
:1025F00002EA8121B3FBF1F701FB1733DB0A0293F7
:10260000D0F8E00504F178410139314402EA802232
:10261000B1FBF2F002FB1011C3EBD1230133694689
:1026200001A8039305F0BEFD20B102280CBF0125CF
:102630006FF0010505F036FD284605B0F0BD6FF0DE
:102640000505F9E76FF00405F6E700BF0070FF1F0E
:1026500000FCFF03014B186000207047080B0020AE
:102660002DE9F04F89B0B0F1006F06460F46009299
:10267000C0F0C580DFF89881664DD8F8E03505EAEE
:10268000832303F10063013B984200F2B8800028E5
:1026900000F0B880002900F0B58040EA02035B0733
:1026A00040F0B080FFF778FF0446A0BB05F0E8FCDF
:1026B000002840F0AA80D8F8E01506F1784205EA33
:1026C0008121B2FBF1F301FB1322009B03F178435C
:1026D000013B3344B3FBF1F001FB1033DB0A013360
:1026E0004FEAD22AA3EBD222012A039388BFC6F372
:1026F0000A050AF58038C6F1080398BF009D0693C5
:1027000088BFC5F500654FEAC828B346039B9A45C4
:1027100005D305F0C7FC204609B0BDE8F08FA6F14F
:102720000803069A1A44954219D804950197CDF8E2
:1027300014B04FF00009059B09EB0301049B994578
:102740003ED3009BAB442F445D1BB5F5006F28BF03
:102750004FF400650AF1010A08F50068D6E753F85E
:10276000081F5A68B2F1FF3F08BFB1F1FF3FD8D050
:10277000294B186810B96FF00504CAE7B8F1000FCB
:1027800004D04FF40062414611F05CFADFF8889003
:10279000D9F80030CBF30A0039461844AAB211F038
:1027A00051FA4FF400614046FFF70CFF08BBD9F81F
:1027B000003001934FF40063CDF814800493B8E720
:1027C000019B07914B4402930120D3E9002305F0BC
:1027D000A3FC88B90799019BD1E9000259F80310BD
:1027E000029B5B689A4208BF884205D109F108093B
:1027F000A1E76FF001048CE76FF0030489E74FF065
:10280000FF3488E76FF0050485E76FF0040482E782
:102810000070FF1F00FCFF03080B0020B1F1006FE8
:1028200070B511D30B4BD3F8E0650B4B03EA86234D
:1028300003F10063013B994206D840B139B192B22D
:1028400011F000FA002070BD4FF0FF30FBE76FF091
:102850000500F8E70070FF1F00FCFF03B0F1006FF8
:1028600010B40DD3084BD3F8E045084B03EA84239A
:1028700003F10063013B984202D810BCFFF7A2BEEF
:102880004FF0FF3010BC70470070FF1F00FCFF03CB
:102890004FF0B04382B0DA6C0243DA64DB6C034081
:1028A0000193019B02B0704770B586B014220021DD
:1028B00001A812F05EFB0120FFF7EAFF0220FFF7FC
:1028C000E7FF0420FFF7E4FF4FF4007101224FF00F
:1028D000904005F0DBFD012502234FF4041401A90B
:1028E0004FF09040CDE90134224E039505F0A8FC4D
:1028F0004FF4441301A94FF09040CDE90235019502
:1029000005F09EFC2023CDE9013401A900243046C6
:10291000039405F095FC4FF4007301A94FF090402B
:10292000CDE90135CDE9035405F08AFC04230DEB14
:1029300003013046CDE90135CDE9034405F080FCC3
:1029400022462146062005F021F9062005F050F91F
:1029500022462146072005F019F9072005F048F91D
:1029600022462146162005F011F9162005F040F9FF
:1029700006B070BD0004004808B51248124A134B57
:10298000C0E9002300230122C0E90232C0E9043378
:10299000C0E90633036205F0EDFE08B100F0E8F887
:1029A0000848002106F066F808B100F0E1F8054893
:1029B000002106F085F818B1BDE8084000F0D8B84D
:1029C00008BD00BFCC0B0020005800405D3E302009
:1029D00070B596B005461422002103A812F0C9FA7A
:1029E0003822002108A812F0C4FA2A68304B9A4213
:1029F0005BD18023089308A84FF440230E9306F080
:102A0000BBFD08B100F0B4F84FF0B0444FF4C05033
:102A1000E36C43F00103E364E36C03F0010302930E
:102A2000029B12230026CDE903030323CDE90563AE
:102A30004FF09040042303A9079305F001FCA36D18
:102A4000DFF870C043F48003A365A36D1A4C03F450
:102A500080030193019B26620D23C4E900C3204635
:102A60008023C4E90266C4E90436C4E9066605F0B9
:102A70001FF908B100F07CF8104AEC63A562104C15
:102A80000E23C4E900231021002380222046C4E93C
:102A90000213C4E90423C4E90633236205F008F9EC
:102AA00008B100F065F8AC63A56216B070BD00BF58
:102AB00000580040440002400C0B00205800024027
:102AC0006C0B002000B59BB04822002108A812F032
:102AD00050FA1822002102A812F04BFA06F016F85C
:102AE0004FF0B0420120D2F8903023F01803C2F822
:102AF0009030D2F8003423F4C06343F40073C2F87A
:102B00000034D2F8003403F4C0630193019B242302
:102B1000089381230B930023CDE91003B02208A86A
:102B2000CDE9122306F06AF908B172B6FEE74F2329
:102B3000CDE90230CDE90400CDE90600022102A86A
:102B400006F0F6FB08B172B6FEE71BB05DF804FBB9
:102B500008B504F093FBFFF7B5FFFFF7A5FEFFF7FD
:102B6000D6FCFFF709FF00F0ECFD00F0F1FDFCE7FB
:102B700072B6FEE700B58DB02C22002101A812F03C
:102B8000F8F91748174B03601F2383604FF080420A
:102B90000023C0E90433C0E9072383614FF4807345
:102BA000436206F06FFE08B1FFF7E2FF0C4806F043
:102BB00095FF08B1FFF7DCFF4FF0005300220793A9
:102BC000074808924FF4807301A9029206920B9372
:102BD00006F0B8FE08B1FFF7CBFF0DB05DF804FBBF
:102BE000200C00200028004010B5044690B0382288
:102BF000002102A812F0BDF92268194B9A422CD18B
:102C00004FF48033029302A84FF480730F9306F0C1
:102C1000B3FC08B1FFF7ACFF4FF0B0430220D3F88C
:102C2000902042F40042C3F890209A6D42F48062F2
:102C30009A659B6D002203F4806311460193019B0A
:102C400004F0A4FF022004F0D3FF00222A20114642
:102C500004F09CFF2A2004F0CBFF10B010BD00BF91
:102C6000002800407047000008B504F01DFB044B2D
:102C70000120C3F88800BDE8084005F09FBF00BFF1
:102C80000004005804F017BB08B504F014FB00F072
:102C90008BFCFFF709FEFFF73AFCBDE80840FFF7A1
:102CA0006BBE08B504F000FBBDE808400121002020
:102CB00005F034BF70477047FEE7FEE7FEE7FEE72A
:102CC000FEE770477047704770470000014806F004
:102CD0002BBF00BF200C0020012005F0DDBB02202F
:102CE00005F0DABB70477047014805F05BB900BFDB
:102CF0000C0B0020014805F055B900BFA00C0020C6
:102D00007047FFF7F7BF7047202005F0C5BB70473D
:102D1000014807F0CDBA00BF000D0020014806F0C1
:102D200035BD00BF200C0020014807F028B900BFC6
:102D3000840C00202DE9F04389B080460020109ECD
:102D40000790894615461F46FDF772FAF0B9104CF8
:102D5000CDE90090CDE9020407AB0E48059314239A
:102D600004933A46434629460068FDF72BFB234669
:102D7000324604F1140153F8044B42F8044B8B42E1
:102D8000F9D1079B337509B0BDE8F0830120FAE75C
:102D9000580C00208C6F01081FB50E4C00233C22FC
:102DA00002A8CDE902336275237500F0B9F8042357
:102DB00003AA009412210848FFF7BCFF0749142218
:102DC000204612F0C6F8B0FA80F35B09637504B0D0
:102DD00010BD00BF6C0C0020B46F0108AE0F0020C6
:102DE000054808B50823036006F0E4FE18B1BDE805
:102DF0000840FFF7BDBE08BD840C00204FF0B04373
:102E000007B55A6E42F001025A665B6E002203F06B
:102E10000103019311463220019B04F0B7FE3220DA
:102E200003B05DF804EB04F0E3BE00000CB407B59A
:102E3000054A05AB1021019311F00EFA03B05DF8BD
:102E400004EB02B0704700BFC66F010830B585B013
:102E5000044602A80D4611F02BF8BDF90C30064AC5
:102E600000931021029B2046FFF7E0FF2046FEF76B
:102E7000FFFA288005B030BDC66F01084FF0B042A0
:102E800010B5936823F40043936011F099F80E4B4A
:102E900001241C7000F0B6F810F062FD0B4810F031
:102EA00079FD0B4B4FF400421A61002010F078FDC1
:102EB000FFF7AEFA00F012F910F06EFE2046002186
:102EC000BDE8104010F088BE900C00204D2E000888
:102ED0000040005810F096BE08B5FFF7A1FA40F682
:102EE000B83398420CD8B0F5E16F0BD3FE23A0F5B0
:102EF000E16058434FF49663B0FBF3F0C0B208BDF5
:102F0000FE20FCE70020FAE77FB5684600F0CAF82B
:102F10000198FFF757F800B207B05DF804FB000016
:102F2000194A38B5D2F88035591C044619D104F035
:102F3000C9F9054604F0D2F9054404F0C9F92B0E8D
:102F4000E3712B0CA3712B0A6371030EE370C0F3C2
:102F50000742C0F307232571C0B2A27063702070CE
:102F600038BD190AC3718171190C1B0E41710371AF
:102F7000D2F88435C370D2F88405C0F30722C0F3B9
:102F80000743000EE9E700BF0070FF1F38B5094B8B
:102F9000D3F8803503600133054609D104F092F976
:102FA000044604F095F9444004F098F944402C603C
:102FB00038BD00BF0070FF1F0121022010F0F6BDD8
:102FC0000021022010F0F2BD00207047024B18785B
:102FD00008B100F013B97047900C002082B0019046
:102FE000019802B000F0A6B94FF0B04382B0DA6C9D
:102FF00042F00202DA64DB6C03F002030193019BEE
:1030000002B070472DE9F043254C87B004F06CF90D
:1030100004F072F904F078F90123002502934FF4CB
:103020008059032301A9204604934FF400580395C7
:103030000595FFF7D9FFFFF7D7FFFFF7D5FFFFF79C
:10304000D3FFCDF8049005F0FBF801A920464FF41A
:103050000067CDF8048005F0F3F801A920464FF48D
:103060000046019705F0ECF801A92046019605F00D
:10307000E7F82A464946204605F008FA2A4641461E
:10308000204605F003FA2A463946204605F0FEF9A7
:103090002A463146204605F0F9F907B0BDE8F0832D
:1030A0000004004810B50446FFF7D4F9074BA360AD
:1030B00040F30F20FEF732FF054B064A2360064B14
:1030C0006060C4E90323002010BD00BF0000484237
:1030D00000007A440D093E00AB0305000020704754
:1030E0000120704708B511F097FF162303604FF0D9
:1030F000FF3008BD08B511F08FFF16230360FEE70F
:1031000070B50D4614460E46731B9C4201DC2046EA
:1031100070BDAFF3008006F8010BF5E770B50D4602
:1031200014460E46731B9C4201DC204670BD16F807
:10313000010B04F08BF8F5E74FF0FF3070474FF4C8
:1031400000534B60002070470120704700207047FB
:103150000B4A116810B5034609B90A491160106895
:1031600009490A4C0344091B8B4206D911F054FF4C
:103170000C2303604FF0FF3010BD1360FCE700BF6D
:10318000940C0020103000200000012000080000F6
:10319000014B1868704700BF9C0C0020032070474B
:1031A00008B501464FF47A7200238002890DFEF7BC
:1031B0002FFF08BD4FF47A73A0FB0303800A40EA97
:1031C00083507047034B98689A689042FBD1C04384
:1031D000704700BF0028004008B5FFF7F3FF014B20
:1031E000186008BD9C0C002008B5FFF7EBFF024BF0
:1031F0001B68C01A08BD00BF9C0C0020024B187849
:1032000008B1FFF7DFBF7047980C002010B5074BDF
:10321000074C0122DA654FF48071204606F07CFAF3
:103220004FF0FF332363002010BD00BF0028004093
:10323000200C002002460021014806F086BC00BF99
:10324000200C002002460121014806F07EBC00BF90
:10325000200C002010B58CB02C220021044601A8BF
:1032600011F087FEFFF7D2FF0C4B0D481B681C4482
:103270000023089306934FF00053E4430793012281
:103280004FF4807301A902940B9306F05BFB08B125
:10329000FFF76EFC00200CB010BD00BF9C0C00209E
:1032A000200C002038B50546FFF78CFF02210446AC
:1032B000074806F051FCC4F309024FF47A71A2FBEF
:1032C0000121920AA30A2A8043EA805038BD00BF38
:1032D000200C00200148002106F03EBC200C0020FC
:1032E0000148012106F038BC200C0020F8B50F4D34
:1032F0002E78CEB90E4C4FF0FF372763FFF73AFC1C
:10330000FFF784FF4FF48071204606F005FA20464F
:10331000276306F0C5FB32462046022106F015FC65
:10332000FFF75AFF01232B700020F8BD980C0020F6
:10333000200C0020014610B54FF47A720023800261
:10334000890DFEF765FE0146FFF73CFF0446FFF7D7
:1033500039FF031B8B4200D310BD00BFF7E710F00D
:1033600037BF000010B5064C0221204606F0F4FBE2
:103370000221421C2046BDE8104006F0E6BB00BF1B
:10338000200C00201648174A08B54FF4E133C0E975
:10339000002300230C22C0E90233C0E90523C0E961
:1033A0000733C0E90933036107F0B5FD08B1FFF742
:1033B000DFFB0B48002107F02AFF08B1FFF7D8FB1D
:1033C0000748002107F043FF08B1FFF7D1FB04488D
:1033D00007F0FDFE18B1BDE80840FFF7C9BB08BD06
:1033E000000D00200044004070B596B0064614223F
:1033F000002103A811F0BDFD3822002108A811F01A
:10340000B8FD3268274B9A424AD10223089308A894
:10341000254B0A9306F0B0F808B1FFF7A9FB4FF06F
:10342000B04300259A6D214C42F400329A659A6DA2
:1034300002F400320292029ADA6C42F00102DA647B
:10344000DB6C03F001030193019B0C220223CDE905
:1034500003230323CDE9055303A907234FF090402D
:10346000079304F0EDFE124925621423C4E900130A
:103470001023C4E9023520468023C4E90435C4E999
:10348000065504F015FC08B1FFF772FB2520F46720
:1034900000220221A66204F079FB252004F0A8FB9B
:1034A00016B070BD0044004004000C00A00C0020C9
:1034B0008000024002680C4B9A4210B5044612D1BB
:1034C0004FF0B0420C21936D23F4003393654FF01D
:1034D000904004F061FFE06F04F05EFCBDE8104036
:1034E000252004F093BB10BD0044004008B50A46F7
:1034F0000146024806F040FE002008BD000D0020F5
:1035000013B5114B114C18604FF40013009302AB2C
:1035100013E90600204607F0FEFD2368DA69D103AF
:10352000FCD4DA695202FCD59A68084842F4800259
:103530009A6007F036FE06490448012207F0A4FD10
:10354000002002B010BD00BF940D0020000D00202F
:103550009C0D002008B5074B1860FEF7D8FFFFF759
:1035600011FF054AD2F8803043F00063C2F8803082
:10357000002008BD980D00200008005808B54FF045
:10358000B04308489A6B42F400329A639A6B22F473
:1035900000329A63FFF78EFF0F2004F037FB002004
:1035A00008BD00BF000D002008B5074807F0B3FCB8
:1035B00008B1FFF7DDFA054804F07AFB18B1BDE861
:1035C0000840FFF7D5BA08BD000D0020A00C002070
:1035D0000268044B9A4203D1034B00201B68184732
:1035E000704700BF00440040980D002002680B4B5C
:1035F0009A4210B504460FD1094B1B682BB1D0F885
:10360000902012B907480121984720460549BDE896
:103610001040012207F038BD10BD00BF004400403B
:10362000940D00209C0D002002480122102104F07E
:103630002DBF00BF0004004802480022102104F002
:1036400025BF00BF0004004810B50A4C23780BB911
:10365000E37C6BB1FFF7A0FB0038074B18BF0120DC
:10366000400018701B78022B02BF00232370E37404
:1036700010BD00BFAE0F0020A40D002038B5114CC6
:103680002378F3B9E37CE3B90F4D2B68012B07D9FD
:103690002B68042B04D80D4A0421012000F012FAF3
:1036A0002B68042B0DD9FFF777FB0038084B18BFA8
:1036B0000120400018701B78022B02BF00232370EA
:1036C000E37438BDAE0F0020A00D0020207001086B
:1036D000A40D002008B5FFF7A7FF01F013FABDE81D
:1036E0000840FFF7A9BF022801D8FFF79DBF704728
:1036F000022801D8FFF7A0BF70470000022808B5D4
:103700001BD8012210210D4804F0C0FE3220FFF723
:1037100065FC0A480022102104F0B8FE01221021A5
:10372000064804F0B3FE3220FFF758FCBDE808401D
:1037300002480022102104F0A9BE08BD0004004880
:10374000704708B5FFF79AFBBDE8084000F060BB82
:103750004FF0FF3010F0BABA704770477047000062
:10376000014BD870704700BF5C000020014B1874FB
:10377000704700BF5C00002020B1037813B10248FD
:1037800010F0D4BC704700BFE40E002008B5022042
:10379000002110F063FABDE80840014810F0C6BCF3
:1037A000FC0E00200021012010F058BA10B5094C81
:1037B00060B12060084810F06BFC2168064810F0EA
:1037C000EFFCBDE81040044810F0B0BC42F21073AA
:1037D0002360EFE774000020FC0E002010B5094CB8
:1037E000206023680BB9084B2360084810F050FC98
:1037F0002168064810F0D4FCBDE81040034810F0E2
:1038000095BC00BF0C000020A0860100140F002012
:1038100010B5044680B190F906306BB9094810F034
:1038200037FC094BE2791A70084B1868FFF7D6FF8E
:10383000074B1868FFF7BAFFBDE8104000210220CF
:1038400010F00CBA980E0020C80E00200C000020CA
:103850007400002038B504460D4607484FF4006157
:10386000FEF7FCFF30B92A4621460348BDE8384040
:10387000FEF7F6BE38BD00BF00F003080A46014956
:10388000FEF7CCBF00F0030838B50C4810F000FC80
:1038900008F042F960B90A4C0A480125257007F082
:1038A000CDFF2078294607F01FFD044810F03EFCAC
:1038B000BDE83840044810F039BC00BFFC0E0020C1
:1038C000000000205C000020CC0E002008F0C0B9F1
:1038D00030B585B0FFF700FB044607F0FBFD054659
:1038E00080B10024384810F0D3FB384B36481968B3
:1038F000A14238BF214610F053FC334810F016FCAB
:1039000005B030BD01464FF4807010F0A7F968464D
:1039100000F0D4FF23B203EB4303FE2203EB431377
:10392000B3FBF2F32A4A0B2111702A495068097837
:10393000DBB28DF80C3001705068457050681A2465
:10394000847050680124C47050680371224B187849
:1039500040B11D700C231370536861F07F01197022
:10396000052314E01D4B1E48197811B90178002970
:10397000F6D0002101701970536802215971BDF809
:1039800000305168180A88715168CB7108231549B5
:10399000154C0978012988BF00235370637A33B12D
:1039A00007F084FD012802D1204610F071FB0F4B77
:1039B0000748D978002207F0A3FD063091D107F01F
:1039C0006FFD04468EE700BFFC0E0020740000204F
:1039D00004000020970E00202C0F0020C30F0020B1
:1039E000AD0F0020A40D0020980E00205C000020E8
:1039F00008B5104B0122002102201A7010F02EF998
:103A00000D4810F093FB0D4B1B788BB10C4B1A78C3
:103A100072B9DB7C63B90B4B1A68042A9EBF1A6823
:103A200001321A600021BDE80840102010F016B9DC
:103A300008BD00BF2C0F0020140F0020C80E00206E
:103A4000AE0F0020A00D0020044B1B78022B03D1E9
:103A50000021082010F002B9704700BF00000020CC
:103A600008B508F062F880B907F020FD01280CD1F4
:103A7000BFF34F8F0549064BCA6802F4E062134357
:103A8000CB60BFF34F8F00BFFDE708BD00ED00E046
:103A90000400FA057047704770477047022807D046
:103AA000202808D0012809D10021022010F0D6B822
:103AB00000210820FAE7024B01221A70704700BF6C
:103AC0002810002070B505460C46164607F002FD8A
:103AD0000346002834D000241A4810F0D9FA1A4BB3
:103AE00018481968A14238BF214610F059FBBDE8BB
:103AF0007040144810F01ABB4A68F05CD05401338F
:103B0000DAB29442F8D8114B0D701B78012B88BFA4
:103B100000244C700E4C637A33B107F0C7FC0128C7
:103B200002D1204610F0B4FA0A4B0B48D978002293
:103B300007F0E6FC0630CED107F0B2FC0446CBE736
:103B40000549DDE7FC0E002074000020A40D0020D4
:103B5000980E00205C00002004000020044B1B781D
:103B600023B9044A05210120FFF7ACBF704700BF0D
:103B7000A40D00202570010810B5002490B03C224F
:103B8000214601A8009411F0F4F92F4B2022DA729B
:103B900019788DF8001059788DF8011099788DF802
:103BA0000210D9788DF8031019798DF8041059791D
:103BB0008DF8051099798DF80610D9798DF80710D0
:103BC000197A8DF80810597A8DF80910997A8DF8BC
:103BD0000A108DF80B2021460DF10B025818013107
:103BE000007B02F8010F1C29F8D193F828208DF8EA
:103BF000282093F829208DF8292093F82A208DF881
:103C00002A2093F82B208DF82B2093F82C206AB1D2
:103C100093F83F2052B10DF12B0100229818013288
:103C200090F82C0001F8010F142AF7D107484FF43F
:103C30000061FEF713FE20B9044840226946FEF7F2
:103C40000FFD10B010BD00BF7800002000F8030881
:103C5000014940220FF0F6BF00F8030870B52A4D65
:103C600028796B794D2BC0B233D1C0EB00108000A6
:103C70000A2838BF0A204FF47A735843234BAC7993
:103C80001860EB794D2BE4B22BD1C4EB0414A400E3
:103C900095F82C301E4E63BB95F83F304BBB42F27B
:103CA0001070FFF783FD3068FFF798FD2B7A194AF3
:103CB0001949DBB213706B7A184ADBB21370002318
:103CC000EA1892F82C20D2B2CA540133142BF7D13F
:103CD00070BD6B79482B0ABF4FF461636B79584311
:103CE000C6E7EB79482B0ABF4FF46163EB795C437D
:103CF000CEE7FFF75BFD012C38BF01244FF47A7348
:103D00005C433460CFE700BF7800002074000020DF
:103D10000C000020C20F0020AE0F0020A40D0020D8
:103D200010B590B000213C2201A8009111F021F9BA
:103D30004022344968460FF085FF9DF800203AB9CB
:103D40009DF801001A2803D19DF8021001290ED018
:103D5000FFF712FF2C48142200210FF07DFF4FF4D3
:103D60007A70FFF73BF9FFF779FF10B010BD274BD2
:103D70001A70587099709DF80310D9709DF804104E
:103D800019719DF8051059719DF8061099719DF8EB
:103D90000710D9719DF8081019729DF80910597211
:103DA0009DF80A1099729DF80B1001F03F01D9722D
:103DB000D87AD1B288421BD89DF8282083F82820D1
:103DC0009DF8292083F829209DF82A2083F82A20AD
:103DD0009DF82B2083F82B200DF12B010022981841
:103DE000013211F8014F80F82C40142AF7D1BAE7BC
:103DF00001F140006844194410F8340C0873013292
:103E0000D6E700BF00F80308AE0F002078000020BE
:103E10001FB5002403A92046039407F069FE03A9F7
:103E2000012007F065FE384B3848009422464FF4D5
:103E3000FA7110F0CFF8364B3648009422464FF412
:103E4000FA7110F0C7F8344B3448009401224FF453
:103E5000FA7110F0BFF82046FEF7FCFB08B1FEF740
:103E600087FE2F4B009400224FF4FA612D4810F08A
:103E7000B1F82D4A002101200FF0ACFF2B4A0021A0
:103E800002200FF0A7FF2A4A002104200FF0A2FF12
:103E9000284A002108200FF09DFF00F095FB2649DD
:103EA000264807F0DBFD264807F0C8FC1B4810F049
:103EB0003DF9244B0021187807F016FA22490094A6
:103EC000224B09682248002210F084F8204810F0A4
:103ED0002DF9FFF725FF1F4A002110200FF07AFF70
:103EE0001D4A00214FF480700FF074FF1B4B1C48DB
:103EF00019681C4B0094002210F06CF8184810F060
:103F000015F904B010BD00BF993A0008E40E002076
:103F10009B3A0008B00E0020953A0008980E002049
:103F2000493A0008CC0E002035B60008D138000808
:103F3000CD38000889380008000003011000002077
:103F40005C00002000000020740000208D37000875
:103F5000FC0E00207D360008D53600080C0000203D
:103F6000140F0020F139000810B50024A2B021463A
:103F70007C2203A8029410F0FCFF53238DF8083034
:103F80004FF48D73ADF80A300123ADF804408DF87D
:103F90000C30FEF7A1FF00B200EB4000FE2300EB67
:103FA0004010B0FBF3F08DF80D0001A800F09CFC70
:103FB000072498B958238DF80E30302280211648F6
:103FC00010F0D7FF224602A9134811F05FF8124AF9
:103FD00021460120FFF776FD22B010BD8DF80E407E
:103FE0008DF80F0000F08EFD0C4B1A6812128DF840
:103FF00010201A688DF811205A6812128DF81220BC
:104000005A688DF813209A689B688DF81530121243
:104010008DF814200E24D0E72D0F0020541000201E
:1040200030B50378592B91B0044640F0E68105295C
:1040300059D84378443B162B55D8DFE813F02501B7
:104040005400150154001D01540054005400540044
:104050008800540000015400540054008D015400A5
:104060005400A40054005400540017008578482DD3
:1040700011D1B04A14210120FFF724FD41F288300C
:10408000FEF7ACFF40F6B830FEF7A8FF11B0BDE870
:104090003040FFF7E5BC532D0ED130228021A648D9
:1040A00010F067FFFFF760FF41F28830FEF796FFE0
:1040B000A14A152101207AE0432D16D1002468463B
:1040C0008DF8004007F032FB9B4A4C2313701A23F3
:1040D00093709DF80030547001204133D0701371FB
:1040E0000521FFF7EFFC11B030BD442DFBD1924C00
:1040F000592323705A236370A57000F0D0FB2C2243
:104100008021201D10F035FF0023257063700125EC
:104110001A23A370E5702571FEF7DEFE8749FE23A2
:10412000B0FBF3F04B6864229BB2B3FBF2F3A371D4
:104130004B6800EB40009BB200EB4010B3FBF2F188
:1041400002FB11336071E37122460821B2E78378E4
:10415000303BDBB2092BC6D879497A4A0B700B7811
:10416000DBB25372744A592313704D2353700B788A
:104170003033937003210120FFF7A4FC11B0BDE898
:104180003040FFF7F9BC8578482D15D16A4A56238F
:104190001370002353701A239370032318210120F6
:1041A0001371937107235171D070D371082111B02D
:1041B000BDE83040FFF786BC432D94D15E4C002112
:1041C0003C2201A8009110F0D4FE6846FFF740FDA4
:1041D0002422802104F10C0010F0CBFE9DF8003069
:1041E00063709DF80130A3709DF80230E3709DF874
:1041F000033023719DF8043063719DF80530A3717D
:104200009DF80630E3719DF8073023729DF8083061
:10421000257063729DF80B509DF80930A3729DF8CC
:104220000A30E3722A4603A9257304F10D0010F049
:104230002DFF05F10D012246C9B2012051E780781A
:1042400039280CD83038C0B2FFF74DFA3A4A2378F3
:10425000137063785370A378937003212AE711B029
:10426000BDE83040FFF77ABC80783928F7D830387D
:10427000C0B2FFF73DFAE9E780783928EFD8303847
:10428000C0B2FFF73BFAE1E78378303BDAB2092AA4
:10429000E5D8C0783038C2B2092AE0D82179A1F136
:1042A0004802D2B20B2ADAD8274D45FA02F2D507D6
:1042B000D5D40A224D2902FB030036D13C235843B2
:1042C0004FF47A735843214B1860214B1860FFF765
:1042D0006DFA194A2378137063785370A37893703A
:1042E000E378D3702379137105210120FFF7EAFBEE
:1042F000144B00221A701A225A7001229A70DA7036
:10430000A278303A02EB8201E278303A02EB4102C5
:10431000D2B21A7122795A710E4A1278D2B21A7236
:10432000074A1278D2B25A7228E74829C8D14FF406
:104330006163C4E72B7001082D0F0020541000208A
:10434000A40D002078000020DEF7FFFF740000209D
:104350000C000020C20F00208278303AD3B2092B23
:104360003FF67DAFC378303BD9B209293FF677AF2E
:104370000079A0F14801C9B20B293FF670AF624D38
:1043800045FA01F1C9073FF56AAF0A214D2801FB43
:1043900002332DD13C2253434FF47A7253435B4A8C
:1043A00013601068FFF71AFA594A2378137063787C
:1043B0005370A3789370E378D37023791371052138
:1043C0000120FFF77FFB534B00221A701A225A700C
:1043D00001229A70DA70A278303A02EB8201E27818
:1043E000303A02EB4102D2B29A712279DA7193E744
:1043F0004828D1D14FF46162CDE7502B48D1022932
:104400007FF671AE4378303B012B3FF66CAE83787C
:10441000312B7FF468AE0B2904D8FFF79FFB0021F6
:104420003B4A47E63B4D0234002214F8013FA918ED
:10443000303B0132DBB20C2A0B73F6D1FFF780F967
:10444000334B50221A211A709970002201215A70A0
:10445000D97003F8041FA9180132097B0C2A01F155
:10446000300103F8011FF6D100232B701A236B7063
:104470000123AB70EB70284B1B78DBB22B72274B00
:104480001B78DBB26B72EA72FFF776FB1121C7E78C
:10449000412B7FF428AE4378432B7FF424AE1629BA
:1044A0007FF421AE1E4D421C002312F8011FE95477
:1044B0000133142BF9D1FFF7C7F81A4B5B7D012BA1
:1044C00019D114490023EA5CC8180133D2B2142B65
:1044D00080F82C20F7D1114B00221A701B78DBB228
:1044E0004B72FFF749FB0A4A631E1534A34206D1FB
:1044F000074A1621DEE5094B02221A70F3E713F88A
:10450000011F02F8011BF1E7DEF7FFFF0C0000209E
:104510002D0F002078000020C20F0020A40D0020E5
:10452000AE0F00206C0C002037B504460D46002964
:1045300039D022480FF0FAFD2B78A3B39CB3606802
:10454000237880B3032B0DD00B2B2ED0022B2AD136
:104550006178012927D00B0625D403B0BDE830408F
:10456000FFF75EBD6378012B07D10078012802D0E8
:10457000022800D008B907F08FF800240DF10700D9
:104580008DF8074007F0D2F80D4A4C2313701A2318
:1045900093709DF80730547001204133D07013712F
:1045A0000521FFF78FFA03B030BD6378012BFAD1F4
:1045B0000378044A03F001031370F4E7B00E0020FF
:1045C0002D0F0020970E0020034B0022C3E902228A
:1045D0000122C3E900227047C40F00200048704741
:1045E000C40F00204FF0B04382B0DA6C0243DA64AB
:1045F000DB6C03400193019B02B070472DE9F04151
:1046000086B000240220154D0594FFF7EBFF04202F
:10461000FFF7E8FF124F03944FF4807601230DEB70
:104620000001CDE901632846032304934FF40058A9
:1046300003F006FE01A93846CDF8048003F000FE21
:1046400022464146384603F021FF2846224631469D
:1046500003F01CFF204606B0BDE8F08100040048CE
:1046600000080048032810B50ED8012810D868B9F2
:1046700002460B484FF4807103F008FF00220948FE
:104680004FF4005103F002FF002010BD0122F0E7BB
:10469000002203484FF4807103F0F8FE0122EEE798
:1046A00000040048000800480220704700207047BE
:1046B0000120704700280CBF0F2016207047000013
:1046C0000D48854602F0D8FD0C480D490D4A0023DF
:1046D00002E0D458C4500433C4188C42F9D30A4AB7
:1046E0000A4C002301E013600432A242FBD310F015
:1046F00099FCFEF72DFAFEE70000012000000020E3
:10470000840A0020C47E0108840A002010300020A2
:10471000FEE74FF0B04382B0DA6C42F00102DA6497
:10472000DB6C03F001030193019B02B070470000B2
:1047300030B587B0FFF7EDFF4FF4805101224FF005
:10474000904003F0A3FE01224FF400614FF090402F
:1047500003F09CFE4FF4C0551123CDE9015301A98C
:1047600001234FF09040039303F06AFD08240A25CB
:1047700000224FF480514FF0904003F087FE01205B
:10478000FEF72CFC01224FF480514FF0904003F0D3
:104790007DFE0120FEF722FC013DE9D14FF40061CE
:1047A0004FF0904003F06CFE08B9013CDFD14FF4AC
:1047B00000614FF0904003F063FE68BBFFF7A9FF74
:1047C00004240123039001A92A48CDE9014303F001
:1047D00037FD284C01220421204603F057FE2120FA
:1047E000FEF7FCFB00220421204603F04FFE2120AF
:1047F000FEF7F4FB01220421204603F047FE2120AE
:10480000FEF7ECFB20460022042103F03FFE4FF4AC
:104810002570FEF7E3FBDDE7FFF77BFF4FF0B043CA
:1048200000249A6D42F480029A659B6D03F4800324
:1048300000934FF4C052009B1223CDE901230323C0
:10484000CDE9034304230DEB03014FF090400593A2
:1048500003F0F6FC08480949094B8460C0E90013DD
:104860000123C0E90334C0E90744446103F082FF37
:1048700007B030BD00040048D40F002000580040AD
:104880001A091020FFF754BF40B94B1E5A425A4133
:104890004FF400714FF0904003F0F8BD704708B539
:1048A0000120FEF720FF6420FEF798FB00F02AF9B4
:1048B000BDE808400120FEF71BBF0000084B1A6846
:1048C0005A6802819A68428110B51A685C689968D2
:1048D00013190B440380034B01221A7010BD00BF53
:1048E00054100020AD0F002010B5044600F008F869
:1048F00010F0FF001FBFEE232370AA23637010BDCA
:104900002DE9F3470024304E304D346021462046D7
:10491000FFF7BAFF21460120FFF7B6FF214602202C
:10492000FFF7B2FF2A4F4FF05208A146012195F838
:10493000640185F86081C5F86891FFF7A5FF032041
:10494000FEF74CFB00228821284602F0E5FB0DF122
:104950000602C021284602F02DFC80BBBDF80620CF
:104960004EF6AA639A422AD14FEA440A0AF1540A3F
:104970005FFA8AFA5146284600F034F9F8B90DF189
:104980000602C021284685F860A102F013FCB0B9E8
:10499000284600F0EBFA90B9326801231A443260DD
:1049A0003A68C5F86831A34013433B600134032CD7
:1049B00005F5C875BAD1306802B0BDE8F0870021AE
:1049C000E0B2FFF761FFF1E74C100020BC000020CF
:1049D000481000202DE9F74F354C834604F5966AC0
:1049E0004FF00A094FF00E0848F2E8074FF490160E
:1049F0004FF48045D4F86821002A51D0204600F0B9
:104A0000A9FD0DF102020DF10101204600F05CFB51
:104A10000DF1030201A9204600F0A1FE002120466D
:104A200000F0E4F801220021204600F0A3F9012261
:104A30001146204600F09EF9BBF1020F0ED81D4B27
:104A40001D4A33F81B501D4B12F80B8053F82B6096
:104A50001B4A1C4B12F80B9053F82B702A4601216D
:104A6000204600F0D2F932460021204600F0CDF970
:104A70003946204600F0D4F842460021204600F096
:104A8000D1F84A460121204600F0CCF80DF102028F
:104A90000DF10101204600F017FB0122C4F87C2132
:104AA00004F5C8745445A5D103B0BDE8F08F00BF2C
:104AB000BC000020407001086070010848700108C7
:104AC000637001085470010810B50B7E9BB9D0F8D3
:104AD0007C21098912B1C0E95E1310BD084BD0F8E2
:104AE00078411A68C2F580734B4304FB02331B12F2
:104AF000C0F87831F1E70123C0F87C31EDE700BF61
:104B0000B80000202DE9F84FDFF8C0A0304DFFF7C6
:104B1000B9FEDAF800300BB12B6813B9FFF7F0FEDD
:104B200028602B682B4E0024A34234607460B4606C
:104B300049DDDFF8A480294DDFF8A4B02046FFF757
:104B400049FF88F80040D5F86831012B31D103FACC
:104B500004F90A272249284600F05CFCB0B95946FE
:104B60002846FFF7B1FF9BF818307BB9D5F87831AC
:104B700046F82430DAF8003043EA0903CAF8003076
:104B800098F8003043F0010388F800300120FEF768
:104B900025FA9BF818301BB1013F17F0FF07D9D158
:104BA000D5F8783140F6C412002B08BF134646F8FA
:104BB000243001200134FEF711FA032C05F5C875E5
:104BC000C1D198F80030BDE8F88F00BF4810002030
:104BD0005010002054100020AD0F0020BC00002019
:104BE0002C1000204A088A2102F096BA152906D80E
:104BF000044BCB40DB0702D50174002070476FF0F7
:104C0000070070470B00300010B50A460C4609211A
:104C100002F0A4FA18B9237803F00103237010BD41
:104C200001F06BBE01F053BD01F04DBEF7B500239E
:104C30000C46174601210DF1070206468DF8073094
:104C400002F08CFA0546D8B9012F9DF8073026D11D
:104C5000042C3AD8DFE804F003171A1D200043F0B3
:104C60001004A3420CD022460121304602F054FA2F
:104C7000054628B9716986F830413046FFF7D0FF04
:104C8000284603B0F0BD43F02804EAE743F00404EB
:104C9000E7E743F04004E4E743F08004E1E7042C55
:104CA00013D8DFE804F00306090C0F0003F0EF044B
:104CB000D7E703F0D704D4E703F0FB04D1E703F010
:104CC000BF04CEE703F07F04CBE76FF00305D7E71F
:104CD00013B500230C460DF1070201218DF80730B2
:104CE00002F03CFA78B99DF80730C3F30012227045
:104CF000C3F3C002A270C3F380026270C3F38012D8
:104D0000DB09E270237102B010BD37B50D460DF11D
:104D10000202F821044602F04DFA70B901AA0421FA
:104D2000204602F067FA40B9BDF802201AB1019B93
:104D3000B3FBF2F32B602B68A36103B030BD037F9C
:104D40000B700020704737B50D460DF1060220218B
:104D5000044602F02FFA28B9BDF8063023B9236AB9
:104D60002B60207703B030BDDB002B602362012372
:104D70002377F7E70529F8B504460E46154635D8DA
:104D800062B100EB810301215A6B0023701E0428DD
:104D900007D8DFE800F00E171A1D24001146012382
:104DA000F4E784F828103444E5B984F8285000204A
:104DB00007E0C2F34F224421204602F0BDF900284B
:104DC000F1D0F8BD84F82A10EDE784F82B10EAE75B
:104DD0005B00FE226021204602F0D5F9EFE71B01BF
:104DE000EF22F7E7012384F82830E0E76FF00300B3
:104DF000E7E7052996BF4018002390F82830137084
:104E000094BF00206FF00300704770B5431804464C
:104E100093F828000E46154618B904EB8106726314
:104E200070BD05291BD8DFE801F00309121416161E
:104E3000626304EB860400206563F1E7C2F34F224E
:104E40004421204602F078F90028E9D1F1E7E26335
:104E5000EFE72264EDE7C2F34F226421F1E76FF040
:104E60000300DDE737B50446154605292CD8DFE8F1
:104E700001F0030717191B1B436B2B60002021E077
:104E80000DF10602442102F095F9D8B9BDF80620CB
:104E900053029AB12B60A363012384F8293011E0F7
:104EA000C36BEAE7036CE8E70DF10602642102F048
:104EB00081F938B9BDF806305B02DEE7A36B2B60E1
:104EC00084F8290003B030BD6FF00300FAE737B56E
:104ED0000D460DF107020121044602F03FF938B9F1
:104EE0009DF8073084F83031DB092B7084F84C30A2
:104EF00003B030BD2DE9F843037C0C4601F8083BB4
:104F00000546FFF702FF40BB207304F1100128465D
:104F1000FFF719FF08BB04F11401284600F021FC3B
:104F2000D8B904F1240705F1270904F1170806464A
:104F30003A46B1B22846FFF795FF70B9013619F825
:104F4000013F08F8013F062E07F10407F0D104F1F4
:104F50003C012846FFF7BBFF08B1BDE8F883211DDF
:104F60002846BDE8F84301F030BD0000F0B500224E
:104F7000054693B0882102F0CFF84FF47A72A5F875
:104F800052214FF4C872A5F854214C4AC5F8582153
:104F900000234B4A85F8F030C5F8D4202B6202A9D3
:104FA0002846FFF7A7FF044670B9ADF8080002AE27
:104FB0000FCE05F110070FC70FCE0FC70FCE0FC7CB
:104FC00096E80F0087E80F003E4BC5F834314FF4E8
:104FD000FA730126A5F838314FF42063A5F83C3167
:104FE0003246802185F85061284602F095F8324615
:104FF0000746FF21284602F08FF80022114607439A
:10500000284602F089F83C4364B204430DF10702DC
:105010009121284602F0A2F864B29DF8073085F885
:105020003A31044332460021284602F075F864B252
:1050300004430022FF21284602F06EF864B20443C4
:1050400000228021284602F067F864B2204340B273
:10505000002488BBA1B2012228460134FFF78AFE52
:10506000062CF6D140BB044668850246042128463A
:10507000FFF780FE00BB024605212846FFF77AFEB7
:10508000D0B94FF490136B634FF48042012128464E
:10509000FFF7BBFE80B94FF40C13FF22C5E90F30B8
:1050A00085F830210121284602F036F8012385F8E1
:1050B000323108B985F8154113B0F0BD856B010098
:1050C000A470090064008403012300F079BD2DE978
:1050D000F0428EB00C460C2304AA1421054602F0BF
:1050E00005F8844600286CD19DF81A309DF81B60A5
:1050F0009DF817209DF81810A07506EB03269DF863
:105100001630206002EB03229DF81930606003EB3B
:1051100001239BB25B029DF8121023619DF81330AE
:10512000B5F8520103EB012392B252029BB2E26046
:10513000A382B0F57A7F9DF8101095F83171B6B260
:105140000AD0704300F5FA704FF47A76B0FBF6F0AF
:105150002E7F002E39D186B2002F40D0B001C0B2D0
:10516000B608E0750DF10F002681CDE90040284614
:1051700001F086FE844620BB9DF80FE084F818E01D
:1051800005F150060FCE07AF0FC796E80700E37D85
:1051900087E80700D4E90301A28AADF83020D4E9FA
:1051A0000149CDE90A01CDE9084907AC8DF8333052
:1051B0008DF834E00FCC50350FC597E8070086E82E
:1051C000070060460EB0BDE8F0822E8C5E43B2EB65
:1051D000262F4FEA262C04D157B948F6E0260020A6
:1051E000BFE780B25043A2EB0C06B0FBF6F0B2E78B
:1051F00042F2B826B2E70000F7B517460E210DF1CE
:1052000006021D460B4C064601F0D4FFBDF80630E1
:1052100004EA43433B6050B90DF106020C213046CD
:1052200001F0C8FFBDF8063004EA43442C6003B027
:10523000F0BD00BF0000FE1F73B590F8DA30013BEF
:10524000022B06460C4634D801AB6A460121FFF713
:10525000D3FF009BB3F57F0F054603D8019BB3F541
:105260007F0F23D915BB34B11349304602B0BDE8D6
:10527000704001F00FBC0422FF21304601F04CFFCA
:105280002A4604467021304601F046FF2A46044370
:10529000FF21304601F040FF64B204432A468021DA
:1052A000304601F039FF64B2044365B2284602B0CB
:1052B00070BD0025FAE700BF5F06002037B5044641
:1052C00001228021057C01F027FF0122FF212046D9
:1052D00001F022FF00221146204601F01DFF94F844
:1052E0003A219121204601F017FF0122002120469A
:1052F00001F012FF0022FF21204601F00DFF0022E5
:105300008021204601F008FF012D29D0032D37D040
:10531000002D3CD101222946204601F0FDFE01234B
:105320008DF80730A0B103B030BD01460DF1070282
:10533000204601F013FF9DF80730DB0705F101055A
:1053400008D538B9B5F5FA6FEFD16FF00600EAE786
:105350000546F0E7B5F5FA6F08BF6FF00600E2E723
:1053600018B929462046FFF767FF02220021204690
:1053700001F0D2FE0028D6D1042384F83231D2E7DE
:1053800018B901212046FFF757FF0422EEE76FF01E
:105390000700C8E738B5057C044625B1204600F073
:1053A00054FD28B138BDFFF789FF0028F6D0F9E792
:1053B000002DF7D1032384F83231F3E773B50646A5
:1053C000002501220B21304601F0A6FE00220446F2
:1053D0000B21304601F0A0FE0DF10702044313211A
:1053E000304601F0BBFE9DF8073064B2044301353E
:1053F0005B0760B2EDB205D0032D08D00028E0D0E5
:1054000002B070BD032D08BF6FF00B00F8E76FF01E
:105410000B00F5E738B50023037404460D46FFF78B
:10542000B9FF50B929462046FFF751FE28B9014679
:105430002046BDE83840FFF7C1BF38BD152970B51B
:10544000054616461C4667D10122FF2101F064FE85
:10545000002211460446284601F05EFE0022044365
:10546000FF21284601F058FE64B204430122802146
:10547000284601F051FE64B20443022285212846E9
:1054800001F04AFE64B204430422FF21284601F0E1
:1054900043FE64B204430022CD21284601F03CFEC5
:1054A00064B204431122CC21284601F035FE64B2D7
:1054B00004430722FF21284601F02EFE64B2044374
:1054C0000022BE21284601F027FE64B204430622D2
:1054D000FF21284601F020FE64B204430922CC21BA
:1054E000284601F019FE64B204430022FF21284639
:1054F00001F012FE64B204430122FF21284601F0AC
:105500000BFE64B2002204431146284601F004FE5B
:1055100064B2204340B270BD042A17D80A2101F0BA
:10552000FBFD0028F7D1231E18BF01231B01EF222A
:105530008421284601F027FE0028ECD185F8DA60A6
:1055400001462846BDE87040FFF738BF6FF00A00FB
:10555000E1E7000070B594B005464022002104A8A0
:105560000FF007FD002301212846ADF806308DF825
:1055700003308DF80430029300F0B8FC95F8142144
:1055800095F81311012A04D840F0AD80202940F28B
:10559000AC8001AA02A9284600F02DFB0446002891
:1055A00040F09E8095F85031002B40F0A280D5F855
:1055B0004C11284601F06EFA0446002840F0908015
:1055C0002346214604222846FFF738FF04460028D8
:1055D00040F086800122FF21284601F09DFD0DF15B
:1055E000060206468421284601F0E4FD22460643D1
:1055F000FF21284601F090FD76B2064374B2002CDC
:105600006ED1BDF806301B01C5F8D43004A9284678
:10561000FFF770FC0446002862D10DF10301284613
:10562000FFF7F2FA044600285AD19DF8033085F8B6
:10563000313104AE0FCE05F110040FC40FCE0FC4EC
:105640000FCE0FC496E80F0084E80F000DF103029F
:105650000121284601F082FD0446002840D19DF832
:10566000033085F83031024601462846FFF7DEFA5E
:105670000446A8BB024602212846FFF7D7FA044693
:1056800070BB0323014685F832310DF1050228462F
:1056900001F019F9044618BB9DF8053085F8E8308B
:1056A0000DF105020121284601F00DF90446B8B9B3
:1056B0009DF8053085F8E03003AA0321284600F064
:1056C00001FF044660B9039BC5F8E43003AA042136
:1056D000284600F0F7FE044610B9039BC5F8DC30FD
:1056E000204614B070BD0C2951E7284600F010F98F
:1056F00054E701495DE700BF6C05002013B50C4677
:105700000DF10702132101F029FD9DF8073013F078
:10571000180F03F0070218BF6FF00500226002B0F7
:1057200010BD13B590F8DA30042B0C460BD101A94B
:10573000FFF7E4FF019B042B01D1012300E00023CC
:10574000237002B010BD01AA142101F007FD00284A
:10575000F7D19DF80430DB07EFD42070F1E700F0BB
:105760004ABA13B50C460DF10602282101F022FDBC
:1057700078B9BDF80620C2F30B0312F4006F18BF0E
:10578000A3F580534FF0FA0214BF13FB02F3534307
:10579000236002B010BDF0B54FEAD20C4FF0FF34D9
:1057A0001C6002F00702664600278E4200D207B155
:1057B000F0BD845D664503BF1441E4B215463D4625
:1057C00014F0010704D005EBC6051D600136ECE7B7
:1057D0000135082D4FEA5404F2D1F7E7034B800955
:1057E00053F82000003818BF012070471808002027
:1057F00010B5B1EBD20F4FEAD20402F0070381BF1C
:1058000001229A40035D13438ABF03556FF03100B4
:10581000002010BD0A460623B02101F049BC0A460B
:105820000623B02101F062BC2DE9F04F85B080461F
:10583000109E0E9D01968A4693461C464FF0000925
:10584000119B994508D10023129A1660F3B16FF0AD
:10585000310005B0BDE8F08F01AB3246294658460D
:10586000FFF799FF019F7B1C0DD00F9BF818FFF7E6
:10587000B5FF504507D13A462046FFF7B9FF7E1CD9
:1058800009F10109DCE76FF03103DDE7214640460D
:10589000FFF7C0FF0028DCD102A94046FFF7BFFF99
:1058A0002544234602AAAB42D3D013F8014B12F889
:1058B000011B8C42F7D0CAE770B5C02288B00E46F3
:1058C000012190F83041054601F026FCF0B901A90C
:1058D0002846FFF79FFDC8B90122FF21284601F0A5
:1058E0001BFC98B93246B621284601F063FC68B922
:1058F0000246FF21284601F00FFC38B9224601215B
:10590000284601F009FC08B985F8304108B070BD9F
:10591000F0B50F4689B01646FF210122044601F07A
:10592000FBFB0246A8B94F21204601F0F5FB80B9E8
:105930002C224E21204601F0EFFB024648B9FF2100
:10594000204601F0E9FB20B9B422B621204601F03F
:10595000E3FB0025C4F82451A4F82851DEB93546EC
:1059600007ABB422CDE903730623CDE900320295DB
:1059700004F5927304F5957231462046FFF754FF03
:1059800030B9012384F8153184F8137184F8146157
:1059900009B0F0BD013505F1B400FFF71FFF002885
:1059A000DED12C2DF6D1DBE710B541F0010200214C
:1059B000044601F0B1FB78B9204600F046FA58B928
:1059C00001462046FFF7FAFC30B902460146204660
:1059D000BDE8104001F0A0BB10BD2DE9F74F4FF01E
:1059E000000B88461746FF21012205461E469DF8FA
:1059F00038A09DF83C908DF807B001F08DFB5A4619
:105A000004465946284601F087FB5A460443FF21C5
:105A1000284601F081FB64B2044364B2B8F1000F80
:105A200032D0BAF1000F06D00C9ACB21284601F0F3
:105A300095FB204344B2B9F1000F07D00DF10702E6
:105A4000EE21284601F08AFB204344B20122FF21C7
:105A5000284601F061FB012204430021284601F0A1
:105A60005BFB64B204430022FF21284601F054FB93
:105A700064B29DF807300D9A204323F0100340B222
:105A8000137003B0BDE8F08FBAF1000F06D03A46AC
:105A9000CB21284601F040FB204344B2B9F1000F6E
:105AA000D4D033468022EE21284601F06CFBCBE7B0
:105AB0002DE9F04387B091460022054688468DF8CF
:105AC00017201E461BB390F830710122114628465C
:105AD00001F022FB044658BB40212846FFF764FF33
:105AE000044628BBB9F1010F13D10DF11703CDE91D
:105AF0000290CDE900830246034649462846FFF757
:105B00006CFF40B10446204607B0BDE8F0831F4655
:105B1000DBE788F80000002EF5D03A460121284640
:105B200001F0FAFA04460028EDD185F83071EAE771
:105B3000002388F800302046E4E72DE9F0430546CD
:105B400087B0884691461E4623B390F830710222F2
:105B50000121284601F0E0FA044660BB01462846D0
:105B6000FFF722FF044630BBB9F1010F14D10DF14C
:105B70001703CDE90209009302460346CDF80480DD
:105B800049462846FFF729FF40B10446204607B0A2
:105B9000BDE8F0831F46DAE788F80000002EF5D054
:105BA0003A460121284601F0B7FA04460028EDD113
:105BB00085F83071EAE7002388F800302046E4E7F2
:105BC000F8B51D46164600232A4690F83071044663
:105BD000FFF76EFF70B903462A4631462046FFF7AD
:105BE000ACFF38B93A460121204601F095FA08B9D0
:105BF00084F83071F8BD2DE9F04F002393B0CDE962
:105C00000A12C0F82431A0F828310122FF21CDE981
:105C10000E33B0F83C818DF8343005468DF83530C0
:105C200001F07AFA0446002840F0E38002464F2152
:105C3000284601F071FA0446002840F0DA802C2250
:105C40004E21284601F068FA0446002840F0D18031
:105C50000246FF21284601F05FFA0446002840F082
:105C6000C880B422B621284601F056FA044600281E
:105C700040F0BF8002468021284601F04DFA0446DC
:105C8000002840F0B68003460DF135020DA92846E4
:105C9000FFF796FF0446002840F0AB800323CDE9D0
:105CA0000203B421062305F5957A05F592790EAE27
:105CB000CDE90031049601464B4652462846FFF78F
:105CC000B3FD0446002840F094800DF136012846CB
:105CD0000E9FFFF7F1FD0446002840F08A80BDF8D2
:105CE0003630434540F2AA80C5F82401A5F82801C2
:105CF00007F1B400FFF772FD08B92B2F7DD90623F9
:105D0000B4224FF0030BCDE90032CDE9027B0496BB
:105D10004B46524601212846FFF786FD002840F0F9
:105D20008B800DF1360128460E9FFFF7C5FD064614
:105D300000287CD1BDF83630434540F282800126F0
:105D40000696BDF83630434560D2A3EB080383EADC
:105D5000E372A2EBE3729DF81860099205F5927365
:105D60004FF0030B0793079B18689B881090ADF8C2
:105D700044303A460FAB06215046FFF70CFD0F9F0B
:105D80007B1C56D007F1B400FFF728FD069B984214
:105D90003CD10BF101033A4648460893FFF728FD32
:105DA000002849D149462846FFF734FD002843D151
:105DB0000DF136012846FFF77FFD00283CD1BDF8E4
:105DC0003620A2EB0803002BB8BF5B42424516D930
:105DD000099A934218D910A92846FFF71BFD079A84
:105DE0000799034610981060BDF844208A806BB173
:105DF0001C46204613B0BDE8F08F013778E7DDF888
:105E000020B009930137AEE7DDF820B00A9BC3F854
:105E100000B00B9B1E70012385F815310A9B1B688F
:105E200085F813310B9B1B7885F81431E1E70446A4
:105E3000DFE76FF03104DCE70446DAE70026B3461B
:105E40007EE70123834606937BE737B500230446AC
:105E50008DF807304FF4FA650DF107012046FFF782
:105E600060FC58B99DF80730012B07D0013D03D0E5
:105E7000204601F0E5F9EFE76FF0060003B030BD12
:105E800002464FF08043934202D8002013B9704776
:105E90009B08F8E7C11891424FEA50009CBFC01818
:105EA000521A9B08F2E773B500228321054601F0E0
:105EB00033F9044688B94FF4FA660DF107028321DD
:105EC000284601F04BF99DF807300343DBB2044646
:105ED0001BB9013EF1D16FF006040122832128464F
:105EE00001F01AF9204340B202B070BD2DE9F04F25
:105EF00090F8F06091B04FF00009072ECDE90799B6
:105F000004460F4600F0A2820122802101F004F92C
:105F100001228046FF21204601F0FEF84A4648EA69
:105F200000084946204601F0F7F84FFA88F848EA99
:105F300000080622FF21204601F0EEF84FFA88F80B
:105F400048EA00080DF115028321204601F006F908
:105F50009DF815204FFA88F848EA000842F004023C
:105F60008321204601F0D8F84FFA88F848EA000863
:105F70000722FF21204601F0CFF84FFA88F80122CE
:105F8000812148EA0008204601F0C6F84FFA88F857
:105F900048EA0008204601F053F94FFA88F848EA29
:105FA000000801228021204601F0B6F84FFA88F857
:105FB00048EA000517F0010B6DB200F01E82F207EF
:105FC00000F11E826B229421204601F0A5F8804644
:105FD0002046FFF768FF06AA48EA000890212046FD
:105FE00001F008F945EA0805069B6DB224229421C8
:105FF00005432046C3F3062AC3F3C03901F08CF8E9
:106000006DB205432046FFF74EFF6DB2054306AA69
:106010009021204601F0EEF8069B6DB21BBA2522B6
:10602000942105432046099301F076F86DB20543AB
:106030002046FFF738FF6DB2054306AA902120469F
:1060400001F0D8F8069B6DB21A0E05431B0C6DB219
:106050008DF828208DF8293017F00203029300F004
:10606000DB8016F0020840F0D780022294212046FF
:1060700001F052F801902046FFF715FF019B0DF14A
:1060800016020343902120461D4301F067F86DB2CC
:106090007B2294210543204601F03EF86DB2054372
:1060A0002046FFF700FF6DB205430DF11702902166
:1060B000204601F053F86DB2772294210543204623
:1060C00001F02AF86DB205432046FFF7ECFE6DB2F1
:1060D000054306AA9021204601F08CF8069B5A0E33
:1060E0008DF82C20C3F386428DF82D20C3F3C622F1
:1060F0008DF82E206DB2C3F30612DB0003F0780397
:10610000942105438DF82F20204678228DF81530F4
:1061100001F002F86DB205432046FFF7C4FE6DB2F0
:10612000054306AA9021204601F064F8069B9DF8DD
:10613000152002EB53728DF83020C3F386528DF890
:106140003120C3F3C6328DF83220C3F306228DF816
:1061500033206DB2C3F346029B0103F04003942148
:1061600005438DF83420204679228DF8153000F053
:10617000D3FF6DB205432046FFF795FE6DB2054390
:1061800006AA9021204601F035F8069B9DF81520BF
:1061900002EB93628DF83520C3F3C6428DF83620AA
:1061A000C3F306328DF837206DB2C3F346129B005D
:1061B00003F07C03942105438DF8382020467A2291
:1061C0008DF8153000F0A8FF6DB205432046FFF7AB
:1061D0006AFE6DB2054306AA9021204601F00AF836
:1061E000069B9DF815208DF83E8002EB93728DF88A
:1061F0003920C3F3C6526DB28DF83A20C3F306427C
:1062000005438DF83B20C3F34622C3F386036DB2EA
:106210008DF83C208DF83D3017F00403019300F019
:10622000F180730700F1EE807B229421204600F07C
:1062300073FF80462046FFF736FE07AA48EA0008AB
:106240009021204600F0D6FF45EA08084FFA88F86A
:1062500048EA00057C229421204600F05DFF6DB2E3
:1062600005432046FFF71FFE6DB2054308AA9021A3
:10627000204600F0BFFF6DB27322942105432046F3
:1062800000F04AFF6DB205432046FFF70CFE6DB2E9
:10629000054306AA9021204600F0ACFF069B6DB294
:1062A0001B0274229421054320461FFA83F800F054
:1062B00033FF6DB205432046FFF7F5FD6DB2054390
:1062C00006AA9021204600F095FF6DB29DF81B3084
:1062D000752294210543204643EA080800F01CFF7C
:1062E0006DB205432046FFF7DEFD6DB2054306AAF9
:1062F0009021204600F07EFF069B6DB21B029BB2F0
:106300007622942105432046039300F005FF6DB2E9
:1063100005432046FFF7C7FD6DB2054306AA90214D
:10632000204600F067FF6DB29DF81B20039B0543DC
:106330006DB21343002281212046039300F0ECFE4E
:1063400006220543FF21204600F0E6FE6DB205431C
:106350000DF115028321204600F000FF9DF8152065
:106360006DB2054302F0FB028321204600F0D4FE0B
:106370006DB205430122FF21204600F0CDFE6DB233
:10638000054301220021204600F0C6FE6DB2054300
:106390000022FF21204600F0BFFE6DB2054300221F
:1063A0008021204600F0B8FE6DB205436DB2039B1C
:1063B000FDB9BBF1000F29D1029AAABB019AAAB17B
:1063C000720713D4079AC4F81821089AC4F81C213C
:1063D0004FEA4822C4F820213BB1A3F5C8534FF43B
:1063E0007A7253431B095B421BB2E3603E4384F85D
:1063F000F060284611B0BDE8F08FD946DA462BE6AA
:10640000CA4629E64FF00008434693E7F007D3D485
:106410000998BDF8282084F813A184F81491C4F8D1
:106420002A01A4F82E21C7E7B107C7D49DF816208A
:1064300084F8F1209DF8172084F8F2200BA904F1CC
:10644000F30002930EF015FE029BB7E74D46D0E72E
:1064500050B10138002330F0FF019AB203F101037B
:1064600003D100EB022080B270474008F3E7C3B2CB
:10647000000A03FA00F0013070470000084B5A434D
:106480004FF47A7302F5FA724FF4FA60B2FBF0F04F
:10649000B2FBF3F203FB0100B0FBF2F0704700BF68
:1064A000002F3A00064B5A434FF47A7002F5FA7205
:1064B000B2FBF0F24A4302F5FA72B2FBF0F0704719
:1064C000002F3A002DE9FF4102294FF00005074651
:1064D00016468DF80350ADF804501CD80DF1020299
:1064E0002946FEF7A1FB044630B90DF1030246210F
:1064F000384600F033FE04469DF80300FFF7B7FF6F
:1065000081B29DF802203846FFF7CCFF306020466C
:1065100004B0BDE8F081032918D10DF1020229462B
:10652000FEF782FB0446002846D101460DF1020227
:106530003846FEF779FB044628B901AA51213846AE
:1065400000F038FE0446BDF80400D7E7042935D131
:1065500002A9FEF7BDFB9DF80B30ABB10DF10202B5
:1065600029463846FEF760FB044658B901AA512176
:10657000384600F01FFE0446BDF80400FFF777FF21
:1065800085B214B1002015E01D460DF10202012173
:106590003846FEF749FB04460028F3D10DF1060208
:1065A0007121384600F006FE0446BDF80600FFF7EC
:1065B0005EFF80B2401BA3E72846A7E728462C468B
:1065C000A4E7F0B5022985B0054616461ED80DF1A0
:1065D00005020021FEF728FB0446A0B99DF805201E
:1065E00031462846FFF74AFF83B2B3F5807F9ABF52
:1065F00000F1FF32D2B2FF22A5F8D820462128466A
:1066000000F08AFD0446204605B0F0BD03291FD1E5
:106610000DF105020021FEF707FB9DF8052031462C
:1066200004462846FFF72AFF80B2FFF711FF024613
:10663000ADF80600A5F8D800002CE4D15121284679
:1066400000F07AFD04460028DDD1C5F8E460DAE701
:10665000042939D102A9FEF73BFB9DF80B70B7B1B5
:106660000DF1050200212846FEF7DEFA0446002857
:10667000C9D10DF106025121284600F09BFD0446C8
:10668000BDF80600FFF7F3FE87B2002CBBD10DF179
:10669000050201212846FEF7C7FA04460028B2D1B8
:1066A0009DF8052031462846FFF7E8FE3844FFF7FD
:1066B000CFFE71210246284600F03EFD0446002828
:1066C000A1D1C5F8DC609EE76FF003049BE7F0B54D
:1066D00085B000238DF80330D30705460F461646D4
:1066E00005D439B9A2F10C03DAB2062A11D96FF038
:1066F0000300E6E0012921D1A2F10803DAB2062A5B
:10670000F5D8062B1AD8DFE803F03B1969198A1966
:106710009D00062B12D8DFE803F004112D112F1174
:10672000310018225721284600F0F6FC0822562195
:10673000284600F0F1FC002840F0C3807408013CBA
:10674000E4B2002F00F09180012FD0D101AA0421E2
:106750002846FFF7B7FE50B922467021284600F0C0
:10676000DBFC20B9019A04212846FFF72AFF85F8AF
:10677000E06099E03022D5E74022D3E75022D1E70C
:106780001022482100F0C8FC08224721284600F0CA
:10679000C3FC022204463221284600F0BDFC0C2234
:1067A00004433021284600F0B7FC64B204430122C0
:1067B000FF21284600F0B0FC64B2044364B23022EA
:1067C0003021284600F0A8FC00220443FF2128467F
:1067D00000F0A2FC64B2204340B2ACE7282248217A
:1067E00000F09AFC08224721284600F095FC03227D
:1067F00004463221284600F08FFC044364B209228B
:106800003021284600F088FC01220443FF2128465D
:1068100000F082FC64B2044364B22022D0E7382244
:10682000482100F079FC08224721284600F074FC3A
:10683000032204463221284600F06EFC044364B271
:106840000822DDE74822114600F066FC08224721B5
:10685000284600F061FC032204463221284600F05D
:106860005BFC044364B20722CAE702AA032128465C
:10687000FFF728FEB0B903AA02212846FFF722FE3F
:1068800080B922465021284600F046FC50B9029AB1
:1068900003212846FFF795FE20B9039A02212846D6
:1068A000FFF78FFE85F8E86058B969692846FEF75A
:1068B000B7F930B9024601230DF103012846FFF76D
:1068C0003CF905B0F0BD13B5144629B1012910D02B
:1068D0006FF0030002B010BD0DF10702502100F06F
:1068E0003DFC0028F6D19DF8073001335B00237092
:1068F000F0E70DF107027021F1E7F0B5002385B054
:106900004FF4FA62CDE9002344F61F63994206462C
:106910000F4604D86FF00305284605B0F0BD02A964
:10692000FEF7D6F905460028F6D19DF809209DF816
:10693000083013439DF80A201343A7F636341BD0C2
:106940006A4602213046FFF7BDFD00283BD19DF885
:1069500008302BB1009B03F24E239C42DAD9E41A93
:106960009DF80A3023B3009B03F2B223B4EB430F2C
:106970004FEA4302CED9A41A9DF80B305BB101AAAD
:1069800003213046FFF79EFD019B03F52573A342CB
:10699000C0D2C0B9E41A9DF80C30002BBCD0A4F2D0
:1069A000262204213046FFF70CFE77610546B3E747
:1069B0009DF80930002BDFD0009B03F525739C4226
:1069C000A8D9E41AD8E70546A6E770B54FF4FA62ED
:1069D00086B00023CDE9022340F636330B600C4627
:1069E00004A90646FEF774F90546002836D19DF83D
:1069F00011209DF8103013439DF81220134319D035
:106A000002AA02213046FFF75DFD002840D19DF823
:106A100010302BB1029B03F24E22236813442360F3
:106A20009DF81230EBB1029B03F2B222236803EB14
:106A3000420323609DF81330EBB99DF814305BB12D
:106A400001AA04213046FFF73DFD019B03F22622F7
:106A5000236813442360D8B923687361284606B0BD
:106A600070BD9DF81130002BE4D0029B03F5257218
:106A700023681344DDE703AA03213046FFF722FD14
:106A8000039B03F525722368134423600028D4D0A8
:106A90000546E3E72DE9F743002406460D46204668
:106AA00015F80480B8F1000F00D010B103B0BDE8B4
:106AB000F083671CB8F1FF0F15F8079029D1A71CC8
:106AC000EB5DB9F1030F36D8DFE809F0020B131BB9
:106AD000271D2C44E27802EB0323A6F834313C4610
:106AE000DEE7271D2C44E27802EB0323A6F83631BB
:106AF000F5E7271D2C44E27802EB0323A6F8383192
:106B0000EDE7271D2C44E27802EB0323A6F83C3185
:106B1000E5E7B8F1040F0ED802344246291901A85E
:106B20000EF0B4FA434601AA4946304604EB080782
:106B300000F0BEFAD3E76FF00300D0E773B500238F
:106B40000E4613600DF1070105461446FEF7F7F8EF
:106B500040B99DF807302BB1B38A2A6A534380337A
:106B60001B0A236002B070BD13B5CB6813601446D6
:106B700001AAFFF7E3FF18B92368019A13442360C1
:106B800002B010BDF8B5B0F85451D0F858016843C0
:106B90008030000A0E464543DDE90717144652B11E
:106BA000B60206EB5202B2FBF4F202EB420252438F
:106BB00002F50042140C069A534301F50042120CF0
:106BC00006200332B2FBF0F2C2EBC202B2F5803F04
:106BD00038BF033103F500433EBFB1FBF0F1C1EB19
:106BE000C10101F500414FEA134334BF090C1B49B1
:106BF00003FB03F338BF494303EB57030B44B3FBD9
:106C0000F7F39B03FE2205F120007F33B3FBF2F381
:106C10005C434FF47A7704F5FA748009B4FBF7F417
:106C20002401FFF72DF904F5FA74BC4228BF4FF494
:106C3000FA63064629BFB4FBF3F300205B19B4FBEB
:106C4000F7F428BFB3FBF4F0FFF71AF9099B86426B
:106C500094BF1E6018600020F8BD00BF0000F0FF68
:106C60002DE9F04F91B0CDE90723036A0E930B692C
:106C700009930546CB680B930F460FAAFFF774FFE5
:106C80000EAA39462846FFF759FF58BB0F9C95F8C6
:106C9000E0B0D5F8DC3005934FF47A7606FB04F1CA
:106CA00001F5004104910E990A910499D5F8E43058
:106CB0000693BBF1080F04F180040CBF02230323E9
:106CC00024F0FF0A090C95F8E820DFF8A081CDF840
:106CD0003CA00C9109D1079BC3F80080089BC5F824
:106CE0004081186011B0BDE8F08F06990D932846D9
:106CF000FFF7C4FB5A46059981462846FFF7BEFBBD
:106D00000D9B5B490C9A814403FB09F94FEAC929A1
:106D100040F2776309F5FA79240AB9FBF6F903FB27
:106D200009F909F5FA79B9FBF6F909FB04F404F15C
:106D30008003099C74430C40B4FBF2F44D4A1B0AD7
:106D4000944228BF1446012B38BF01230C204FF476
:106D5000167258435443FFF793F83B7E3A894FEA43
:106D6000400B002B7FD14249049B0B4003F5FA7185
:106D7000414B5A4341F25C23B2FBF3F20A9B73434B
:106D8000B3F5481F28BF4FF44813A1EB4303B1FBF1
:106D9000F6F1B3FBF6F31B02B3FBF1F63602C6F5D0
:106DA0008036564306F50046360C06F580367608E2
:106DB0007643B60B4FF44870704304F5004300F57A
:106DC00000401B0C5B43000C00FB0030FFF758F841
:106DD00003046422323341F28837B3FBF2F340F606
:106DE000B532B3FBFBF302FB0377244B9F429CBFFE
:106DF00042F21073B7FBF3F7DDE90532134403F5F4
:106E0000FA734FF47A7B4FF4FA62B3FBFBF0B3FBF7
:106E1000F2F202F5C812B2FBF0F088BF4FF47047EF
:106E2000FFF72EF8000200F5FA70B0FBFBF04043CC
:106E300007FB0700FFF724F80BFB00F0079B0B9AFA
:106E4000404528BF40461860089BC5F84001CDE981
:106E500002934FF4487300930194334651462846F9
:106E6000FFF790FE3EE74FF48036A3E7AE878F0230
:106E70000000FFFF666666009A9906000F279F24B0
:106E80002DE9F04F8BB0002711F0780FDDE914B831
:106E90000446019299468DF80E708DF80F708DF8AA
:106EA00010708DF81170ADF812700997C1F3C30A14
:106EB00000F0AF80AAF10503DBB20A2B01D86B4AC0
:106EC000D75C0DF10E0200212046FDF792FF9DF8E0
:106ED0000E500646D5B1002840F09D8009AB05AAAA
:106EE00059462046FFF7BCFE002840F09680099BDB
:106EF000ABF80A30014606AA2046FDF7B3FF069D0F
:106F000025B1059B9D422CBF0025012520B904AA6F
:106F100002212046FDF76DFF9DF8106026B3002882
:106F20007DD107AA02212046FDF79CFF88B90122E6
:106F3000FF21204600F0F0F858B90DF11202B621F9
:106F4000204600F037F920B90246FF21204600F024
:106F5000E3F8BDF81230079E5B02C4F848311EB159
:106F60009E422CBF0026012628B90DF111020321F3
:106F70002046FDF73EFF9DF8113093B1002873D1F4
:106F8000B9F1000F03D0019B1B02B3FBF9F908AA6A
:106F900003212046FDF766FF089B4B4594BF002365
:106FA000012320B9012F3CD1FF2288F8002098F856
:106FB00000200AB9ABF80A200DF10F02012120468A
:106FC0000193FDF716FF08BB9DF80E20019B002AD8
:106FD00008BF0125BAF1040F18BF9DF80F2084F8EF
:106FE0002E501ABFB2FA82F25209012284F82F20E1
:106FF0009DF81020002A9DF8112008BF0126002AC4
:1070000008BF012384F8306084F831300BB0BDE84C
:10701000F08F012755E700257EE735467CE70026FF
:10702000A9E70AF1FF32092A0AD8DFE802F00505CC
:1070300005090907090B070B0522B6E70422B4E787
:10704000012E01D10322B0E7BAF1040F01D0012BC8
:1070500001D10222A9E7012D1BBF002388F80030CF
:1070600088F800502B46A2E70023A0E766700108CD
:1070700007B502F10A03009393B20A4690F8601133
:10708000D0F85C0101F0C8FB03B05DF804FB13B558
:1070900002F10A0390F860410093D0F85C0193B2CA
:1070A0000A4644F0010101F04DFC02B010BD0000A1
:1070B0003F2BF8B50E46054611461C4611D80A4F1F
:1070C00038461A4600F8016B0DF0E0FF621C3946A5
:1070D0002846FFF7CDFF00280CBF00206FF01300FB
:1070E000F8BD6FF00300FBE76010002073B5154694
:1070F0008DF8071001220DF1070104461E46FFF727
:10710000B7FF28B9324629462046FFF7C0FF08B12D
:107110006FF0130002B070BD08B5064B19705A70BD
:1071200019460222FFF7A4FF002814BF6FF01300D6
:10713000002008BD6010002008B5074B1970110A27
:1071400059709A7019460322FFF792FF002814BF66
:107150006FF01300002008BD6010002037B5154601
:107160008DF8071001220DF107010446FFF780FF9B
:1071700028B9012229462046FFF789FF08B16FF0A0
:10718000130003B030BDF7B515460DF107020646F2
:107190000F461C46FFF7E2FF50B99DF807301D402F
:1071A00044EA0502394630468DF80720FFF7B4FF60
:1071B00003B0F0BD73B514468DF8071001220DF130
:1071C00007010646FFF754FF18B16FF0130002B035
:1071D00070BD074D022229463046FFF758FF0028B0
:1071E000F3D12A786B7803EB02232380EFE700BF0B
:1071F0006010002073B514468DF8071001220DF1C0
:1072000007010646FFF734FF18B16FF0130002B014
:1072100070BD0A4D042229463046FFF738FF00288A
:10722000F3D16B782A781B0403EB0263EA781344EA
:10723000AA7803EB02232360E9E700BF6010002077
:1072400008B50220FBF7CAFE002008BD37B5084B81
:107250000190084C187894254FF47A73012201A903
:1072600005FB004003F0D0FD019803B030BD00BF26
:10727000A0100020A41000207047000010B50320CB
:1072800000F072FC01F0AAFD064B18600F20FBF71E
:107290009BFE044618B9FBF70EFD204610BD0124E5
:1072A000FBE700BF280800204FF0E022136923F01D
:1072B0000203136170474FF0E022136943F00203A9
:1072C00013617047014BD3F8900570470070FF1FA2
:1072D000014BD3F8940570470070FF1F014BD3F8A2
:1072E000980570470070FF1F024A536823F001039E
:1072F00053607047002004E0024A536823F0020301
:1073000053607047002004E0024A536823F00403EE
:1073100053607047002004E08068C0F3800070472D
:10732000F7B5002301930446002800F0E980856D3D
:1073300025B9FBF717F8E56584F8545023689A6877
:10734000D00040F1A1809A68D10000F1B480A26D14
:1073500042F01002A265E26D42F00102E2650125F1
:107360001846FFF7D9FFA26D02F01002024340F069
:10737000C980A26D206922F4817242F00202A265E6
:107380009A68D2075DD4226BA67E94F82CC0003A8E
:1073900018BF01221703D4E902120A43217E42EAF0
:1073A0008132617E42EAC13242EA4632002842EA34
:1073B0004C02B4BF20F000414FF400113A430A439D
:1073C00094F82010012903D1002E76D142F48032A6
:1073D000616A21B1A66A01F4E07131430A43D968B8
:1073E000E66C21F4FE3121F4FF711143D96094F869
:1073F0003C206168012A01F0404C4CEA060609D1A4
:10740000D4E910273A433243A66C324342EA0C02D5
:1074100042F001061F693E4A3A4032431A6121F0A8
:107420000042B2F1804F0CD0B1F1004F09D0394E7B
:10743000D6F8082701F4701122F470120A43C6F836
:1074400008275A69666BA16B22F0070232435A6122
:107450005A6922F0700242EA01125A61002835D1BD
:107460009A6A62F00F029A625B6903F007039E4218
:107470003CD10023E365A36D23F0030343F0010334
:10748000A365284603B0F0BD9A68234922F0104254
:1074900022F0170242F080529A60204A1268B2FB32
:1074A000F1F2013252000192019A002A3FF44BAFEF
:1074B000019A013AF7E7002552E7A16D41F020015A
:1074C000A165E16D41F00101E16581E7B0F5001FC3
:1074D000CAD19A6AE269013A92006FF00F0102F094
:1074E0001C0201FA02F2216E0A43BCE7A36D23F0ED
:1074F000120343F01003A365E36D43F00103E3655A
:107500000125BEE7A36D43F01003A365F8E700BFB4
:1075100002FCFF1F00200140400D0300280800204E
:10752000F8B54569082D04460E460AD00368DB68A5
:10753000D80705D5A36D43F02003A3650120F8BD4E
:107540000425FBF743FD074623681A682A4221D029
:10755000A26D42F40072A265DA6812F4406F14D191
:10756000A27E92B91A6812070FD51846FFF7D4FE0B
:1075700028BB5A6822F00C025A60A26D22F4807275
:1075800022F0010242F00102A265207E00BB0C2223
:107590001A60D4E7711CD8D0FBF718FDC01BB042AD
:1075A00001D8002ED0D123681B682B40CCD1A26D0E
:1075B00084F8543042F00402A2650320BFE7A26DB4
:1075C00042F02002A265E26D42F00102E265DCE7D2
:1075D0000020B4E70368186C70470000F7B500237B
:1075E000019390F85430012B044600F0C5800568E3
:1075F0000669012380F854302846FFF78DFE0028E5
:1076000040F0B480D1E90020022826F0040300F005
:107610008280B3F1004FC2F3110E13D1AB6A43EA7B
:107620000E03AB628B68686903EA022323F07C4394
:1076300023F0FF0320EA02210B43002A6B6126DBC3
:10764000002055E0236E00F01F074FF00F0C0CFADE
:1076500007FC6FEA0C0623EA0C0CBEF1000F11D1F7
:10766000C2F38463BB4043EA0C0323668008E369EA
:1076700001309842D6D8A86AC2F38363BB40064063
:107680003343CEE792FAA2F3B3FA83F3EAE73B4936
:107690003B48D1F80837824203F0E07519D11B024C
:1076A000CED4D1F8083723F0E0732B4343F4000322
:1076B000C1F80837334B1A68334BB2FBF3F20C2393
:1076C00002FB03330193019B002BB9D0019B013BCB
:1076D000F8E72E48824210D113F08070B0D1D1F873
:1076E000083723F0E0732B4343F08073C1F8083769
:1076F000002384F8543003B0F0BD254882429FD166
:1077000013F480009CD1D1F8083723F0E0732B43A9
:1077100043F48003EAE7B3F1004F01BFAB6AC2F361
:1077200011018B43AB62002A8ADA15481349824261
:10773000D1F8083709D1D1F8082703F0A07322F057
:10774000E0721343C1F808377AE71048824204D147
:10775000D1F8082703F44003F1E70D4882427FF493
:107760006FAFD1F8082703F0C073E8E7A26D42F0CD
:107770002002A2651846BBE70220BCE700200140BA
:10778000001000B028080020400D0300004000B8A1
:10779000002000B4026838B504461046FFF7BCFD6F
:1077A00008B9002038BD9368990707D4936823F07F
:1077B000004323F0170343F010039360FBF706FC2C
:1077C000054623689B685B07EBD5FBF7FFFB401B77
:1077D0000228F6D923689B685A07F2D5A36D43F0B7
:1077E0001003A365E36D43F00103E3650120D9E7CE
:1077F00073B50023026801939368DD07044602D540
:10780000002002B070BD9168214B194209D0A36DD0
:1078100043F01003A365E36D43F00103E36501202A
:10782000EFE7936823F0004323F0170343F00103CD
:107830009360184BD3F8083718021CD4637E012BD1
:10784000DED0FBF7C3FB144E054622681368DB0746
:10785000D6D49368D9075FBF9368334043F00103E0
:107860009360FBF7B3FB401B0228EED923681B682B
:10787000DA07EAD4CBE7094B094A1B68B3FBF2F3FA
:1078800001330193019B002BD8D0019B013BF8E70A
:107890001700008000200140E8FFFF7F280800203B
:1078A000400D030038B504460068FFF735FD054676
:1078B00020BB94F85430012B20D0012384F854309D
:1078C0002046FFF795FFB0B9A36D226823F47063DB
:1078D00023F0010343F48073A3651C23E065136068
:1078E00084F85400936823F0004323F0170343F017
:1078F0000403936038BD84F85450FBE70220F9E795
:10790000026838B5936891680446C80701D400201E
:1079100038BD9907FBD4936803F00503012B19D1F7
:10792000936823F0004323F0170343F002039360AE
:1079300003231360FBF74AFB054623689B68DB07BC
:10794000E5D5FBF743FB401B0228F6D923689B686B
:10795000DA07F2D5A36D43F01003A365E36D43F09E
:107960000103E3650120D3E770B5044600284BD03E
:10797000836D43F002038365FFF70CFF054668B98A
:107980002046FFF7BDFF054608B90123A36522681D
:10799000936823F0104323F01703936023685A6819
:1079A00022F4677222F003025A6040F29F321A609A
:1079B000D968164A0A40DA601A6922F040421A6110
:1079C0005A6922F007025A611A6A02F0F0221A621A
:1079D0005A6A02F0F0225A62DA6A02F0F022DA629F
:1079E0009A6A0B4A00269E62D2F8083723F0FE738B
:1079F000C2F808372046FAF7C9FCE6652666A66590
:107A000084F85460284670BD0125FBE700023E83E0
:107A10000020014010B590F85430012B044615D0D9
:107A2000012380F85430FFF7B5FE58B92046FFF720
:107A300067FF38B9A36D23F4807323F0010343F08B
:107A40000103A365002384F8543010BD0220FCE735
:107A5000F7B50023019390F85430012B04467FD0F2
:107A6000012380F85430FFF74BFF23689A6812F027
:107A70000102054607D0A36D43F01003A365002360
:107A800084F854302DE0A16D364F21F4817141F01E
:107A90000201A165DE68D96826F4FF4626F07C065F
:107AA00021F40041360421F00301360CD96008208E
:107AB0009968394041F0004199609968002913DACA
:107AC0000199013101910199B1F52E3FF5D3A36DD3
:107AD00023F0120343F01003A365002384F854300D
:107AE0000125284603B0F0BDD3F8B410013801F0E9
:107AF0007F010A44DCD199681A48014041F0010134
:107B00009960D3F8B41021F07F0141EAD202C3F8A2
:107B1000B4209A68024042F002029A60FBF756FADB
:107B2000074623689A68D20708D4DA683243DA60D5
:107B3000A36D23F0030343F001039FE7FBF746FA2D
:107B4000C01B0228EDD923689B68D907E9D5A36D2E
:107B500043F01003A365E36D43F00103E365BFE762
:107B60000225BEE7E8FFFF7F0749CA6822F4E0620A
:107B70000302120403F4E063120C134343F0BF63E7
:107B800043F40033CB60704700ED00E0164B30B596
:107B9000DC68C4F30224C4F10703251D042B28BFAD
:107BA0000423062D4FF0FF358CBF033C002405FA5B
:107BB00003F321EA0303A54022EA0502A3400028BB
:107BC00043EA0203ACBF00F16040084A4FEA0313E6
:107BD000B8BF00F00F00DBB2AABF00F5614013543C
:107BE00080F8003330BD00BF00ED00E014ED00E090
:107BF000002807DB044A4109012300F01F008340ED
:107C000042F82130704700BF00E100E000280CDBA3
:107C10004309064900F01F0020330122824041F849
:107C20002320BFF34F8FBFF36F8F704700E100E059
:107C300070B5D0E913456560446D14B1D0E91645BF
:107C40006560D0E9105404F01C060124B4406C6057
:107C5000046863608368102B0BBFA260A160E160C1
:107C6000E26070BD0268416CD3B210B5083B1424C9
:107C7000B3FBF4F30B4CA24288BF0B4A21F0030183
:107C800099BF01F1804202F5023252180733826433
:107C9000064AC26403F01F03012202FA03F30365DC
:107CA00010BD00BF070402401C08024080080240CB
:107CB00038B500285ED002682F4B9A424FF014016D
:107CC0004CD82E4B1344B3FBF1F32D499B00C0E974
:107CD0001013022380F825301368056923F4FF434D
:107CE00023F070031360D0E9024323432B4345691B
:107CF00011682B4385692B43C5692B43056A2B43C8
:107D00000B431360FFF7AEFFB4F5804F04BF0023B1
:107D100043604268816C02F07F030B60D0E913146A
:107D2000013A032A4C6020D8164A174981651A4443
:107D3000013B9200012103F0030301FA03F3002148
:107D40004265C3651160114A536400230122C36375
:107D500080F8243080F82520184638BD0C4B134499
:107D6000B3FBF1F30B499B00B1E70023C0E91533E6
:107D7000C365EAE70120F0E707040240F8FFFDBF12
:107D8000000002403F82001040090240000902400A
:107D9000F8FBFDBF0004024038B5002841D002685E
:107DA000136823F0010313601F4B9A424FF0140134
:107DB00030D81E4B1344B3FBF1F31D499B00C0E9BF
:107DC0001013012403F01C0304FA03F300251560CB
:107DD0004B60FFF747FF836C41681D60D0E91332A9
:107DE0005A604A1E032A06D8124B0B449B0094404B
:107DF0001D60114B5C640023C363C0E91533C0E907
:107E00000B33C0E90D33C36580F8253080F824308A
:107E1000184638BD094B1344B3FBF1F308499B00E6
:107E2000CDE70120F5E700BF07040240F8FFFDBFE2
:107E3000000002403F82001000090240F8FBFDBF35
:107E40000004024070B590F82450012D04463BD048
:107E500090F825600125AE4280F824504FF00006CE
:107E60002CD1022580F825500568C6632E6826F0BF
:107E700001062E60FFF7DCFE036BBBB12B6843F0FD
:107E80000E032B60A36C1A68D20342BF1A6842F437
:107E900080721A60636D1BB11A6842F480721A60B6
:107EA0002B6843F001032B60002070BD2B6823F08A
:107EB00004032B602B6843F00A03E2E78023C363CB
:107EC00080F824602846F0E70220EEE7034640B140
:107ED00090F82520022A06D00422C263002280F8EE
:107EE0002420012070470268806C116821F00E0187
:107EF0001160016821F480710160116821F00101B5
:107F00001160D3E9100202F01C0101228A40426094
:107F1000D3E9132151605A6D32B1116821F4807197
:107F20001160D3E9162151600122002083F8252039
:107F300083F82400704710B590F82530022B03D049
:107F40000423C363012010BD03681A6822F00E02E7
:107F50001A601A6822F001021A60826C136823F416
:107F600080731360D0E9101303F01C0201239340C7
:107F70004B60D0E913325A60436D33B11A6822F472
:107F800080721A60D0E916325A60012380F82530D9
:107F9000836B002480F8244013B198472046D2E731
:107FA0001846D0E770B4426C046C036826681D68FC
:107FB00002F01C020421914031420FD015F0040F51
:107FC0000CD01A6892065EBF1A6822F004021A608A
:107FD000036B6160002B33D070BC184702219140C5
:107FE000314217D015F0020F14D01A68940606D447
:107FF0001A6822F00A021A60012280F82520114A2C
:1080000093428CBF104B114B5960002380F82430F1
:10801000C36ADFE708219140314211D029070FD50B
:10802000196821F00E011960012303FA02F262605F
:10803000C36380F82530002380F82430436BC9E700
:1080400070BC704780000240000402400000024003
:108050000A4A536943F4802330B55361EFF3108427
:1080600072B60023CD58C5500433B3F5807FF9D1E3
:108070001369DB03FCD484F3108830BD0040005842
:10808000064B5A69002ABFBF054A9A6002F188323E
:108090009A60BABF5869C00F00207047004000586E
:1080A00023016745044B5A6942F000425A615869FE
:1080B000C043C00F704700BF0040005870B5054670
:1080C000FAF784FF124E04463369D90313D4336997
:1080D000DA0744BF012232614CF2FA32134011D167
:1080E0000B4E306910F480200BD0FAF76FFF001BA5
:1080F000A842F6D304E0FAF769FF001BA842E3D3D5
:10810000032070BD024A1361024A01205360F8E760
:1081100000400058381100202DE9F041184D9846D4
:108120002B78012B06460C46174626D001232B70D0
:108130004FF47A7000236B60FFF7C0FFA0B9012EE7
:1081400016D1104A536943F0010353612760BFF30E
:108150006F8FC4F804804FF47A70FFF7AFFF094ABD
:10816000536923EA0603536100232B70BDE8F081B5
:1081700039462046FFF76CFFEDE70220F6E700BF27
:108180003811002000400058054A536923F47E73DB
:1081900043EAC00040F4803040F002005061704774
:1081A000004000582DE9F041234F3B78012B054654
:1081B00088463FD001233B704FF47A7000237B60E8
:1081C000FFF77CFF044688B92B68042B13D11B4AA8
:1081D000536943F4803343F0040353614FF47A70DE
:1081E000FFF76CFF0446154B1A681B6800233B70B1
:1081F0002046BDE8F0814FF0FF33C8F800306E68CC
:10820000D5E901321344B3420AD93046FFF7BCFF27
:108210004FF47A70FFF752FF50B1C8F8006004467F
:10822000064A536923F47E7323F002035361DAE7AD
:108230000136E5E70224DBE7381100200040005852
:108240002DE9F04F524C00234FF00F090A6832FA23
:1082500003F501D1BDE8F08F012505FA03F818EA0E
:10826000020200F08E804E68032706F003054FEAF5
:10827000430E07FA0EFC6F1E012F6FEA0C0C32D86A
:10828000876807EA0C0ACF6807FA0EF747EA0A0779
:108290008760476827EA0808C6F300179F4047EA47
:1082A00008074760C76807EA0C088F6807FA0EF7E7
:1082B00047EA0807022DC76017D14FEAD30800EB41
:1082C000880803F0070AD8F820704FEA8A0A09FAEA
:1082D0000AFB27EA0B0B0F6907FA0AF747EA0B07B5
:1082E000C8F8207001E0032DDCD1076805FA0EF50F
:1082F00007EA0C073D4316F4403F056041D023F0E8
:10830000030707F1804707F5803703F0030CBD68CA
:108310004FEA8C0C4FF0070E0EFA0CFEB0F1904FA6
:1083200025EA0E0E2FD01B4DA8422ED005F58065F4
:10833000A8420CBF0225072505FA0CF545EA0E05F3
:10834000BD602568D74316F4801F0CBF3D40154320
:108350002560656816F4001F0CBF3D40154365603D
:10836000D4F8805016F4803F0CBF3D401543C4F84C
:108370008050D4F88450B60354BF3D401543C4F830
:108380008450013362E70025D6E70125D4E700BF1A
:108390000008005800040048374A2DE9F04F002338
:1083A0004FF0010A4FF0070B4FF00F0931FA03F4B9
:1083B00001D1BDE8F08F0AFA03FC1CEA010654D093
:1083C00023F0030404F1804404F5803403F0030730
:1083D000A568BF000BFA07F8B0F1904F08EA050E48
:1083E00045D0264DA84244D005F58065A8420CBF73
:1083F00002250725BD40754517D1D2F8805025EAE2
:108400000605C2F88050D2F8845025EA0605C2F865
:108410008450156825EA06051560556825EA0605A5
:108420005560A56825EA0805A560056803265C0077
:1084300006FA04F423FA06F6254300EB86060560E7
:1084400003F00705376AAD0009FA05F527EA0507C5
:108450003762856825EA04058560456825EA0C05CC
:108460004560C56825EA0404C46001339EE7002521
:10847000C0E70125BEE700BF00080058000400481F
:108480000369194214BF0120002070470AB18161BD
:108490007047816270470000044AD168014208B504
:1084A00002D0D060FBF7FAFA08BD00BF0008005800
:1084B00003689A69910744BF00229A629A69D207B9
:1084C0005EBF9A6942F001029A61704730B5039D20
:1084D00004682B4343EA0243064A6068C1F309017A
:1084E0000B4342EA555223F0004320EA02000343C3
:1084F000636030BDFF63FF0303682DE9F0419C69B1
:1085000014F0100405460F4616466FD010220024C2
:10851000DA61A0462B689A69900661D4B8F1000F21
:1085200035D044F0040401202E68B369D90541BF59
:108530004FF48072F26144F0010401205A0541BFFA
:108540004FF4806244F00804F26101209B054FD58E
:108550004FF4007344F00204F3612846FFF7A8FFCC
:10856000736823F0FF7323F48B3323F4FF7323F03A
:10857000010373606B6C23436B64202385F84130E7
:10858000002385F8423085F84030012032E07A1C23
:10859000C1D0FAF71BFD801BB84201D8002FB9D11A
:1085A0002B68596895F8422098690004D2B20AD520
:1085B000490408D4202A06D05A6842F480425A60FE
:1085C000FAF704FD06462B689B699B06A2D4FAF7CE
:1085D000FDFC801B1928F6D920244FF0010899E7EB
:1085E000B8F1000F9DD12022DA619AE720469BE77F
:1085F0000028B2D1BDE8F08170B504460D4616469C
:1086000023689B699B0701D5002070BD324629462F
:108610002046FFF771FFA0B96A1CF1D0FAF7D6FC2B
:10862000801BA84201D8002DEAD1636C43F02003DF
:108630006364202384F84130002384F8423084F8B6
:1086400040300120E1E770B504460D461646236828
:108650009B695B070ED4324629462046FFF74CFF44
:1086600038BB23689A69910625D59A69520703D5C4
:10867000228D0AB1002070BD9A6912F010021CBF51
:108680001022DA614FF0200118BF04226264D96120
:108690005A6822F0FF7222F48B3222F4FF7222F029
:1086A00001025A60002384F8411084F8423084F8B3
:1086B00040300120DFE7FAF789FC801BA84201D88F
:1086C000002DC4D1636C43F020036364202384F83D
:1086D00041300023EBE72DE9F041069F0446884630
:1086E00016461D462268936938EA03030CBF01232E
:1086F0000023B34201D0002015E06B1CF3D0FAF741
:1087000065FCC01BA84201D8002DEBD1636C43F07F
:1087100020036364202384F84130002384F842302E
:1087200084F840300120BDE8F08170B504460D4664
:10873000164623689B699B0601D5002070BD324612
:1087400029462046FFF7D8FE90B9FAF73FFC801B78
:10875000A84201D8002DECD1636C43F02003636480
:10876000202384F84130002384F8423084F84030DC
:108770000120E3E710B5044600284AD090F84130C4
:1087800003F0FF021BB980F84020FAF721F92423F7
:1087900084F8413023681A6822F001021A60626886
:1087A00022F070621A619A6822F400429A60D4E959
:1087B0000221012924D142F400429A605A6842F011
:1087C000007242F400425A60DA6822F40042DA6031
:1087D000D4E904210A43A16942EA0122DA60D4E91A
:1087E00007210A431A601A6842F001021A60002049
:1087F0002023606484F84130206384F8420010BD77
:1088000042F4044202299A6004BF4FF400625A60A5
:10881000D4E70120F3E700002DE9F347984690F8EC
:1088200041300A9F202B04460E46914640F0868038
:1088300090F84030012B00F081804FF0010A80F861
:1088400040A0FAF7C3FB19230546009052464FF4A7
:1088500000412046FFF73FFF18B1012002B0BDE8FC
:10886000F087212384F84130102384F8423060647B
:10887000A4F82A80638DC4F824909BB2FF2B606318
:108880002F4B26D9FF22228500934FF0807331466B
:108890002046FFF71BFE638D9BB22A4639462046D1
:1088A000FBB9FFF742FF0028D7D123682021D96107
:1088B0005A6822F0FF7222F48B3222F4FF7222F007
:1088C00001025A6084F8411084F8400084F84200A4
:1088D000C4E7628D009392B222854FF00073D2B24A
:1088E000D5E7FFF789FE0028B7D1636A226813F83D
:1088F000011B91626362638D228D013B9BB2638594
:10890000638D013A92B29BB22285002BC3D0002A1C
:10891000C1D100953B4680212046FFF7DCFE0028B0
:108920009BD1638D9BB2FF2B03D9FF222285009040
:10893000ABE7628D009092B22285CEE702208DE7F0
:10894000002000802DE9F347984690F841300A9FB7
:10895000202B04460E46914640F0878090F8403028
:10896000012B00F082804FF0010A80F840A0FAF756
:108970002DFB19230546009052464FF40041204636
:10898000FFF7A9FE18B1012002B0BDE8F08722234D
:1089900084F84130102384F842306064A4F82A80BF
:1089A000638DC4F824909BB2FF2B6063304B26D9B3
:1089B000FF22228500934FF0807331462046FFF757
:1089C00085FD638D9BB22A4639462046FBB9FFF7E9
:1089D000ACFE0028D7D123682021D9615A6822F043
:1089E000FF7222F48B3222F4FF7222F001025A60ED
:1089F00084F8411084F8400084F84200C4E7628D96
:108A0000009392B222854FF00073D2B2D5E7FFF700
:108A10001AFE0028B7D123685A6A636A1A70636A1B
:108A2000228D01336362638D013B9BB26385638D4D
:108A3000013A92B29BB22285002BC2D0002AC0D14B
:108A400000953B4680212046FFF745FE00289AD13D
:108A5000638D9BB2FF2B03D9FF2222850090AAE7EA
:108A6000628D009092B22285CDE702208CE700BF94
:108A70000024008010B590F84120202A0346D4B28B
:108A80001CD190F84020012A18D0242280F84120DF
:108A90000268106820F001001060106820F4805017
:108AA00010601068014311601168002041F001015D
:108AB000116083F8414083F8400010BD0220FCE7BC
:108AC00010B590F84120202A0346D4B21BD190F86B
:108AD0004020012A17D0242280F841200268106823
:108AE00020F001001060106820F4706040EA01215D
:108AF00011601168002041F00101116083F84140CC
:108B000083F8400010BD0220FCE70000024A136811
:108B100043F4807313607047000400580D4B10B588
:108B20005B690C4628B99A0507D500F027F820B1F3
:108B300010BD9B0501D400F019F8074A1369012CF8
:108B400023F00403136101D130BFF1E740BF20BF20
:108B500020BFEDE70004005800ED00E0024B18686C
:108B600000F4C060704700BF00040058024A136858
:108B700043F4804313607047000400580C4A1368A4
:108B800023F4804313600B4B1B6832214B430A498B
:108B9000B3FBF1F35169890500D533B9536913F477
:108BA000007F14BF032000207047013BF2E700BFA5
:108BB000000400582808002040420F000B4A1368A8
:108BC00023F0070343F002031360094B1A690128DD
:108BD00042F004021A6105D130BF1A6922F0040282
:108BE0001A61704740BF20BF20BFF6E7000400585D
:108BF00000ED00E04FF0B0431868C0F3404070470C
:108C00004FF0B0431868C0F3400070474FF0B042D7
:108C1000536823F47F4343EA0023536070474FF0C7
:108C2000B0431868C0F34060704700007FB54FF054
:108C3000B0432C4AD3F80831C0F3031003F00F03FC
:108C400052F82040284A52F82330B4FBF3F4FFF7DF
:108C500085FF264B054693E80700B5F5007F04AB7A
:108C600003E9070010D0224B9C4218D303F5B70349
:108C700003F67F539C4229D903F5741303F510635F
:108C80009C4225D802230BE01A4B9C4207D91A4B71
:108C90009C421BD903F5370303F5D853F0E70023B3
:108CA00004AA02EB830353F80C4C144D2B6823F0F9
:108CB000070323432B60FAF789F906462B6803F074
:108CC00007039C4206D1002004B070BD0123E7E7F2
:108CD0000024EAE7FAF77AF9801B0228EED903208C
:108CE000F2E700BFD470010874700108106F01082A
:108CF000C0CF6A00BFEA21013F9334020040005810
:108D00004FF0B04310B59A68D96812F00C0205D044
:108D10000C2A4AD101F00303012B50D14FF0B0418E
:108D20002B480B6813F0080306D00B6813F00803F8
:108D300037D1D1F8941007E00C68240756BFD1F85A
:108D400094300968C3F3032350F82330002A0CBF82
:108D5000184600204FF0B0418A6802F00C020C2A3D
:108D60001ED1CA6802F00302022A2ED0032A06D1BD
:108D70000B68184A13F4801F174B18BF13464FF0A7
:108D8000B042D068D168D268C0F306205843C1F31E
:108D900002130133B0FBF3F0530F0133B0FBF3F0D8
:108DA00010BD0B68C3F30313CEE7042A0AD0082AC8
:108DB00005D11B6813F4801304D10748CAE70023C8
:108DC0001846C7E703480023C4E7024BD7E700BFB4
:108DD000D47001080024F4000048E80108B5FFF74A
:108DE0008FFF4FF0B043044A9B68C3F3031352F85C
:108DF0002330B0FBF3F008BD747001082DE9F04199
:108E00000446002853D04FF0B0439D68DE680368E5
:108E10009B0605F00C0506F0030668D5026A1DB135
:108E20000C2D46D1012E44D1002A40D04FF0B04342
:108E3000A16A1A68170756BFD3F894301B681B093C
:108E400003F0F00399421FD90846FFF7EFFE002810
:108E50002DD14FF0B042136843F00803136013683C
:108E6000A16A23F0F0030B431360606AFFF7CEFEA4
:108E7000FFF7B4FFAB4B1860AB4B1868FAF7A4F8D8
:108E8000002834D0BDE8F0814FF0B042136843F0C1
:108E900008031360136823F0F0030B431360606A48
:108EA000FFF7B4FE0846FFF7C1FE0028E0D001201E
:108EB000E8E74FF0B043002A54D01A6842F00102AC
:108EC0001A60FAF783F80746FFF79AFE002842D0A7
:108ED0004FF0B042136843F0080313601368A16AAF
:108EE00023F0F0030B431360606AFFF78FFE2368E3
:108EF000D80748D42368990700F18C8023681E079F
:108F000040F1FA80A3694FF0B046002B00F0E180F9
:108F1000D6F89430E16903F01002914200F0C48069
:108F200003F00302022AC2D0D80740F1B380D6F87A
:108F3000943023F00103C6F89430FAF747F8074657
:108F4000D6F89430990740F1A580FAF73FF8C31B93
:108F5000112BF5D904E0FAF739F8C01B0228B3D970
:108F600003208FE71A6822F001021A60FAF72EF840
:108F70000746FFF745FE0028B9D0FAF727F8C01BCF
:108F80000228F6D9ECE7082D03D00C2D05D1032ECD
:108F900003D16368002BADD189E74FF0B043A168DE
:108FA0001A6822F480120A431A606268B2F5803FA0
:108FB00010D11A6842F480321A60FAF707F80746AF
:108FC000FFF718FE002895D1FAF700F8C01B6428B7
:108FD000F6D9C5E7B2F5041F04D11A6842F40012AD
:108FE0001A60E6E7196821F480311960196821F4E4
:108FF00000111960002AE0D1F9F7E8FF0746FFF7F2
:10900000F9FD00283FF476AFF9F7E0FFC01B6428B4
:10901000F5D9A5E7042D236903D00C2D0ED1022E1E
:109020000CD1002B3FF443AF4FF0B042616953685D
:1090300023F0FE4343EA016353605FE74FF0B0461D
:10904000BBB1336843F480733360F9F7BFFF074661
:1090500033685A0507D57368626923F0FE4343EA13
:10906000026373604AE7F9F7B1FFC31B022BEFD924
:1090700076E7336823F480733360F9F7A7FF074678
:1090800033685B057FF53AAFF9F7A0FFC31B022BEE
:10909000F6D965E74FF0B042E169D2F8943023F099
:1090A00010030B43C2F894304FF0B047D7F8943018
:1090B00043F00103C7F89430F9F788FF0646D7F864
:1090C00094309A0718D4F9F781FF831B112BF6D936
:1090D00046E7D6F8943023F00103C6F89430F9F748
:1090E00075FF0746D6F894309B0705D5F9F76EFF54
:1090F000C31B112BF6D933E72368580754D50B4F00
:109100003B68D90514D4FFF701FDF9F75FFF064668
:109110003B68DA050CD4F9F759FF831B022BF7D90A
:109120001EE700BF280800202C080020000400587B
:10913000E3684FF0B046002B58D023F08003052B96
:1091400002BFD6F8903043F00403C6F890304FF0D9
:10915000B046F9F73BFFD6F8903043F001030746DD
:10916000C6F8903041F28838D6F890309B0705D485
:10917000F9F72CFFC31B4345F6D9F1E6E36823F06A
:109180000403812B1BD1F9F721FFD6F8903043F06F
:109190008003C6F8903007464FF0B04641F2883859
:1091A000D6F89030180504D5E06A00284AD100208E
:1091B00068E6F9F70BFFC01B4045F1D9D0E6F9F797
:1091C00005FFD6F8903023F08003C6F890300746AC
:1091D0004FF0B04641F28838D6F890301905E3D503
:1091E000F9F7F4FEC01B4045F6D9B9E6F9F7EEFEF3
:1091F000D6F8903023F080030746C6F8903041F24D
:109200008838D6F890301A0516D4F9F7DFFED6F86C
:10921000903023F00103C6F8903007464FF0B04875
:1092200041F28836D8F890309B07BDD5F9F7CEFECD
:10923000C31BB342F6D993E6F9F7C8FEC01B4045FD
:10924000DFD98DE60C2D4ED04FF0B04302281A68BE
:1092500022F080721A6033D1F9F7B8FE0546FFF7A5
:10926000DEFC38BBD4E90C314FF0B0420B43D06880
:109270002D4901400B43E16B0B43216C0B43616CA7
:109280000B43A16B43EA0123D360136843F080735F
:109290001360D36843F08053D360F9F797FE044618
:1092A000FFF7BDFC002882D1F9F790FE001B0A28C9
:1092B000F6D955E6F9F78AFE401B0A28CFD94FE6C2
:1092C000F9F784FE0446FFF7AAFC30B94FF0B0422C
:1092D000164BD1680B40D360D4E5F9F777FE001B3D
:1092E0000A28F0D93CE601283FF4CCAD4FF0B0435A
:1092F000226BDB6803F0030191427FF4D8AD616B10
:1093000003F070028A427FF4D2ADA16B03F4FE42F7
:10931000B2EB012F7FF4CBAD626C03F0604393425C
:109320003FF445AFC3E500BF8C80C111FCFFFEEEEA
:109330002DE9F0410D46044610B90120BDE8F08149
:10934000684E336803F007038B4216D323689A07ED
:1093500027D54FF0B047A268BB6823F0F003134352
:10936000BB60F9F733FE0646BB68DB0319D4F9F797
:109370002DFE831B022BF7D911E0336823F007037E
:109380000B433360F9F722FE0746336803F0070307
:10939000AB42DBD0F9F71AFEC01B0228F5D9032037
:1093A000CCE72368580617D54FF0B0476269D7F865
:1093B000083123F00F0343EA1213C7F80831F9F715
:1093C00005FE0646D7F80831D90305D4F9F7FEFDA6
:1093D000831B022BF6D9E2E723685A0713D54FF017
:1093E000B047E268BB6823F4E0631343BB60F9F75E
:1093F000EDFD0646BB689B0305D4F9F7E7FD831B2B
:10940000022BF7D9CBE72368180714D54FF0B047E4
:109410002269BB6823F4605343EAC203BB60F9F7D7
:10942000D5FD0646BB68590305D4F9F7CFFD831B6C
:10943000022BF7D9B3E72368DA070FD4294C236846
:1094400003F00703AB4239D8FFF7C8FC264B18607E
:10945000264BBDE8F0411868F9F7B6BD6268022AEC
:109460001DD1FFF7C7FB00283FF467AF4FF0B046B0
:1094700041F28838B36823F003031343B360F9F76C
:10948000A5FD0746B368626803F00C03B3EB820FD7
:10949000D4D0F9F79BFDC01B4045F3D97FE7032AE1
:1094A00002D1FFF7BCFBDEE712B9FFF7A9FBDAE751
:1094B0004FF0B0431B685B05D8D43EE7236823F028
:1094C00007032B432360F9F781FD0646236803F069
:1094D0000703AB42B8D0F9F779FD801B0228F5D914
:1094E0005DE700BF00400058280800202C0800203D
:1094F00008B5FFF773FC4FF0B043044A9B68C3F311
:10950000022352F82330D84008BD00BFB4700108D0
:1095100008B5FFF763FC4FF0B043044A9B68C3F300
:10952000C22352F82330D84008BD00BFB4700108F0
:109530004FF0B043D3F89000C0F3400070474FF0B5
:10954000B0410209D1F8883002F47F22000123EAF9
:10955000020300F47F200343C1F8883070474FF0C6
:10956000B041020CD1F88830120423EA020343EA26
:109570000040C1F88800704770B5066816F4803660
:10958000044638D0FFF7C2FAF9F720FD614E0546D0
:109590003368DB0529D54FF0B043616BD3F89020D9
:1095A00002F44072914214D0D3F89010D3F8902076
:1095B00042F48032C3F89020D3F8902021F4407018
:1095C00022F480328D07C3F89020C3F8900000F198
:1095D00090804FF0B042616BD2F8903023F440732A
:1095E0000B43C2F89030002605E0F9F7EFFC401B72
:1095F0000228CDD903262568E8070AD54FF0B041E7
:109600006268D1F8883023EA124392B21343C1F85A
:109610008830A9070AD54FF0B041A268D1F8883048
:1096200023EA124392B21343C1F88830AA0609D53F
:109630004FF0B0422169D2F8883023F440630B43E5
:10964000C2F88830AB0502D5206AFFF788FF6805AD
:1096500002D5606AFFF783FF290502D5A06AFFF7EC
:109660007EFF6A0602D56069FFF769FF2B0602D507
:10967000A069FFF764FFE80502D5E069FFF75FFF27
:10968000E90610D54FF0B042E168D2F8883023F4F3
:1096900040730B43C2F88830B1F5807F02BFD368B6
:1096A00043F08073D3602A040ED54FF0B042216B93
:1096B000D2F8883023F040430B43C2F8883019B900
:1096C000D36843F08073D3606B0410D54FF0B04281
:1096D000E16AD2F8883023F040530B43B1F1005FC8
:1096E000C2F8883003D1D36843F48033D360304666
:1096F00070BDF9F76BFC41F288360546FFF718FF9D
:1097000001283FF466AFF9F761FC401BB042F5D980
:1097100070E700BF0004005830B590F82C30012BE2
:1097200002464FF0020022D0174B82F82D00CA24C7
:10973000012582F82C505C6253245C62B1F5807F75
:10974000146B996914D121F488519961596C24F0F2
:10975000010421F0004159641463DD650A4BFF21C7
:1097600059620020012382F82D3082F82C0030BD90
:1097700021F408519961D96C24F0020421F00041D0
:10978000D9641463D865E9E70028004070B50B4E32
:10979000036B756D1D40EA07044603D50123F3658D
:1097A000F9F7DDFDAB0704D50223F365204600F091
:1097B000CBF9012384F82D3070BD00BF0028004094
:1097C00038B50A4CE36823F02003E360F9F7FEFBA9
:1097D0000546E3689B0601D5002038BDF9F7F6FB86
:1097E000401BB0F57A7FF4D90320F6E7002800404B
:1097F0002DE9F041114DEC6814F0400407461AD1F0
:10980000EB6843F08003EB60F9F7E0FB4FF00308EF
:109810000646EB685B0601D4032C02D12046BDE866
:10982000F081F9F7D3FB801BB0F57A7F84BF87F80E
:109830002D800324EDE70024F0E700BF002800405E
:1098400038B50F4CE36823F08003E360A3699B06FF
:10985000054606D4FFF7B4FF10B1032085F82D00AC
:1098600038BDA36923F02003A361FFF7A9FF10B15E
:10987000032085F82D00A36943F02003A361EFE7DF
:109880000028004038B5044600284BD090F82D3011
:1098900003F0FF021BB980F82C20F9F7A5F9022389
:1098A000214D84F82D30EB68DB0632D4CA236B627D
:1098B00053236B622046FFF79BFF78BBAB6923F015
:1098C0008E6323F04003AB6121696368AA690B438F
:1098D0001343A2691343AB61D4E9022343EA024371
:1098E0002B61D4E90931EA680B4322F4F85213439F
:1098F000EB602046FFF7A4FF80B9D4E90713AA69FB
:109900000B4322F06042134362691343AB61FF23B0
:109910006B62012384F82D30002002E0024BFF220D
:109920005A6238BD0120FCE70028004000230928C6
:1099300003D840EA0310C0B270470A380133C0B2FE
:10994000F5E700002DE9F04790F82C30012B054693
:109950004FF0020069D0012385F82C304E4B85F87A
:109960002D00DE6806F44076B6F5807F78D04C692D
:10997000087891F8019091F802A091F82470002ADB
:1099800055D19B6913F0400308BFCB70FFF7CEFFA2
:1099900080464846FFF7CAFF02465046FFF7C6FF1B
:1099A00081463846FFF7C2FF0B6ACF78234343EA6C
:1099B000875343EA090343EA084343EA022343EA9D
:1099C0000063354ACA205062532050628C6A88690D
:1099D000B4F5807F946945D124F4885494610124BE
:1099E000D465B6F5807F09BFCB6913640343536424
:1099F00018BF5064284B4A681A672A6B42F001026C
:109A00002A639A6942F488529A61244AD2F88030D3
:109A100043F40033C2F880301F4BFF225A6200200B
:109A2000012385F82D3085F82C00BDE8F087B4F1CE
:109A3000803F07D0B4F5000F04D09B6913F04003BA
:109A400008BFCB700B6ACA781C4344EA0A0444EA94
:109A5000004343EA092343EA825343EA0763B0E73A
:109A60000023AEE724F4085494610224D465B6F5CB
:109A7000807F09BFCB6993640343D36418BFD0646C
:109A8000054B4A685A672A6B42F002022A639A69B8
:109A900042F40852B8E700BF002800400008005810
:109AA00090F82C20012A03464FF0020012D00A4AF7
:109AB00083F82D00CA21516253215162916941F00E
:109AC00020019161FF2151620020012283F82D20A5
:109AD00083F82C00704700BF0028004090F82C202D
:109AE000012A03464FF0020019D00D4A83F82D00D9
:109AF000CA2151625321516291690A4841F08001A3
:109B00009161D0F8801041F48021C0F88010FF21CD
:109B100051620020012283F82D2083F82C00704729
:109B20000028004000080058064B5A6D520610B538
:109B3000044603D54022DA65F9F714FC012384F8C2
:109B40002D3010BD002800407047890001F1804190
:109B500001F531410A607047890001F1804101F54A
:109B60003141086870470000034AD2F8903043F44E
:109B70000043C2F89030704700040058034AD2F8FE
:109B8000903023F40043C2F890307047000400582E
:109B9000074B1A6822F040021A6040F441704FF4FB
:109BA000B85218605A601A6842F040021A60704752
:109BB0000000015837B5054600284ED0837903F0E0
:109BC000FF046BB1032C0BD0254B4FF400629A615C
:109BD0002868FFF7DDFF002401232B71AC602FE024
:109BE00000236B712846F9F709F91E4AD2F8903024
:109BF00043F48053C2F89030002CE5D102234FF09B
:109C0000B042AB71D2F8943023F40043C2F89430E0
:109C1000154B1B681C214B43DB0C64214B43019308
:109C2000019B93B90124AC60FFF79EFF0C4B9A682F
:109C300042F400629A604FF400629A61002CC7D02F
:109C40000123AB71204603B030BD019B013B019362
:109C5000D2F894305B04E3D4E6E70124F2E700BFD6
:109C600000040058000800582808002037B5174D98
:109C70002B6802461C204343DB0C642043431448FA
:109C80000193019B93B901209060114C21732B68C3
:109C90001C214B43DB0C64214B430193019B6BB9AB
:109CA000012090600A4BDB6803B030BD019B013B93
:109CB000019383689C07E4D50020E6E7019B013B04
:109CC0000193A368DB07E9D5ECE700BF2808002073
:109CD0000000015837B5184D2B6802461C2043433D
:109CE000DB0C6420434315480193019BA3B9012079
:109CF0009060124CFF2323732B681C256B43DB0CF5
:109D000064256B430193019B73B9012090600B4B59
:109D1000DB680B7003B030BD019B013B019383688E
:109D20009C07E2D50020E4E7019B013B0193A36877
:109D3000DB07E8D5EBE700BF28080020000001584A
:109D40000F4B13B51B680F4C182253431B0D642295
:109D50005343014601936269019B02F0040223B957
:109D600002238B60012002B010BD019B013B0193D7
:109D7000606910F00200F6D0002AECD11046F2E73C
:109D8000280800200004005807B50379012B0FD1E3
:109D90000A4B1B68182253431B0C0193FFF7EEFE7E
:109DA000019B013B0193019B002BF9D1FFF7DCFEE6
:109DB00003B05DF804EBFFF7C3BF00BF2808002025
:109DC000F8B51E468379012B154604460F46DAB2D4
:109DD0002DD14379012B2AD0022342718371FFF7E1
:109DE000D3FF0D212046FFF7C9FEFFF73FFF390AD9
:109DF0002046FFF73BFFF9B22046FFF737FF2E441E
:109E0000B5420ED12046FFF7AFFEFFF799FFA068DD
:109E100001230038A3714FF0000318BF01206371C4
:109E2000F8BD15F8011B2046FFF720FFE8E70220E8
:109E3000F6E7F8B51E468379012B154604460F4612
:109E4000DAB22FD14379012B2CD04271FFF79CFF5E
:109E50001D212046FFF792FEFFF708FF390A204632
:109E6000FFF704FFF9B22046FFF700FF002120466C
:109E7000FFF7FCFE2E44B5420ED12046FFF774FEDC
:109E8000FFF75EFFA06801230038A3714FF00003C5
:109E900018BF01206371F8BD29462046FFF71AFF5D
:109EA0000135E8E70220F6E7F8B51F468379012B74
:109EB000154604460E46DAB22CD14379012B29D03F
:109EC0004271FFF761FF06F0EF03A3F184025342F2
:109ED0005341237131462046FFF750FEFFF7C6FE7F
:109EE0002F44AF4210D1FFF73FFE842E02D0204610
:109EF000FFF726FFA06801230038A3714FF000038D
:109F000018BF01206371F8BD15F8011B2046FFF74B
:109F1000ADFEE6E70220F6E7F8B51E468379012B91
:109F2000154604460F46DAB227D14379012B24D0D7
:109F30004271FFF729FF39462046FFF71FFEFFF762
:109F400095FE00212046FFF791FE2E44B5420ED12A
:109F50002046FFF709FEFFF7F3FEA0680123003853
:109F6000A3714FF0000318BF01206371F8BD2946AB
:109F70002046FFF7AFFE0135E8E70220F6E737B5E8
:109F80000023ADF8043001AA022312210546FFF791
:109F9000C3FFBDF80440022364BA01AAA4B2194663
:109FA0002846FFF781FFE20702D5284609F0DAFBD1
:109FB000A30702D5284609F0DBFB600702D5284637
:109FC00009F000FC210702D5284609F001FCE20651
:109FD00002D5284609F002FCA30602D5284609F05E
:109FE000EBFB600602D5284609F0C8FB210606D522
:109FF00014F4807118BF0121284609F0C5FBA205A1
:10A0000002D5284609F0D0FB630402D5284609F0A2
:10A01000EBFB03B030BDF8B51E468379012B154626
:10A0200004460F46DAB227D14379012B24D042717E
:10A03000FFF7AAFE0E212046FFF7A0FDFFF716FE50
:10A0400039462046FFF712FE2E44B5420ED1204677
:10A05000FFF78AFDFFF774FEA06801230038A371A3
:10A060004FF0000318BF01206371F8BD15F8011B04
:10A070002046FFF7FBFDE8E70220F6E7F8B51E46AD
:10A080008379012B154604460F46DAB22BD143796A
:10A09000012B28D04271FFF777FE1E212046FFF7E3
:10A0A0006DFDFFF7E3FD39462046FFF7DFFD002198
:10A0B0002046FFF7DBFD2E44B5420ED12046FFF7C8
:10A0C00053FDFFF73DFEA06801230038A3714FF058
:10A0D000000318BF01206371F8BD29462046FFF731
:10A0E000F9FD0135E8E70220F6E7026852E8003F93
:10A0F00023F0C00342E8003102680029F5D102F1E3
:10A10000080353E8003F23F4000302F1080C4CE875
:10A1100000310029F3D12023C0F8883070470000B7
:10A1200010B5026852E8003F23F4907342E8003112
:10A1300002680029F5D10F4C02F1080353E8003FF3
:10A14000234002F1080C4CE800310029F4D1C36E21
:10A15000012B07D152E8003F23F0100342E8003101
:10A160000029F7D12023C0F88C300023C366436751
:10A1700010BD00BFFEFFFFEFF8B504461346D4F84C
:10A180008850202D32D1F1B1EAB1E06FA4F8562009
:10A19000A4F8542000262122C4F890602165C4F858
:10A1A0008820226888B1124FC762124F0763124F8E
:10A1B0002832C0E90D76FDF745FE30B11023C4F812
:10A1C0009030C4F8885001200FE0236840221A62C2
:10A1D000226802F1080353E8003F43F0800302F1D4
:10A1E000080141E800300028F3D1F8BD0220FCE767
:10A1F000FDA1000845A2000851A2000808B50346C9
:10A20000806A1B681B6813F0200317D1A0F8563032
:10A21000026802F1080353E8003F23F0800308328C
:10A2200042E8003102680029F2D152E8003F43F0D1
:10A23000400342E800310029F7D108BDF9F7C8F919
:10A24000FBE7704708B5806AFFF7FBFF08BD704762
:10A25000806A38B50468D0F88830D0F88C50A2688D
:10A26000120606D5212B04D10023A0F85630FFF7A3
:10A270003CFFA3685B0606D5222D04D10023A0F87D
:10A280005E30FFF74DFFD0F8903043F01003C0F878
:10A290009030FFF7DCFF38BD08B5806A0023A0F8D6
:10A2A0005E30A0F85630FFF7D2FF08BD70470000BF
:10A2B0000368D9691A682DE9F04140F60F0631426A
:10A2C0009D68044610D18E0640F1978002F020066A
:10A2D00005F080573E4300F09080436F002B00F064
:10A2E0008580BDE8F0411847AB4EAC482E40104089
:10A2F000304300F08280CF0709D5D00507D5012073
:10A300001862D4F8900040F00100C4F890008F0764
:10A3100009D5E80707D502201862D4F8900040F06C
:10A320000400C4F890004F0709D5E80707D50420BA
:10A330001862D4F8900040F00200C4F890000F07B3
:10A340000BD502F02000304307D008201862D4F863
:10A35000900040F00800C4F890000E050AD55001A6
:10A3600008D54FF400601862D4F8903043F0200311
:10A37000C4F89030D4F89030002B37D08B0609D534
:10A3800002F0200205F080552A4303D0636F0BB121
:10A39000204698472668D4F89020B36802F0280237
:10A3A00003F0400353EA0205204621D0FFF7B8FE30
:10A3B000B3685F0617D5226802F1080353E8003F2F
:10A3C00023F04003083242E800310029F3D1D4F8E9
:10A3D000800040B1724B8363FDF7ADFD30B1D4F81E
:10A3E0008000836B7DE72046FFF731FFBDE8F081F9
:10A3F000FFF72DFFC4F89050F8E7E06E012840F019
:10A400008980CE0640F18680D00640F183801022FC
:10A410001A629A6851064BD5D4F8802011684A68B0
:10A4200092B2002AE2D0B4F85C009042DED9A4F8DF
:10A430005E200A6892062FD453E8002F22F480721F
:10A4400043E800210029F7D103F1080252E8002F68
:10A4500022F0010203F1080040E800210029F3D1B5
:10A4600003F1080252E8002F22F0400203F1080035
:10A4700040E800210029F3D12022C4F88C20E166B5
:10A4800053E8002F22F0100243E800210029F7D101
:10A49000D4F88000FDF71AFD02232367B4F85E307C
:10A4A000B4F85C10C91A89B22046FFF7FFFE9DE799
:10A4B000B4F85E20B4F85E00B4F85C1080B292B2DA
:10A4C000002893D0891A89B200298FD053E8002F31
:10A4D00022F4907243E800200028F7D1314D03F1B7
:10A4E000080252E8002F2A4003F1080646E800203F
:10A4F0000028F4D12022C4F88C206067E06653E87D
:10A50000002F22F0100243E800200028F7D1022398
:10A510002367C9E7CF0209D56E0207D54FF4801231
:10A5200020461A62BDE8F04100F0F2BD08060BD5E6
:10A5300002F0800005F40005284305D0A36F002B2E
:10A540003FF454AF2046CCE64F0611D556060FD542
:10A5500053E8002F22F0400243E800210029F7D100
:10A560002023C4F88830A1672046F9F731F83DE789
:10A570000D0206D5500004D52046BDE8F04100F09C
:10A58000C9BDCB017FF532AF002ABFF62FAF204601
:10A59000BDE8F04100F0BDBD010000102001000445
:10A5A00099A20008FEFFFFEFD0F88C20B0F86010F1
:10A5B000222A08B5036855D15B6A826D0B4013707F
:10A5C000836D01338365B0F85E30013B9BB2A0F828
:10A5D0005E30B0F85E309BB2002B42D1026852E888
:10A5E000003F23F4907342E8003103680029F5D15D
:10A5F00003F1080252E8002F22F0010203F1080CD7
:10A600004CE800210029F3D12022C0F88C20184A00
:10A6100041679342016705D1C26E012A0ED0F8F757
:10A62000E5FF1EE05A681102F6D553E8002F22F02C
:10A63000806243E800210029F7D1EDE70022C266DD
:10A6400053E8002F22F0100243E800210029F7D13F
:10A65000DA69B0F85C10D20644BF10221A62FFF724
:10A6600025FE08BD9A6942F008029A61F9E700BF29
:10A6700000800040D0F88C20B0F86010222A08B585
:10A68000036852D15A6A1140826D22F8021B82651A
:10A69000B0F85E20013A92B2A0F85E20B0F85E20D9
:10A6A00092B2002A40D153E8002F22F4907243E87E
:10A6B00000210029F7D103F1080252E8002F22F00F
:10A6C000010203F1080C4CE800210029F3D12022FB
:10A6D000C0F88C20174A41679342016705D1C26ECA
:10A6E000012A0ED0F8F782FF1EE05A681102F6D553
:10A6F00053E8002F22F0806243E800210029F7D1BF
:10A70000EDE70022C26653E8002F22F0100243E872
:10A7100000210029F7D1DA69B0F85C10D20644BFF5
:10A7200010221A62FFF7C2FD08BD9A6942F00802C2
:10A730009A61F9E7008000402DE9F74F0368B0F80F
:10A740006080DF691A689D68D0F88C100192222918
:10A75000044640F0B480B0F86890DFF86CA1DFF8F0
:10A760006CB10026B9F1000F01D0BB0621D4B4F8BA
:10A770005E309BB2D3B1B4F868209A4216D92268F1
:10A7800002F1080353E8003F23F08053083242E807
:10A79000003122680029F2D14D4B636752E8003F37
:10A7A00043F0200342E800310029F7D103B0BDE8AF
:10A7B000F08F2368A26D5B6A03EA08031370A36D30
:10A7C0000133A365B4F85E30013B9BB2A4F85E3060
:10A7D0002368DF6978072CD0F9070AD5019AD205DA
:10A7E00007D501211962D4F8901041F00101C4F895
:10A7F0009010B80709D5E90707D502211962D4F8E6
:10A80000901041F00401C4F890107A0709D5E807C8
:10A8100007D504211962D4F8903043F00203C4F83C
:10A820009030D4F8903023B12046FFF710FDC4F8E3
:10A830009060B4F85E309BB2002B93D1216851E850
:10A84000003F23F4807341E8003023680028F5D1ED
:10A8500003F1080252E8001F01EA0A0142E8001071
:10A860000028F5D120215B45C4F88C106067206773
:10A870000AD05968090207D553E8001F21F080610A
:10A8800043E800100028F7D1E16E012913D1E666F4
:10A8900053E8001F21F0100143E800100028F7D111
:10A8A000D969CA0644BF102119622046B4F85C1069
:10A8B000FFF7FCFC56E72046F8F798FE52E79A6946
:10A8C00042F008029A6171E7FEFFFFEF008000404E
:10A8D000A9A500082DE9F74F0368B0F86080DF698B
:10A8E0001A689D68D0F88C1001922229044640F025
:10A8F000B280B0F86890DFF868A1DFF868B1002690
:10A90000B9F1000F01D0BB0621D4B4F85E309BB280
:10A91000D3B1B4F868209A4216D9226802F108032C
:10A9200053E8003F23F08053083242E800312268A8
:10A930000029F2D14C4B636752E8003F43F02003FB
:10A9400042E800310029F7D103B0BDE8F08F236859
:10A95000A26D596A08EA010122F8021BA265B4F847
:10A960005E20013A92B2A4F85E20DF6978072CD00D
:10A97000F9070AD5019AD20507D501211962D4F841
:10A98000901041F00101C4F89010B80709D5E9070B
:10A9900007D502211962D4F8901041F00401C4F8DF
:10A9A00090107A0709D5E80707D504211962D4F871
:10A9B000903043F00203C4F89030D4F8903023B1C3
:10A9C0002046FFF744FCC4F89060B4F85E309BB2B8
:10A9D000002B95D1216851E8003F23F4807341E8B2
:10A9E000003023680028F5D103F1080252E8001F67
:10A9F00001EA0A0142E800100028F5D120215B4558
:10AA0000C4F88C10606720670AD05968090207D51E
:10AA100053E8001F21F0806143E800100028F7D1BF
:10AA2000E16E012913D1E66653E8001F21F0100101
:10AA300043E800100028F7D1D969CA0644BF1021A5
:10AA400019622046B4F85C10FFF730FC58E7204646
:10AA5000F8F7CCFD54E79A6942F008029A6173E76F
:10AA6000FEFFFFEF0080004075A6000838B50446E1
:10AA700003682169A2681D68C0690A4361690A43C5
:10AA80007D49024329400A431A605A68E16822F46A
:10AA900040520A435A60794AA16993421CBF226A14
:10AAA00011439A6822F06E4222F430620A439A609F
:10AAB000DA6A616A22F00F020A43DA62704A93424C
:10AAC0001CD14FF0B043D3F8883003F0030343F4B4
:10AAD0004033A3F54033013B022B00F2C780694AA3
:10AAE0009B5CB0F5004F40F08980082B24D8DFE84C
:10AAF00003F061C08323802323236500624A9342CD
:10AB000009D14FF0B043614AD3F8883003F00C0309
:10AB100043F44023E4E7594A93420DD14FF0B04348
:10AB2000D3F8883003F44063B3F5006F1AD005D82A
:10AB300053B1B3F5806F12D0012009E0B3F5406F37
:10AB4000FAD14FF400400EE0FEF7D2FC58B90020D5
:10AB50004FF00113A3660023C4E91D3338BDFEF78F
:10AB6000CFF8F3E74A4865684A4B626A05EB45014E
:10AB700033F81220B0FBF2F39942DDD8B3EB053F76
:10AB8000DAD800231946F7F743FA090241EA1061BF
:10AB90006B080002C0182A464FF0000341F1000183
:10ABA000F7F736FA3C4BA0F540729A42C4D82368B6
:10ABB000D860CCE7FEF79CFC0028C8D06168354B14
:10ABC000626A33F81220B0FBF2F24B0803EB420347
:10ABD0004FF6EF72B3FBF1F3A3F110019142ABD842
:10ABE00023F00F02216892B2C3F342031343CB60F8
:10ABF000ADE7FEF785F8DFE72548DFE7082B9BD8B0
:10AC000001A252F823F000BF51AC00085DAC00086F
:10AC100069AC000839AB000863AC000839AB000828
:10AC200039AB000839AB00082DAC00084FF40040E8
:10AC30006368616A174A32F81120B0FBF2F000EB4A
:10AC40005300B0FBF3F04FF6EF73A0F11002ACE746
:10AC5000FEF74EFC00283FF47AAFE9E7FEF758FC18
:10AC6000F8E7FEF74DF8F5E70948E1E7B0F5004FE2
:10AC7000F4D1FEF74DFC9FE7F369FFCF0080004061
:10AC80000038014014710108004400401771F507B5
:10AC90000024F40024710108FFFC0F00836ADA0726
:10ACA00010B506D50168C46A4A6822F4003222430E
:10ACB0004A609C0706D50168046B4A6822F480321A
:10ACC00022434A60590706D50168446B4A6822F45A
:10ACD000802222434A601A0706D50168846B4A68BD
:10ACE00022F4004222434A60DC0606D50168C46BA8
:10ACF0008A6822F4805222438A60990606D5016848
:10AD0000046C8A6822F4005222438A605A060FD5E6
:10AD10000168446C4A6822F480122243B4F5801F13
:10AD20004A6005D14A68846C22F4C00222434A601A
:10AD30001B0606D50268C16C536823F400230B433D
:10AD4000536010BD2DE9F041DDF8188004460E4631
:10AD500015461F462268D36936EA03030CBF012358
:10AD60000023AB4201D0002027E0B8F1FF3FF2D032
:10AD7000F8F72CF9C01B4045206802D8B8F1000F45
:10AD80001DD150E8003F23F4D07340E80032002A80
:10AD9000F7D100F1080353E8003F23F0010300F16D
:10ADA000080141E80032002AF3D12023C4F888309A
:10ADB000C4F88C3084F884200320BDE8F081036857
:10ADC0005A07C7D5C3691B05C4D54FF40063036296
:10ADD00050E8003F23F4D07340E80032002AF7D156
:10ADE00000F1080353E8003F23F0010300F10801DC
:10ADF00041E80032002AF3D12023C4F88830C4F897
:10AE00008C30C4F89030D5E72DE9F7439846D0F858
:10AE10008830202B04460E46174643D1002943D0E4
:10AE2000002A41D021230025C0F89050C0F8883076
:10AE3000F8F7CCF8A368A4F85470B3F5805F8146A6
:10AE4000A4F8567003D123690BB935461E46B4F8F1
:10AE50005620CDF8008092B24B4642B940212046A0
:10AE6000FFF770FF48B92023C4F8883006E00022BD
:10AE700080212046FFF766FF18B1032003B0BDE82C
:10AE8000F08322685EB935F8023BC3F3080393628E
:10AE9000B4F85620013A92B2A4F85620D7E716F833
:10AEA000013BF4E70220E9E70120E7E773B5044638
:10AEB0000026C0F89060F8F789F823681B681A0725
:10AEC000054619D423681B685B070AD56FF07E43DB
:10AED000009300222B464FF480012046FFF732FFFB
:10AEE000B0B900202023C4F8883084F88400C4F866
:10AEF0008C30E06620670CE06FF07E4300933246B2
:10AF000003464FF400112046FFF71CFF0028D9D05C
:10AF1000032002B070BD10B5044650B3D0F888309D
:10AF20001BB980F88430F8F75FFA22682423C4F84C
:10AF30008830136823F0010313602046FFF796FD65
:10AF4000012816D0A36A13B12046FFF7A7FE236895
:10AF50005A6822F490425A609A6822F02A029A6053
:10AF60001A6842F0010220461A60BDE81040FFF75F
:10AF70009DBF012010BD000030B581658168A0F83B
:10AF80005C200023B1F5805FA0F85E20436735D1D7
:10AF90000369002B40F2FF1318BFFF23A0F86030B5
:10AFA0000023C0F890302223C0F88C30016801F1F2
:10AFB000080353E8003F43F00103083141E800343F
:10AFC0000368002CF2D1456E84680169B5F1005F19
:10AFD00034D1B0F86850954230D8B4F5805F1DD1B7
:10AFE000254A264C002918BF22464267C1B153E8C2
:10AFF000002F42F4807243E80021F7E729B9036982
:10B00000002B14BF7F23FF23C8E7B1F1805FC5D1B8
:10B010000369002B0CBF7F233F23BFE7174AE4E7F8
:10B0200003F1080252E8002F42F0805203F10800B9
:10B0300040E800210029F3D1002030BDB4F5805F45
:10B040000FD10F4A0F4C002918BF2246426751B159
:10B0500053E8002F42F4907243E800210029F7D111
:10B06000EAE7084AF2E753E8002F42F0200243E8FB
:10B0700000210029F7D1DFE7D5A8000839A700088B
:10B0800075A60008A9A50008D0F88C30202B30B494
:10B0900015D1B9B1B2B100230468C3660A4B9C4212
:10B0A0000AD063681B0207D554E8003F43F0806371
:10B0B00044E80035002DF7D130BCFFF75DBF02201A
:10B0C00030BC70470120FBE700800040436E30B584
:10B0D0002BB90123A0F86A30A0F8683030BD0368AE
:10B0E000094D9A689968094C490FC2F342626B5C3A
:10B0F000615CDB00B3FBF1F3A0F86A30AB5CA25CEF
:10B10000DB00B3FBF2F3E7E7447101083C7101088F
:10B110007047704770471FB504AB03E9060090F80D
:10B120008430012B04463AD0012380F88430242354
:10B13000C0F8883003681A6822F001021A609A6821
:10B1400022F440120A439A6071B95A68BDF80C00A3
:10B150009DF80E1022F0100202435A605A6822F045
:10B160007F4242EA01625A601A6842F001021A60A4
:10B17000F7F72CFF6FF07E42034600924FF48001F8
:10B1800000222046FFF7DEFD38B92023C4F88830BE
:10B19000002384F8843004B010BD0320F8E70220B7
:10B1A000F9E790F88430012B0FD0012380F8843028
:10B1B000016851E8002F42F0020241E80023002B11
:10B1C000F6D180F88430184670470220704710B5D9
:10B1D00090F88430012B044617D02423C0F888301F
:10B1E00003681A68196821F00101196042F00052E1
:10B1F0004FF0005141661A60FFF768FF2023C0F846
:10B200008830002084F8840010BD0220FCE770B56F
:10B2100090F88430012B044617D005682423C0F829
:10B2200088302E682B6823F001032B60AB6823F075
:10B2300060431943A960FFF749FF20232E60C0F83F
:10B240008830002084F8840070BD0220FCE770B5CF
:10B2500090F88430012B044617D005682423C0F8E9
:10B2600088302E682B6823F001032B60AB6823F035
:10B2700060631943A960FFF729FF20232E60C0F8FF
:10B280008830002084F8840070BD0220FCE70000B4
:10B2900038B5084D052455F8043B2BB9013C14F092
:10B2A000FF04F8D1204638BDDB6898470028F5D068
:10B2B000F9E700BF6C120020034BD870034B1B68EA
:10B2C0001B6C03B1184770478012002068120020E1
:10B2D000034B1874034B1B685B6C03B11847704732
:10B2E0008012002068120020F0B5314D314B95F9E5
:10B2F0000420314E91B00C46012795F905108DF8C8
:10B30000047002288DF809208DF80A1010D18DF8EC
:10B310000800D8711C7202F09FFD337803B114B19C
:10B3200001A803F003FA254B059A1A6011B0F0BD8D
:10B3300059714FF480711A71D9801C7233788DF86D
:10B34000087053BB1F2306A88DF81C208DF81830F9
:10B3500002F064FF20238DF8183006A82B798DF8B1
:10B360001C3002F05BFF22238DF8183006A86B79A1
:10B370008DF81C3002F052FF21238DF8183006A8FA
:10B380006B798DF81C3002F049FF29238DF81830B5
:10B3900006A80B4B079302F041FF02F05DFD01236D
:10B3A00006A88DF818308DF81C3002F037FFB4E78E
:10B3B00080120020300800205C1200206012002063
:10B3C000000400017FB5092301A88DF8043003F0C3
:10B3D000ADF90038044B059A1A6018BF01204042AD
:10B3E00007B05DF804FB00BF6012002070B5044692
:10B3F0000B46134962784A700020A2780A720870DE
:10B400001A884A729A788A72DB780B746368CB6008
:10B410000C4B1B68DA6A2AB1237803F0FB030A2B72
:10B4200000D09047084E052556F8043B1BB15B6AD7
:10B430000BB120469847013D15F0FF05F4D170BDD2
:10B440003C080020681200206C12002070B50446F1
:10B4500010480123037063784370A3788372E36814
:10B46000C360E378037623694376237943720A4BFA
:10B470001B689B6A03B19847084E052556F8043BA4
:10B480001BB19B690BB120469847013D15F0FF05A4
:10B49000F4D170BD50080020681200206C1200200A
:10B4A000014B1868704700BF6012002000B58BB0D8
:10B4B000012368468DF8003002F088FD38B99DF808
:10B4C0000400003818BF01200BB05DF804FB002019
:10B4D000FAE7000008B501F073FE48B9FFF7E6FF90
:10B4E000012806D0054BD879197AFFF7FDFE012017
:10B4F00008BDBDE80840FFF7CBBE00BF3008002004
:10B500002DE9F04186B005460E46174601F058FE7B
:10B5100000287FD101F06CFE044640B9FFF7C6FF5A
:10B52000012807D03D4B197AD879FFF7DDFE6FF07F
:10B53000020462E0DFF8E88088F80860003E18BF87
:10B5400001268DF80460374E687833798DF8123013
:10B55000694602F0D9FC00283ED08DF804400394DF
:10B56000ADF810406FF0060495E803002E4B83E819
:10B570000300337988F80A30394601A803F0DAF974
:10B580002A4B059A1A60112841D801A353F820F0DC
:10B59000EFB5000815B600080FB600080FB6000892
:10B5A0000FB600080FB600080FB600082FB5000848
:10B5B0000FB600080FB600080FB6000809B600085D
:10B5C0000FB600080FB6000815B6000815B600083B
:10B5D00015B6000803B600082B788DF808306B7894
:10B5E000ADF810306B6803934FF0FF34BCE7104B9D
:10B5F00000221A70E31D18BF1446204606B0BDE8AD
:10B60000F0816FF00404F8E76FF00504F5E74FF000
:10B61000FF34F2E76FF00104EFE700BF30080020CD
:10B6200050080020801200206008002060120020D6
:10B630006412002037B501F0E5FD144D052455F8DE
:10B64000043B5BB11B694BB155F8043C9B682BB1C3
:10B65000984718B155F8043C1B699847013C14F011
:10B66000FF04ECD1FFF714FE68B9094D2B7853B1F4
:10B67000084BADF80040D978019422466846FFF7A0
:10B680003FFF00B92C7003B030BD00BF6C1200202A
:10B69000641200208012002030B58BB0054601F006
:10B6A0008FFD0446002839D1FFF700FF012838D16B
:10B6B00068468DF8004002F089FC10B14FF0FF3071
:10B6C00004E09DF80430AB4202D100200BB030BD45
:10B6D000012DF3D0022D11D0002DF7D1002BF4D085
:10B6E00068468DF8045002F099FD0028E6D10E4B13
:10B6F0001B681B6B002BE8D09847E6E7002BDDD1D9
:10B7000068468DF8045002F089FD0028D6D1064B1A
:10B710001B681B6B002BD8D02846EDE76FF00100AB
:10B72000D4E76FF00200D1E76812002010B504469C
:10B730008AB018B94FF0FF300AB010BD0023684638
:10B740008DF8003002F042FC0028F3D19DF804305F
:10B750002370F1E77FB500220B4620498DF80720C2
:10B7600001220A7042784A700446002A33D10279D5
:10B770000A721A884A729A788A72DB780B740369A3
:10B78000CB60C378164D8DF80830037B8DF80930F7
:10B79000836803932B68DB6A0BB102A898472B6878
:10B7A0009B6B13B1227E02B198470E4E052556F8C9
:10B7B000043B1BB1DB690BB120469847013D15F0F6
:10B7C000FF05F4D10DF10700FFF7B0FF637913B166
:10B7D000054B01221A7004B070BD00BF3C08002068
:10B7E000681200206C1200206412002010B504467C
:10B7F0008AB018B94FF0FF300AB010BD2023684658
:10B800008DF8003002F0E2FB0028F3D1024A9DF9E6
:10B81000043023701371EFE78012002000B58BB065
:10B820002323019068468DF8003002F0F7FC0038C1
:10B8300018BF012040420BB05DF804FB70B5654CA9
:10B8400001468EB01822204606F0FEF8624B002218
:10B850001A70F8F7C3FE23784068012202FA03F158
:10B86000014004D15D4B084608F0E4F8FEE75C496E
:10B870005C481A4602F032F918B14FF0FF300EB0B2
:10B8800070BD272304A88DF8103002F0C7FC564E77
:10B89000564D002870D1012333702B68DB690BB142
:10B8A00000209847272304A88DF8103002F08EFB63
:10B8B000059B93F84820227093F8182193F81A31C9
:10B8C0006270A370464BD3E9020105F0AFFF054655
:10B8D0000028D2D1464E062304A88DF8103002F07D
:10B8E00075FB059B736104A802F098FC022304A871
:10B8F0008DF81030059602F069FB0836032304A882
:10B900008DF81030059602F061FB0F2606F052F814
:10B91000012304A88DF814308DF8106002F07EFC2D
:10B9200010230DEB03008DF810308DF8145002F049
:10B9300075FC04238DF8103004A8A3788DF814301A
:10B9400002F06CFC3A238DF8103004A8636905936B
:10B9500002F064FC02A920788DF8086004F0E8F891
:10B96000003818BF0120E0711420FFF757FFE0797D
:10B9700003F0A4F9284682E728238DF810302B68BD
:10B980001B6943B104A802F021FB2B6805981B69D1
:10B9900040F2C4519847272304A88DF8103002F0D4
:10B9A0003DFC50B9012304A88DF8103002F00EFBC5
:10B9B0009DF81430002B7FF46EAF3378002B7FF4AA
:10B9C0006CAF052204A88DF81020059302F026FC28
:10B9D00078E700BF80120020641200204C7101083B
:10B9E000A8120020C01200205C1200206812002063
:10B9F0004412002037B500230D4601930446D0B908
:10BA000000F0A8FB0190019BD3B10F4A42F824300B
:10BA10000E4A9A620E4A1268916B1963916C5963CF
:10BA200092690C49D9625A6128465B680A49F22238
:10BA30009847002006E001A900F092FB0028E2D020
:10BA40004FF0FF3003B030BD6C120020E9B20008A7
:10BA500068120020C5B3000850110020194B07B52B
:10BA60001860194B194A1A60194A5A60194A9A60A3
:10BA7000194ADA60194B02681A6042685A60826893
:10BA80009A60C268DA60164A1A6182695A61154B77
:10BA9000C26B5A60144A019119609A601946134AA0
:10BAA000DA600020FFF7A6FF48B901A800F056FBB6
:10BAB000003818BF0120404203B05DF804FB4FF08E
:10BAC000FF30F9E768120020C01200204DB40008D2
:10BAD00055B700086DBB0008EDB30008A8120020A0
:10BAE000E1FA000898120020B9B20008D1B20008AB
:10BAF00051B118B1012804D000207047044B0B60ED
:10BB00007047044B0B60F7E74FF0FF30704700BF02
:10BB1000000400010100010208B503F0EBF8002861
:10BB200014BF6FF00100002008BD08B502F0BCF999
:10BB3000002814BF6FF00100002008BD10B50446B6
:10BB40008AB018B94FF0FF300AB010BD2123684603
:10BB50008DF8003002F03AFA0028F3D1024A9DF93C
:10BB6000043023705371EFE7801200202DE9F0417B
:10BB70002E4D2F4F00232B7043786B703B689B6AD0
:10BB80008AB004460BB128469847DFF8A8800526FE
:10BB900058F8043B1BB11B6A0BB120469847013E85
:10BBA00016F0FF06F4D12378052B2FD00B2B35D0C0
:10BBB000012B25D1204C062368468DF8003002F079
:10BBC00005FA0199E07905F077FE10B91B4B019A4F
:10BBD0005A611B48FFF70AFE1A48FFF7AFFF6B7860
:10BBE0008BB9A371184B5878FFF756FD3B685B6A19
:10BBF0000BB1114898476B7813B9E07905F0ECFE6A
:10BC00000AB0BDE8F081FF23A371EFE70F4B0122DB
:10BC10005A74227A9A74627ADA74F1E76378002BA4
:10BC2000EED00AB0BDE8F041FFF7CCBB50080020D1
:10BC3000681200206C1200203008002044120020FE
:10BC40003408002035080020801200203C08002025
:10BC500030B58BB0FFF769FF0446F0B903F048FF39
:10BC6000831C1DD0F8B9134D2B685B69DBB127230A
:10BC700068468DF8003002F0A9F92B6801985B69DD
:10BC80004FF4B961984703F045FF78B92CB9094BD7
:10BC90001B68DB690BB10120984720460BB030BD13
:10BCA0006FF00704EFE74FF0FF34ECE74FF0FF349D
:10BCB000F3E700BF68120020014B1878704700BFFF
:10BCC000D4120020014B5878704700BFD4120020D6
:10BCD00070470000044B9A7A0AB101225A70034B54
:10BCE0005B6903B118477047D41200206C0800202C
:10BCF00073B5224C6378002B33D008F085F9666861
:10BD00000546FFF7CDFB0644AE4214D2A37A93B1A9
:10BD1000E0228DF800208DF80130217AE36801934C
:10BD200001226846FFF7ECFB08B1073010D1002371
:10BD30006370A372656094F83430EBB1002384F82B
:10BD400034300F4B5B6BBBB102B0BDE8704018479D
:10BD500040F2DC510B4808F023FA0A4808F0E6F9F3
:10BD6000E8E794F83520002AE5D094F8360084F806
:10BD70003530FFF791FCDEE702B070BDD412002031
:10BD80006C0800200C13002037B5104D104CC8B1C2
:10BD9000C1B10123627200222860E16023700D4866
:10BDA0000D4B00924FF0FF3108F014F900250B48BD
:10BDB00025822022294605F05BFE6570A574A586C4
:10BDC00003B030BD00232B602370EFE7D0120020BA
:10BDD000D41200200C130020D5BC0008E81200206B
:10BDE0002DE9F0478E4C23788CB0002B56D0C278CA
:10BDF0000AB9837B13B1238A01332382437B002B4F
:10BE00004CD0E02A4AD10023A372876897F80080BB
:10BE1000B8F1220F27D8B8F1220F30D8DFE818F098
:10BE20004100FB0052005A0061006E0075008E0058
:10BE30009D00B400C7002F002F002F002F002F00FF
:10BE40002F002F002F002F002F002F002F002F007A
:10BE50002F002F002F002F002F002F002F002F006A
:10BE6000C900D000D400B8F17E0F00F0CC80B8F14A
:10BE70007F0F00F0DF80B8F17D0F00F0AB80A57A76
:10BE8000002D00F05B81674C637A3BB94FF47A7107
:10BE9000204608F085F9204608F048F90CB0BDE8C6
:10BEA000F087E36801220021A2721970A37AE16889
:10BEB0009818A0720620C854A37AE1689818A07256
:10BEC000CA54DCE7584B9B6A002BD8D001210220D2
:10BED0009847D4E77B7884F83630012384F83530EE
:10BEE000CDE704238DF804307B78003B18BF012395
:10BEF00001A88DF8083002F091F9C0E77878003891
:10BF000018BF012002F0DAFEB9E7484E0FCE01ADAE
:10BF10000FC50FCE0FC596E8070085E807007B78B0
:10BF20000A2BACD8424A12685268002AA7D00CA942
:10BF300001EB830353F82C0C9047A0E77878431E5D
:10BF4000012B9CD83A4B01381B6818BF0120207286
:10BF50009B68002B93D0984791E7E2680123082162
:10BF6000A3721170627A057BA17AAA4228BF2A4681
:10BF7000934284D285685A1CEB5CE56801334E1C01
:10BF8000A6726B54D3B2EDE7E3680122A2720922D4
:10BF90001A70A37AE268218A581CA072D154A27A3E
:10BFA000238AE1681B0A501CA0728B5467E7238226
:10BFB00065E705238DF8043001A802F0B7FB5EE7C2
:10BFC000194BDB6A98475AE7194B78781B686075FC
:10BFD000DB68BEE7037B072B7FF451AF06238DF8A8
:10BFE0000430B7F80130ADF808307B793A791B049A
:10BFF00043EA0223FA781343642253430393BB7941
:10C000008DF81030D8E73B2201A88DF804208DF878
:10C01000083002F003F9012384F834302FE700BF21
:10C02000D41200200C1300206C0800201C6F0108A3
:10C03000D01200202A2301A88DF8043001F0C6FF99
:10C0400094F80A90E6689DF808009DF809509DF85C
:10C050000A709DF80BC09DF80D309DF80E209DF8DC
:10C060000F109DF80CE009F1010A84F80AA006F807
:10C070000980354E94F80A903668D4F80C8009F19E
:10C08000010A84F80AA096F803A008F809A094F819
:10C090000A90D4F80C8009F1010A84F80AA096F8F5
:10C0A00002A008F809A094F80A90D4F80C8009F1CD
:10C0B000010A84F80AA096F801A008F809A094F8EB
:10C0C0000A9009F1010A84F80AA096F80080E6684F
:10C0D00006F8098094F80A80E66808F1010984F8F6
:10C0E0000A9006F808C094F80AC0E6680CF1010846
:10C0F00084F80A8006F80C70A77AE66807F1010C4C
:10C1000084F80AC0F555A57AE6686F1CA7727055C9
:10C11000A07AE568461CA6722954A17AE0684D1CF5
:10C12000A5724254A27AE168501CA0728B54A37A83
:10C13000E268591CA17202F803E0A0E6034807F088
:10C14000A7FF6570AAE600BFD01200200C130020E4
:10C1500070470000004870476C08002000207047BE
:10C160004FF0FF3070470000044B054A93F8183138
:10C17000022B18BF062382F890347047E81800207D
:10C18000B01E0020034BD3F8483313B15B6903B1F1
:10C1900018477047B01E0020034A137843F0040389
:10C1A0001370FFF7EFBF00BFAC1E00201FB50A4B96
:10C1B0008DF8090093F87C208DF80A2093F88C20E4
:10C1C00093F848000D3202A98DF8082003F0B0FC66
:10C1D000C0B205B05DF804FBE818002010B5074CAC
:10C1E00004F5806007F054FF94F81A3413B101236A
:10C1F00084F81934BDE81040FFF7C4BFB01E00201A
:10C2000010B50C4CD4F8403343F08003C4F84033ED
:10C2100094F81A3413B10020FFF7E0FF94F891343A
:10C2200023F0120343F0120384F89134BDE8104068
:10C23000FFF79ABFB01E00202DE9F041DFF8AC8077
:10C2400098F81831022B06460D4602D0284BDB6ABF
:10C25000984702F0E9FD044628B1022002F0DAFD19
:10C26000002002F0DCFD98F81831012B17D102F004
:10C27000DDFD074630B1002002F0CDFD002002F0C8
:10C28000CFFD3C4602F0D4FD48B1002002F0C4FDD1
:10C29000002002F0C6FDBDE8F041FFF765BF002CAD
:10C2A000F9D1144C94F8902494F81A34BAB90BB11B
:10C2B00084F84164304602F065FFD8F82C0007F09E
:10C2C000ADFED4F8B4339842E5D30B4807F0E0FE56
:10C2D00094F8913443F0100384F89134DBE70BB108
:10C2E00084F84154284602F04DFFF1E7E818002099
:10C2F000D0780108B01E00204822002073B5164CEB
:10C30000164D04F57A76EB6C95F8502095F9781077
:10C3100095F84800009603F031FC95F8303184F828
:10C32000FC3395F8480040F2012304F224423146E0
:10C33000A4F8FA3303F02EFC58B194F8243484F8AE
:10C340006A34074B00205B6B984794F8FB3384F802
:10C35000903402B070BD00BFB01E0020E81800206D
:10C36000D0780108074A10B5137843F00203137020
:10C37000FFF708FFBDE81040034B01220021022017
:10C3800007F058BBAC1E002095710108074A10B594
:10C39000137843F008031370FFF7F4FEBDE8104074
:10C3A000034B01220021022007F044BBAC1E0020F9
:10C3B000A57101082DE9F0410F4616461D4680463D
:10C3C00007F022FE0B4A0C4C1378278123F011034F
:10C3D00043F011031370C4E9000866812573FFF769
:10C3E000D1FEBDE8F041054B01220021022007F0FB
:10C3F00021BB00BFAC1E00205C240020B5710108E9
:10C4000013B507F001FE0D4B6C461860204607F08F
:10C410004FFD94E803000A4A0A4B83E803001378AF
:10C4200043F020031370FFF7ADFE074B01220021FC
:10C43000022002B0BDE8104007F0FCBA6C240020D6
:10C44000AC1E0020E8210020C2710108F8B5334D70
:10C4500095F81841012C06464BD0022C51D064B9F6
:10C4600038B9D5E91B0105F1740383E803002046C0
:10C47000F8BD01283DD0022801D00324F7E7284F5A
:10C4800085F8180107F5747EBEE80F0007F57A7C81
:10C49000ACE80F009EE8030095F8E9308CE8030053
:10C4A00087F8FB63E3B195F80031022B18D1D5F87A
:10C4B00004316B67C7F8EC3395F87D3095F80821A7
:10C4C00087F8F83395F88C3085F8782087F8F933B9
:10C4D00097F81B2487F8E82340F20133A7F8FA33D2
:10C4E000002387F81A340F4BDB6A9847FFF706FFE3
:10C4F000BDE702F0A4FC04460028B8D185F8186115
:10C50000B5E70028B9D1064B85F81801062283F853
:10C510009024044BDB6A98473446A8E7E8180020CB
:10C52000B01E0020D07801082DE9F04192B00646F7
:10C5300002F07AFC002840F05981AD4D95F8183191
:10C54000012B09D02B6BAB4C93B194F80431BBB1E8
:10C55000042B6FD0032003E002F068FC18B10F2019
:10C5600012B0BDE8F08102F063FC0028EAD0F6E7E3
:10C57000B5F82031D4F81C24013B53432B63E4E786
:10C580009D4803F00CFA002840F02C8194F80C31FF
:10C5900023802B6B0C930DF1180895F839308DF82A
:10C5A0003830404695F81C318DF83A3007F0A6FC3B
:10C5B000D5F82831009302AF98E80600D5F8243169
:10C5C000384607F032FC97E803000FAB83E803001E
:10C5D000EB6A0D9300238DF844302388ADF8463084
:10C5E00095F8303101228DF839201BB98DF844209F
:10C5F0008DF83930814B0093814B95F84800A3F1B9
:10C6000079020CA903F009FBC0B10B28A8D1D4F81A
:10C61000941499B1002EA3D0D4F84033794843F054
:10C620002003C4F8403307F0BBFD764807F07EFDD9
:10C63000002095E7704803F0E6F9A4E795F8487004
:10C6400095F9693095F9392095F87D106E4E384688
:10C6500003F0F0FA009641B2EB6C95F850203846A2
:10C66000183603F08BFA0096EB6C95F8502095F98C
:10C67000701095F8480003F081FAD4F8C413AB6D3C
:10C68000D4F8DC230B44C4F8B033EB6D1344C4F886
:10C69000B43394F80431042B07D02B6E0B44C4F848
:10C6A000B0336B6E1344C4F8B4330023089395F889
:10C6B000303183B108A802F095FC00284ED195F9DD
:10C6C000390094F837629DF82070FFF76FFD3E4403
:10C6D00080B2B04240D300238DF8133095F8393042
:10C6E0008DF8213095F838308DF82230D5F880302B
:10C6F0000993D5F884300A932388ADF82C3095F847
:10C70000303194F81B648DF82E3095F848003F4B7B
:10C710008DF820600DF1130208A903F043FA0123FC
:10C7200084F8413495F8393084F842349DF8133058
:10C7300084F84334D4F81C34C4F85064C4F8483442
:10C74000C4F8583402F076FB50B1D4F81C0402F05F
:10C7500083FB28B1102003E7082001E71320FFE640
:10C7600095F81831012B01D102F078FB02F065FB3E
:10C770000023059394F8043195F9395094F81B641B
:10C780009BB1042B7FF4E6AE05A802F067FE58BB10
:10C7900094F8183413B1059B013B0593164B05988B
:10C7A0003246E9B202F0C0FE02E0134802F090FE09
:10C7B000C0B9D4F8403394F80C11218043F002033F
:10C7C000C4F8403394F8183411480133DBB284F8CC
:10C7D000183484F845340F4B00259B6AC4F89854EC
:10C7E000984725E71120BBE61220B9E60E20B7E6F0
:10C7F000E8180020B01E0020B81F002018190020E3
:10C80000442300201822002068220020CC2200208F
:10C81000B21E0020D0780108F0B5504C504EB4F84C
:10C82000DC202287D4E92D0194F8B12084F8692016
:10C8300004F16C0282E80300D4E92F0104F17402D0
:10C8400082E80300B4F8C420A4F87C2091B0D4F8A6
:10C85000CC20D4F8C810C4F884200025D4F8D02007
:10C86000C4F888200123A4F82031C4F8801084F88B
:10C870003051A56284F81B5184F83A5084F81D5158
:10C8800084F81E51C4F83451C6F89854A6F81854C8
:10C8900086F81A54A4F838518DF8183004F5097345
:10C8A000039304F50A7394F84800A4F846510493DE
:10C8B00003A92C4B84F84551C4E94F55059303F067
:10C8C00045F9E36EC6F8D43394F87D3086F8E0334A
:10C8D00094F88C3086F8E1334FF48073A6F8E23395
:10C8E00086F8D05394F8303186F8E43306F574773F
:10C8F0000FCF06F57A740FC497E8030040F20123C6
:10C9000084E80300A6F8FA33D6F8483386F81B54B7
:10C91000CDE901551BB15A685B6901920293124B34
:10C920000793A3F148020892A3F1140209920F4A57
:10C930000B9229330A93A2F19C030C93A2F1980362
:10C940000D93131D0E9301A902F14C0307A802F5E4
:10C9500099620F9302F05DFA11B0F0BDE818002063
:10C96000B01E0020CC23002018230020CC1900206A
:10C97000F8B50D4F0D4C0E4E0D4607F089FB3B6B85
:10C98000984796F8480004F22442294603F002F939
:10C9900048B194F8243484F86A34706D7B6B9847FE
:10C9A000EB7C84F89034F8BDD0780108B01E0020EC
:10C9B000E81800200F4890F81B3480F8B8330E4B6D
:10C9C00093F8692080F8BB2393F87D2080F8C82372
:10C9D00093F88C2080F8C92393F8303180F8CC3359
:10C9E0000022A0F8CA2300F56E7100F56070FFF711
:10C9F000BFBF00BFB01E0020E8180020114890F80B
:10CA00009034EBB190F81B3480F8D0330E4BDA6ED3
:10CA1000C0F8D42393F87D2080F8E02393F88C208D
:10CA200080F8E12393F8303180F8E4334FF48072DA
:10CA3000A0F8E22300F5747100F56670FFF798BF67
:10CA4000704700BFB01E0020E818002070B5344CBD
:10CA50002421204605F00EF8636A984218BF6062F0
:10CA60004FF01C012F4814BF0125002505F002F8E6
:10CA7000636C984218BF60644FF480712A4818BFF5
:10CA800045F0020504F0F6FFD4F84831984218BF8B
:10CA9000C4F848014FF0D401244818BF45F00405FC
:10CAA00004F0E8FFD4F82032984218BFC4F82002FE
:10CAB0004FF000011E4818BF45F0080504F0DAFFEA
:10CAC000D4F82432984218BFC4F824024FF460719D
:10CAD000184818BF45F0100504F0CCFFD4F8A8356D
:10CAE000984218BFC4F8A8054FF01401124818BFA7
:10CAF00045F0200504F0BEFFD4F8C03598420F4B36
:10CB000018BFC4F8C005D3F8483318BF45F0400536
:10CB10002BB11B691BB12846BDE87040184770BD9A
:10CB2000E81800201019002030190020341A0020C5
:10CB30000C1B0020101B0020941E0020B01E0020A3
:10CB40002DE9F04F91B04FF00008012B05460F463C
:10CB500002928DF81580ADF8188003D8C84EC146F2
:10CB6000B94502D311B0BDE8F08F15F8090002F005
:10CB700077FA4844B842F5DC15F8093009F10104A8
:10CB8000023BE4B2112BEDD801A252F823F000BF12
:10CB9000D9CB00080BCC00080BCD000835CD000820
:10CBA000BDCD0008E5CD000857CE000889CE0008AD
:10CBB00005CF000865CB000865CB000863CF0008EF
:10CBC00065CB000865CB000821D0000849D00008DB
:10CBD0008DD00008CBD00008052002F0EDFA90B10E
:10CBE0000521002002F0ACFA2A5DA64B09F10304EE
:10CBF00009F102095FFA89F983F85C2415F8092024
:10CC000083F85D24E4B2A146AAE700238DF816302C
:10CC10008DF817308DF81C308DF82030B8F1000FEA
:10CC20006CD14FF0050896F87C208DF83920631EF2
:10CC300096F839208DF83B202B4496F838200D9338
:10CC40008DF83C2096F81A3196F868208DF83D2032
:10CC5000D6F82C218DF83A300C9273B37B1C1B1B39
:10CC6000DBB28DF8383008AB019307AB009396F830
:10CC700048000DF117030DF116020CA902F09EFFFA
:10CC80008DF8150000F00700072813D196F9392018
:10CC90009DF9163086F839309A429DF8173086F89B
:10CCA0003830B8BF01229DF81C30B8BF86F81D216E
:10CCB00086F868304FF0000909E00523D1E701222A
:10CCC0000DF11501032002F0DBF809F101095FFA0B
:10CCD00089F29DF82030B3FBF8F19142EFD823445C
:10CCE000DCB2631EDBB29F420DD9EA5C032A9AD004
:10CCF000A74288BF1C464FF0010884E709F10509E7
:10CD00005FFA89F4F7E71C46F5E72B5D012203F093
:10CD10000F0309F1020986F81B3102FA03F35FFAE7
:10CD200089F9A6F82031002206A9042002F0A8F80B
:10CD30004C4668E707238DF815302B5D96F84800C0
:10CD4000C3F3021203F00F038DF8303009F103032F
:10CD5000DBB28DF83120EA5C09F10403DBB209F1A2
:10CD60000504EB5C09F102095FFA89F91B0443EA47
:10CD7000022315F809201343642253430CA90D9391
:10CD800002F02BFF00F00703072BE4B28DF815002B
:10CD90000CD19DF8303086F8703086F878300D9BD5
:10CDA000F36673679DF8313086F869308DF81800A6
:10CDB000012206A9052002F063F824E7314BD3F8DD
:10CDC00048336BB11B685BB19847029B8DF8180024
:10CDD00003F03F038DF81930022206A90620EAE786
:10CDE000FF20F2E703238DF815302B5D8DF82430FA
:10CDF0000CAB089309F10303DBB209F10604EA5C0A
:10CE000096F8480009F10403DBB208A9EB5C1B04A7
:10CE100043EA022309F10202D2B209F10509AA5C30
:10CE20001343642253435FFA89F90C9300230D9353
:10CE300015F809308DF8383002F0D5FEC3B200285D
:10CE4000E4B28DF81530FFF6DEAE8DF81830012211
:10CE500006A90720AFE72B5D03F00F03012B4FF46A
:10CE60007A7238BF0123534309F10209B3651344B1
:10CE70005FFA89F9F365002206A9082056E700BF8A
:10CE8000E8180020B01E00202B5D96F84800C3F380
:10CE900040128DF81D2007A9C3F3001203F00F0301
:10CEA0008DF81C208DF81E3002F0A3FE09F1020956
:10CEB00001305FFA89F93FF43BAFBDF81C30914A6D
:10CEC000A6F87C309DF81E309DF81C40D05CF5F72C
:10CED00021F80223C6F880000CA996F848008DF8C6
:10CEE00030308DF8324002F023FE96F93930089048
:10CEF00040B29842B8BF184686F83900002206A909
:10CF0000092013E703238DF815302B5D8DF83030A1
:10CF100009F10303DBB209F10504EA5C96F8480065
:10CF200009F10403DBB209F10209EB5C5FFA89F94C
:10CF30001B0443EA022315F80920134364225343D8
:10CF40000CA90D9302F05BFEC3B20028E4B28DF889
:10CF50001530FFF658AE8DF81830012206A90A20C8
:10CF600029E7092002F028F9DFF89CA1002854D015
:10CF70000921002002F0E4F80023ADF8263009F181
:10CF80000203DBB24FF47A71EA5C09F10303DBB20E
:10CF90000DF1300BEB5C1B0443EA02232A5D1343C3
:10CFA00009F10402D2B209F1060409F10509AA5CEB
:10CFB0005FFA89F943EA026315F8092003934A43AB
:10CFC00012125846ADF8242006F072FF039B03F1BD
:10CFD000965303F5A91303F5EC530893DAF83C33A1
:10CFE00000930DF1200999E80600DAF838330AA811
:10CFF00006F01BFF0B9B00939BE806000A9B48462C
:10D0000006F0F8FE99E8030006F02AFF01F021FF80
:10D010000123E4B28AF83834F5E58AF83804F2E5F9
:10D020000C2002F0C9F800283FF4EDAD0C210020DF
:10D0300002F086F8344B93F89034043B012B7FF6D2
:10D04000E2AD01F002FFDEE509F10203DBB22A5D89
:10D05000E95C09F10303DBB209F10504EB5C09F1BA
:10D0600004095FFA89F91B0415F8090043EA012352
:10D0700013436421594300F00F0001F0E7FEE4B2CE
:10D080008DF81800012206A9112094E60D2002F067
:10D0900093F800283FF4B7AD0D21002002F050F8BE
:10D0A00009F10203DBB2194AE85C2B5D126809F151
:10D0B000040409F103095FFA89F943EA002015F82D
:10D0C0000910E4B201F0C4FE9DE52A5D09F10203F6
:10D0D00009F1040409F10309DBB25FFA89F9E95C9B
:10D0E00015F809301B0443EA012313436420584315
:10D0F00001F0B0FEE4B28DF81800012206A9132059
:10D1000059E600BFCF710108B01E00205C2400204A
:10D110000E4B93F89124920703D593F88F24012A9C
:10D1200008D90B4991F81A2122B18A6A501C18BFFC
:10D1300001328A620022A3F8182483F81A24D3F853
:10D14000402322F00202C3F840237047B01E0020A3
:10D15000E818002070B5184C184D04F55A7006F008
:10D1600097FFD4F84033D4F89804D5F8906023F0B2
:10D170002003C4F8403338B106F050FF864203D292
:10D18000002385F83A3070BD0120FFF7CDF9002863
:10D19000F9D00B28F7D095F8393084F842340920BB
:10D1A00094F8183484F8453484F8410401F0EAFF17
:10D1B000BDE87040FFF7ACBFB01E0020E8180020AB
:10D1C000094BD3F84023012A0AD008490978C90736
:10D1D00008D43AB993F89204013818BF0120704777
:10D1E0000020704701207047B01E0020AC1E0020B8
:10D1F000034BD3F84003431E58425841704700BFC9
:10D20000B01E00202DE9F04FA9B0EFF3108272B6E6
:10D21000DFF8F4820021D8F80030C8F8001082F35B
:10D220001088BA4C002B00F0E480DAB29B0603921F
:10D2300064D5B74D95F81831022B02D0B54BDB6A97
:10D240009847EFF3108972B6B34F06F0DDFE3E68E3
:10D25000D4F8B013361A3144B04806F0A1FFAF48F5
:10D2600006F064FFD4F8B413AD48314406F098FFDB
:10D27000AB4806F05BFF89F3108894F81A34002B52
:10D2800000F06D81152312A995F848008DF84830FB
:10D2900002F04EFCD4F8B4130F900144A14806F0FC
:10D2A0007FFFA04806F042FF3B6894F81B24EB6226
:10D2B0000DAF38468DF870201D9306F01FFED5F88F
:10D2C0002831009306AE97E80600D5F824313046A1
:10D2D00006F0ABFD96E803001FAB83E80300D4F82B
:10D2E0001C341E9395F8303195F84800003B18BF68
:10D2F00001231CA98DF8713002F023FC039BDF068B
:10D300004BD5834DDFF820A2D5F8E420BAF90A30D6
:10D31000059298F800200493002363F300020A9317
:10D3200088F8002084F84434049AA4F8223484F85D
:10D330002534C4F82834A4F82C3484F82E34C4F8E6
:10D34000303484F82034C4F8343484F83834C4F8E1
:10D350003C34704B9AF90C90A4F88C2494F89024E7
:10D36000DB6A84F88E9484F88F24DAF80470BAF8B3
:10D370000860984794F88F3413B9694806F088FE1E
:10D380003146384601F04EFD8346002800F0EA8021
:10D39000049BA4F87E3484F88094039B19071AD563
:10D3A0005B4B93F81831022B02D05A4BDB6A98473B
:10D3B0000220FEF7D9FE84F8410401F0E3FE94F860
:10D3C0001A3413B1012384F8193494F8913443F0DA
:10D3D000100384F89134039B5A0703D506210520D6
:10D3E000FEF72AFF039B9B0703D504210320FEF7CA
:10D3F00023FF01F035FD94F89124D7065FD5002373
:10D4000084F89234D4F840331E0644BF23F08203DC
:10D41000C4F8403312F0050F00F0FC820B2001F03D
:10D42000CBFE002800F0F68294F89134DD0700F17D
:10D43000F182580740F10883D4F8403323F0020307
:10D44000C4F84033D4F8402382BB94F8915415F0CB
:10D4500001011EBF2B4662F3000384F8913494F857
:10D4600091345E0744BF6FF3820384F89134012343
:10D4700084F8923421B1D4F844332C481B6898477F
:10D480006D070BD52A4801F0A3FE01F0D1FE28B1AB
:10D4900094F8913443F0040384F8913401F0CEFC05
:10D4A00094F891346FF3041384F89134012384F8D1
:10D4B000923494F8913443F0200384F8913494F832
:10D4C000913418070AD56FF3C3031A4984F89134CD
:10D4D000D4F84433A1F12400DB68984794F89134E0
:10D4E00099070AD56FF34103124984F89134D4F8AF
:10D4F0004433A1F16C005B68984794F89034022B98
:10D500001AD1FEF7FBFE17E0AC1E0020B01E002073
:10D51000E8180020D07801086C2400203022002078
:10D5200048220020B02200205C240020F0220020AD
:10D53000042300203C23002094F891349A0640F103
:10D54000C6826FF3451384F89134D4F84033002B2E
:10D5500040F0BD8229B0BDE8F04FFFF777BA84F8FC
:10D560004134A1E695F81821012A0CD101F05EFCA6
:10D57000804668B1584601F04EFC584601F050FC18
:10D58000042384F88F347EB9012384F8213450E1D8
:10D5900001F04EFC0028F6D0404601F03DFC40462C
:10D5A00001F03FFC0523ECE73B7804935B09013B6A
:10D5B000062B00F21882DFE813F007001602950030
:10D5C0001602920016020702102EDDD995F83031AE
:10D5D0001297F6B28DF84C60002BD5D11CA804F040
:10D5E0005DF912AA1CA9FF2002F0B2F89DF858308C
:10D5F000C3F3030307468DF82C3095F8480095F8DF
:10D600007D308DF82D3007220BA902F0A4FA002FEF
:10D610005DD100285BD09DF853309DF852201599BC
:10D62000C5F8E4101B0443EA02239DF851200220B0
:10D630001343C5F8E03004F03FF99DF8583095F8F1
:10D64000480085F82E71C3F30212C3F3030385F873
:10D65000703085F878309DF8593085F86920012BB5
:10D6600038BF01234FF47A725343AB651344EB6523
:10D670000DF15A034FF001081093113E94F81B343A
:10D680008DF83C300FA985F868808DF8446002F071
:10D690006AFA0223404685F8303101F08DFD18B159
:10D6A0004146384601F04CFD94F88F34012B00F2CE
:10D6B000A88194F81A34002B40F09B8194F891349F
:10D6C00043F0100384F89134FEF74EFD65E6012027
:10D6D00001F072FD0028E7D001210720E2E70123D5
:10D6E00084F8203495F87D308DF82E3094F8243469
:10D6F0008DF82D3095F88C3095F848000D330BA936
:10D700008DF82C3002F014FAA6F10D031BB209902B
:10D7100023EAE37300B283423FF736AF0B2E7FF666
:10D7200033AFBB4B25931CA8FF231C978DF8746067
:10D730008DF8983002F0D8F8074600287FF424AF1F
:10D7400095F81831012B13D101F070FB002873D02C
:10D75000384601F060FB384601F062FB04239DF877
:10D760007C101E9884F88F34C1F3001101F077FB10
:10D770009DF87C301E99C4F8341413F00F0203D0C6
:10D780009DF89000002863D19DF89800002862D091
:10D79000002A7FF4F9AE9DF89020002A0CBF4FF0CC
:10D7A00002084FF0030800220A92D5F8EC209142BB
:10D7B00054D195F8E910002950D0D5F80C1195F8FE
:10D7C000EAB009680A9195F81811022902D10321DB
:10D7D00084F88F14B8F1030F7FF4D6AE13F0600F06
:10D7E0007FF4D2AE0592012795F82E31BBF1000FE0
:10D7F00037D0BBF1010F38D1012B34D16FF00906BE
:10D8000046FA08F606F00106C6F10206F6B2BDF8C1
:10D810007E100AAA304601F02DFE40B307280CBF47
:10D820000823012384F821340A9BC4F83034C4F857
:10D830006C34FEF7E5FCB0E501F0FAFA002897D069
:10D84000384601F0E9FA384601F0EBFA052386E79D
:10D850004FF00008A7E74FF00108A4E74FF0010BD5
:10D86000C2E70426D3E70326D1E70123DAE71CAB9E
:10D87000009305990A9B3246584601F0BBFE20B141
:10D8800002280CBF0A230B237FE60A9BC4F830341E
:10D89000C4F86C349DF87C3084F82104C3F3401341
:10D8A00084F82E3484F8443494F88F3484F8227445
:10D8B000012B9EBF0122A86285F81E21012FC4F80A
:10D8C000280484F82C0484F8410438D1022284F816
:10D8D000202495F83A20002A4AD19DF87C20D606CB
:10D8E00046D4012B94F840149DF87C2005D80129DA
:10D8F00001D1900601D501F05FFBB8F1020F94F859
:10D900008F3443D0B8F1030F0AD09DF87C10B8F1E2
:10D91000010F4A4601F00F0120A83BD0FFF710F994
:10D920009DF8903084F82334259BC4F828349DF862
:10D93000983084F82C34012384F82D3430E0049A94
:10D9400002F0E002A02A1BD195F82E11012285F8E1
:10D950003A2009B927996963012B84F8202407D953
:10D96000D5F89020C4F83C24DAF80020C4F89824B4
:10D9700095F81821002AB4D1012284F82524B0E7B3
:10D98000002285F83A2084F82024A6E79DF8981014
:10D9900025984A46FFF7D4F89DF8903084F8233450
:10D9A0009DF89020E02A08D195F81F312BB984F812
:10D9B0002324C4F82834A4F82C3494F8913443F088
:10D9C000020384F891346FE6114D013EB2B2791C26
:10D9D000284604F039F80323A4F82034C4F8285466
:10D9E00084F82C64E9E7012384F82134FEF708FC6D
:10D9F0005AE694F84434002B3FF460AE0020FEF762
:10DA0000EDFB94F88F34022B3FF45EAE56E600BF78
:10DA1000E820002094F89134590715D5012001F031
:10DA2000CBFB60B1012001F09DFB08B984F818041C
:10DA3000D4F8403323F00203C4F8403304E0062056
:10DA400001F0BAFB0028F3D194F89134DA077FF59E
:10DA5000F9AC94F840240AB1032A18D11D4A94F86D
:10DA6000181492F86820914205D29B0723D594F8A8
:10DA70008F34012B1FD8184806F00AFBD4F8403326
:10DA800023F02003C4F84033FFF742FBDAE4012A15
:10DA900011D194F81924002A3FF4D4AC0D4A94F81B
:10DAA000181492F868209142E5D29F0703D594F8A4
:10DAB0004434002BDFD194F8913400206FF3041329
:10DAC00084F8913484F81904FFF744FBBAE429B0D0
:10DAD000BDE8F08FE8180020182200202DE9F04F53
:10DAE00089468DB090460746002800F08F810029B6
:10DAF00000F08C810368002B00F088814368002BC4
:10DB000000F084818368002B00F08081C368002BC3
:10DB100000F07C81104602F007F8002800F07881C0
:10DB2000BD4CBE4D384601F0C1FA40F2C45200214E
:10DB3000204603F09DFF40F21C520021284603F0CE
:10DB400097FFB74BC4F82C3104F50973089304F51B
:10DB50000A7300264046099308A9B24B84F848800E
:10DB60000A9384F8186184F88C608DF82C6001F0B9
:10DB7000EDFF0F2306A994F848008DF8183001F046
:10DB8000D7FF801B18BF01204FF00A0B84F81C013F
:10DB900006A994F848008DF818B001F0C9FF4FF0BD
:10DBA000060A84F8DC0006A994F848008DF818A04D
:10DBB00001F0BEFF102384F8DD0006A994F84800A8
:10DBC0008DF8183001F0B4FF1123C4F89C0006A9A9
:10DBD00094F848008DF8183001F0AAFF1223C4F819
:10DBE000A00006A994F848008DF8183001F0A0FFB5
:10DBF0001323C4F8A40006A994F848008DF818303F
:10DC000001F096FF1423C4F8A80006A994F8480070
:10DC10008DF8183001F08CFF1623C4F8AC0006A96B
:10DC200094F848008DF8183001F082FF172384F82B
:10DC3000B10006A994F848008DF8183001F078FF7B
:10DC400018230DEB0301C4F8B400C4F8BC0094F829
:10DC500048008DF8183001F06BFFC0B21D2384F826
:10DC6000B80084F8C00006A994F848008DF8183070
:10DC700001F05EFF1E2384F8C40006A994F8480052
:10DC80008DF8183001F054FF1F2384F8C50006A951
:10DC900094F848008DF8183001F04AFF2023C4F8AA
:10DCA000C80006A994F848008DF8183001F040FF2C
:10DCB0000B23C4F8CC0006A994F848008DF818305E
:10DCC00001F036FF0C2306A9A4F8D00094F8480010
:10DCD0008DF8183001F02CFFD4F89C306365D4F82F
:10DCE000A030A365D4F8A430E365D4F8A830236647
:10DCF0004FF00108D4F8AC300590A4F8D200636668
:10DD000084F8B080C4F894B084F898A0C4F84CB0FB
:10DD100084F850A084F8688084F81F81C5F848937F
:10DD2000FEF77AFD404B009632464FF0FF3105F585
:10DD30005A70C5F84473C4E90B6684F8198185F8F4
:10DD40009164C5F8408306F045F9384B0096324699
:10DD50004FF0FF3105F5607006F03CF9344B00964A
:10DD600032464FF0FF3105F5667006F033F902AF29
:10DD7000304B009632464FF0FF3105F5806006F0DB
:10DD800029F9384606F0BAF897E8030004F59273CB
:10DD900083E80300284B294F1E60294BC5F84C33FC
:10DDA000284BC5F85433284BC5F85C33274BC5F8CE
:10DDB0005033274BC5F8583305F553703B689847E7
:10DDC00004F5A67003F088FB20B1112630460DB093
:10DDD000BDE8F08F204601F01DFB0028F5D101F0D1
:10DDE00041F8B8B91B4801F067FB06460028ECD1A2
:10DDF0007B69984703F006FEBB6D94F819019847BC
:10DE0000FB6A9847012385F89234DFE70326DDE7B4
:10DE10000926DBE71326D9E7E8180020B01E00200A
:10DE200000040001CC23002055D10008B5C900082A
:10DE3000FDC90008DDC10008AC1E0020D078010833
:10DE400001C40008B5C3000899C100088DC30008CB
:10DE500065C30008D019002008B5034B0020C3F8A3
:10DE60004003FEF781F908BDB01E002010B5FFF792
:10DE7000A7F90A4C60B90A4B93F81831022B02D16A
:10DE8000084BDB6A98470123C4F84033002010BDDB
:10DE9000D4F84003013818BF0120F8E7B01E002075
:10DEA000E8180020D078010838B5134C04F55A70F2
:10DEB00006F0EEF804F5607006F0EAF804F5667016
:10DEC00006F0E6F804F5806006F0E2F800F0B5FF31
:10DED0000A4B0025DB6A9847C4F84053FEF7B6FDAD
:10DEE0000749084840F2C45203F0AEFD0123C4F8CC
:10DEF0004033284638BD00BFB01E0020D07801084E
:10DF0000E81800202413002070B52E4B8AB0054677
:10DF100093F8DD008DF8090093F8DC008DF80A0015
:10DF200029489A6A90F81804039200268DF80B008D
:10DF300004960C46002940D00692D3F88820079218
:10DF40001A8F93F81A118DF8151052BAADF82020D7
:10DF500093F87C2093F848308DF8243003AB8DF88B
:10DF600022008DF8232000930DF10A020DF10B031E
:10DF70000DF1090105A88DF8146000F0DDFE9DF992
:10DF80000900FEF713F9607004A801F02BF8B0B98E
:10DF9000049A0F2A0DD863789A420AD81544AB42E6
:10DFA000A3EB02012CBF002001202170C0000AB0A9
:10DFB00070BD002323700820F9E70320F7E7132042
:10DFC000F5E700BFE8180020B01E00201FB504468A
:10DFD000002800F012810078412800F20881DFE873
:10DFE00010F0420048004D00520056005A005F00F9
:10DFF00006010601060106010601060106010601E9
:10E0000066006A006E0079008000830086008B0045
:10E0100089008D009100940097009A009D00A00057
:10E02000AF00B300BB00B700BF00C200C600CF0006
:10E03000CB00CD000601D300060106010601060152
:10E040000601060106010601060106010601060198
:10E05000060106010601DB00DF00E300E800EC003A
:10E06000F000F400FD00674B93F81831237104B001
:10E0700010BD644B93F83031237102E0606803F007
:10E08000C7FB0020F3E7606803F008FCF9E75D4B8D
:10E0900093F81A31F0E75B4BD3F8E0306360F0E7B8
:10E0A000584B211D93F8300103F010FCE9E7554B64
:10E0B00093F81931E0E7534B93F88C30DCE71C23DD
:10E0C0008DF808304F4B02A993F8480001F030FD5D
:10E0D0006060D6E74C4B043493E8030084E8030007
:10E0E000CFE74A4B0434F7E7494B0434F4E7494B94
:10E0F0000434F1E71A23E3E71923E1E7414B93F8EE
:10E100006830B9E73F4B5B6DC8E73E4B9B6DC5E799
:10E110003C4BDB6DC2E73B4B1B6EBFE7394B5B6E85
:10E12000BCE702238DF80830364B02A993F87C2017
:10E1300093F848008DF80A2001F0FAFC2071A0E75E
:10E14000304B93F8DD3097E72E4B93F8393093E757
:10E150002C4B93F8DC308FE72A4B93F838308BE761
:10E16000284BDB6C9AE7274B93F8503084E7254B1C
:10E17000D3F88430636084E7224B8FE7264B8DE72A
:10E18000204BD3F8CC30F5E71E4BD3F82C3163602D
:10E1900001F05CFDA06074E71A4BD3F890307DE786
:10E1A000184B93F81F3167E7164BB3F88830A380FC
:10E1B00067E7144BB3F88A30F9E7124BB3F8D03065
:10E1C000F5E7104BB3F8D230F1E70E4B93F8482047
:10E1D0000AB1062A13D1B3F8A035E8E7094B93F842
:10E1E00048200AB1062A0AD1D3F8A43556E72046BA
:10E1F00004B0BDE8104000F024BE032037E718202B
:10E2000035E700BFE8180020541900209C190020B1
:10E210005C190020A4190020241300207FB50446B7
:10E2200010B9032004B070BDA44DD5F840339A074F
:10E2300000F171820278412A00F26A82DFE812F06E
:10E240004200480056005C00600065006A007700EC
:10E25000820088008E0094009A00A000A600AC0006
:10E26000B6006802BB00DD00F000170139012A0189
:10E2700044014D015101550159015D0168026101DF
:10E2800073019B018901AD01B301BA01BF01C40152
:10E2900068022A026802680268026802680268026C
:10E2A000680268026802680268026802680268021E
:10E2B0006802680236023B02400245024A024F02EF
:10E2C00054025E020079FEF7C1F80028AAD105E0E9
:10E2D0000379022BA5D07A4A82F8303195F891342F
:10E2E00043F0200385F8913400209BE7406803F059
:10E2F00081FA0028F2D094E7406803F0BFFAF8E70B
:10E300006F4B027983F81A21E8E76D4B4268C3F836
:10E31000E020E3E76A4E416896F8300103F0CCFA5A
:10E3200000287FF47EAF6368C6F8E430D6E7416822
:10E3300000293FF476AF002001F0EEF90028CDD09F
:10E3400011206FE7416800293FF46BAF0120F3E72C
:10E35000416800293FF465AF0820EDE741680029D6
:10E360003FF45FAF0920E7E7416800293FF459AF68
:10E370000C20E1E7416800293FF453AF0D20DBE7B3
:10E38000416800293FF44DAF0E20D5E741680029D0
:10E390003FF447AF0F20CFE74A4C494B007983F851
:10E3A0001901A36D9847E36A984797E7444B0279B0
:10E3B00083F88C2092E7424E037A8DF8043096F869
:10E3C000480096F87D308DF80530072201A901F04C
:10E3D000C2FB00283FF425AF636896F8480001931C
:10E3E000002201A901F0B7FB00283FF41AAF6C36F8
:10E3F000D4E9010186E8030070E7314E037A8DF815
:10E40000043096F8480096F87D308DF805300722E4
:10E4100001A901F0A0FB00283FF403AFB436E7E701
:10E42000274E037A8DF8043096F8480096F87D3030
:10E430008DF80530072201A901F08DFB00283FF47B
:10E44000F0AED4E9010106F1740383E8030096F805
:10E450001831022B7FF442AF96F83031002B3FF495
:10E460003DAF184BDB6A9847FDF748FF36E7144E7F
:10E47000037A8DF8043096F8480096F87D308DF8D0
:10E480000530072201A901F066FB00283FF4C9AE60
:10E49000BC36ADE74368029301238DF80C30084B7E
:10E4A00002A993F8480001F063FB00287FF416AF3F
:10E4B000B7E6436802930023EFE700BFB01E0020D9
:10E4C000E8180020D078010803795A1E0E2A3FF67A
:10E4D000A8AE934A82F8683000E7914B42685A65CB
:10E4E000FCE68F4B42689A65F8E68D4B4268DA6528
:10E4F000F4E68B4B42681A66F0E6894B42685A662E
:10E50000ECE6874C037994F848008DF80430062235
:10E5100001A901F020FB00283FF483AE9DF80430F0
:10E5200084F8DD30DAE67E4C03798DF8043094F817
:10E53000480094F87C308DF80630052201A901F0DE
:10E540000AFB00283FF46DAE9DF8043084F83930A2
:10E55000C4E6734C037994F848008DF804300A221D
:10E5600001A901F0F8FA00283FF45BAE9DF80430F1
:10E5700084F8DC30B2E66A4C037994F848008DF8F0
:10E580000430092201A901F0E6FA00283FF449AE5F
:10E590009DF8043084F83830A0E6614B4268C3F837
:10E5A0009420DA649AE65E4B027983F8982083F827
:10E5B000502093E65A4B4268C3F884208EE6584BAD
:10E5C0004268C3F8CC2089E6012B40F0A480554C6A
:10E5D0002421204603F04EFA636A984201D01720A6
:10E5E00020E61C2104F1280003F044FA636C9842F1
:10E5F000F5D14FF4807104F1480003F03BFAD4F8F0
:10E6000048319842EBD1D42104F5A67003F032FAD8
:10E61000D4F820329842E2D1002104F5097003F0C9
:10E6200029FAD4F824329842D9D14FF4607104F514
:10E630000A7003F01FFAD4F8A8359842CFD11421FC
:10E6400004F2AC5003F016FAD4F8C0359842C6D1A3
:10E65000334E2146304640F2C45203F0F5F92046CD
:10E6600040F2C452002103F003FA95F81B3485F8F8
:10E67000E833736FC5F8EC3396F87D3085F8F833DE
:10E6800040F20123A5F8FA33274B96F819019B6D48
:10E69000984723E68379012B3FF6C3AD204B4268B0
:10E6A0004068C3F82C2100F0D1FE47E61C4B4268BD
:10E6B000C3F8902012E61A4B027983F81F210DE669
:10E6C000174B8288A3F8882008E6154B8288A3F8A8
:10E6D0008A2003E6124B8288A3F8D020FEE5104B77
:10E6E0008288A3F8D220F9E50D4B93F848200AB1AF
:10E6F000062A12D1A288A3F8A025EFE5084B93F8CB
:10E7000048200AB1062A08D16268C3F8A425E5E5C5
:10E7100000F099FBD9E5012084E5182082E500BFCF
:10E72000E818002024130020D07801082DE9F043D8
:10E7300087B00023ADF800300646002800F0ED80D9
:10E740000361FEF73DFD20B10124204607B0BDE87E
:10E75000F08300F073FD0028F6D100F069FD01465A
:10E7600018B96F48142203F083F96E4D95F891346F
:10E77000012243F0040385F8552485F89134337859
:10E780008DF804300021013B8DF80520ADF806100E
:10E790000C2B00F2BA80DFE803F007B8B8B8788134
:10E7A000B8B88FB8AC99A800D5F8407317F0200717
:10E7B000CAD196F80480B8F1020F45D1DFF868811C
:10E7C0005A4CFEF729F896F9051098F848003A4691
:10E7D00001F01BFA88F83900B37988F838303846E8
:10E7E00007238DF80530FDF731FEFF2304F5867011
:10E7F000A5F80C31C5F8084185F8047103F04EF80E
:10E8000004F58A7003F004F83846FDF78DFE0446DF
:10E8100040B196F9051098F84800012201F0F5F989
:10E8200088F83900D5F894343361002C71D000F0A9
:10E83000FFFC002889D195F8913485F81A0460F31B
:10E84000820385F8913480E7B8F1010F4FF002049C
:10E85000E8D1DFF8D4908DF8144099F8480089F891
:10E860001D7102A901F072F9337989F830318DF800
:10E8700005708DF80680FDF785FC95F8913443F01E
:10E88000100385F891340024CCE700226946022069
:10E8900000F0F6FA0028F6D01324C3E7244BB28820
:10E8A000DB6B96F90C10B0689847D5F8403343F00D
:10E8B0000203C5F84033E6E702A90D2000F060FB33
:10E8C0000028E0D0002269460D20E1E7164B93F8BE
:10E8D0001831D3B9347904F0070000F0ADFA8DF89F
:10E8E0000040012269461020D2E70022694612202A
:10E8F000CEE78DF8072000F090FA044638B900F012
:10E9000089FA204600F08BFA8CE702248AE701247A
:10E9100088E701A800F0DEFB17E7032415E700BF36
:10E9200004230020B01E0020E8180020B21E0020A2
:10E93000D07801082DE9F04F99B08046059118B9BB
:10E94000032019B0BDE8F08F00230361FEF738FC07
:10E950000646002840F0AB8045460FCD0EAC0FC4F4
:10E960005A4C98F800A0B8F80C7098F90EB0142220
:10E9700004F58860314603F07BF8012284F84124D5
:10E98000534C94F83021022A35460BD194F81821C3
:10E99000022A07D194F81E2122B9BAF1010F38BF1B
:10E9A0004FF0010ABAF1010F2DD0BAF1030F2CD0AC
:10E9B000BAF1000F35D102229DF83C30DDF84090CD
:10E9C000029362F34715012694F87C108DF83210FB
:10E9D00002220CA994F848008DF8302001F0A8F824
:10E9E00094F81A3194F830C194F81D1140B2022203
:10E9F000002B6FD0BCF1010F65D1002963D1002E2F
:10EA00006DD1104627E00422D6E70023DDF83C90C4
:10EA1000BDF840709DF942B0029365F01F050126D4
:10EA2000D2E74FF0000BD946CDF808B0CCE74FF055
:10EA3000010084F81A04DDE005F29A420BA900F007
:10EA4000DDFA002800F020811320049B33871F4B40
:10EA5000002283F81A241D4BD3F89434C8F81030E0
:10EA60006FE705F29A452A460BA900F0C7FA00287D
:10EA7000EAD10B9B84F82801C4F82C5184F830317A
:10EA800002E1B9F1000F00F0FF80002A00F0FC80E5
:10EA90004946E01C02F0D8FF94F837320133238056
:10EAA000F2E01220D1E70220CFE70720CFE70120D4
:10EAB00047E7064B93F8912483F840A442F0010203
:10EAC00083F89124C7E7EEB90220C4E7B01E002006
:10EAD000E8180020002E94D05845B8BF584694F846
:10EAE0007C308DF82000052294F848008DF8223003
:10EAF00008A901F030F800283FF422AF9DF820303B
:10EB000084F83930694A6A4BD2F89804D3F89040B7
:10EB100038B105F083FA664B84423CBF002283F88B
:10EB20003A20198F1A8F93F830010491996A09914C
:10EB300052BA0028B9D093F81B0100B9186393F8B2
:10EB40001801ADF85820013893F87C2093F81A4149
:10EB50001491D0F1000BD3F888108DF85B204BEBAB
:10EB6000000B93F8482093F83A0093F868308DF83A
:10EB70005A3009AB00934F4B03904FF001008DF8D2
:10EB80004C0015918DF85C20A3F12F01A3F1300208
:10EB900013A88DF84D4000F0CFF8039B4FEA0B1BF4
:10EBA0004BEA431B00264BEA801B4BEAC413B145DA
:10EBB0003E4C039308BF37463A46494604F59C70DD
:10EBC000CDE90A669B46268084F81A6402F03CFF71
:10EBD000E9B2A570C5F34215FAB2042D344E039B79
:10EBE00084F837223FF423AF072D3FF44AAF022DBC
:10EBF0007FF459AF304D84F80D110420029984F848
:10EC00000401FF2084F80C0184F8281184F81431E1
:10EC1000D6F8E410C4F8085105F59B730AA8C4F8A7
:10EC2000101184F83021C4F82C3100F017FC0028B2
:10EC30007FF437AF0A9BA4F844040BA8A4F816315C
:10EC4000C4F84C3400F0CEF900287FF4FDAE0B9BE5
:10EC5000D3B196F93900FDF7A9FA94F83732002BB1
:10EC60003FF4FFAE0B9B0F2B3FF6E6AE05F58B7224
:10EC70000BA90F2000F0C2F900287FF4E5AE0B9B32
:10EC800063F3030B84F814B10598FDF74DFC0028DD
:10EC90007FF4DBAE099B86F83A00B36200F07EF9A0
:10ECA00000283FF406AF1320D1E600BFB01E0020BD
:10ECB000E818002050190020B21E002037B50B4D77
:10ECC0008DF8040004460F2295F8480001A900F0D1
:10ECD00042FF40B1064A85F81C4192F8913443F056
:10ECE000200382F8913403B030BD00BFE818002043
:10ECF000B01E002010B5FFF7B9F8044688B90A48DD
:10ED000005F0C6F9094805F0C3F9094805F0C0F94E
:10ED100000F093F8FDF780FD064BDB6A984720462C
:10ED200010BD0124FBE700BF182200203022002084
:10ED300048220020D07801082DE9F04F8BB04778A9
:10ED40000093149B90F90C8090F90D6090F80E9050
:10ED50008B464168196004469246002F57D0022323
:10ED60008DF8103004A9C37B007C8DF8123000F0C0
:10ED7000DFFEB4F808C0618943B260689845454633
:10ED80006144B8BF1D46604534BF00270127884253
:10ED900009D30A218DF81010207C019304A900F0FA
:10EDA000C7FE019B46B2B4F808C0608961680CEBED
:10EDB000400E714520D3A1EB0C01B1FBF0FC00FB30
:10EDC0001C11C9B998450ADC237833B10223207C91
:10EDD0008DF8243006A900F0B9FE4FF00109212377
:10EDE0008DF81030207CE37B8DF8115004A98DF84C
:10EDF000123000F09DFE45B2009B8BF80050384663
:10EE00008AF8006083F800900BB0BDE8F08F4546AB
:10EE1000F2E77047704770477047002070477047AF
:10EE200070477047002070470020704700207047EF
:10EE300000207047002070477047704770470220DD
:10EE400070470220704702207047704700207047CB
:10EE50007047704700207047002070477047704728
:10EE60007047000010B5054C4FF403722046002196
:10EE700002F0FEFD0020C4E9000010BD7024002057
:10EE80002DE9F8438146174600293FD0244B002541
:10EE900003F1010C1A462801103312F8018FB8F162
:10EEA000000F36D19A42F8D11E4E33680BB9C6F81E
:10EEB00000C073680BB1C3F800C0331800240135DB
:10EEC0009C6083F80C900D302B01BAB206EB05154F
:10EED0003044F750C6F804C002F0B6FDB9F1110F86
:10EEE0004FF0000398BF104C6B71D6F8083298BFF2
:10EEF00024FA09F403F1010398BF04F001043B4430
:10EF00002C71C6F808324046BDE8F8834FF001087E
:10EF1000F9E70135202DBBD14FF00208F3E700BF20
:10EF200077240020702400202007020010B510B3C1
:10EF3000124A1368984204D103681360002304E066
:10EF40000B4613B119688842FAD15168884208BF4C
:10EF500053600BB101681960D2F808328168013B37
:10EF600000245B1A04602146C2F80832102202F025
:10EF70007FFD204610BD0120FCE700BF702400206B
:10EF8000054B1B6813B11A798242FAD1002B0B6032
:10EF90000CBF0320002070477024002010B5054BE3
:10EFA000186800B910BD037B04680BB9FFF7BEFFFA
:10EFB0002046F6E77024002038B5084B084C186846
:10EFC00000B938BD03790568112B05D824FA03F37D
:10EFD000DB0701D5FFF7AAFF2846F1E770240020E0
:10EFE0002007020028B1044BD3F808320360002048
:10EFF00070470120704700BF702400202DE9F041C8
:10F0000007460E4615463AB331B3144B1C6800232D
:10F010002CB93046FFF7E6FF0020BDE8F081A2687A
:10F02000F91A0132914210D32279EA54581C2289EC
:10F030005FFA80F8611D55FA80F002F005FDA368C3
:10F04000246898445FFA88F3E2E720462468FFF7D3
:10F050006DFF002CF9D1DCE70120DEE770240020F1
:10F060000238C0B211289ABF014B185C00207047CB
:10F07000DF71010830B50B4B93F820200446084699
:10F0800072B100211C330578A54208D001319842A5
:10F09000CDB20CBF04480430AA42F4D8002030BDE1
:10F0A0001046FCE77C2600208826002010B5084C7E
:10F0B00000232060142204F10C00FF2184F820308A
:10F0C000C4E9010002F0D4FC012384F8213010BD12
:10F0D0007C26002010B50E4A92F82010042915D87D
:10F0E000936804781C7044785C70C4788078987059
:10F0F0000131DC7082F8201002F11C018B4214BF38
:10F10000043302F10C039360012010BD0020FCE7E2
:10F110007C260020094B93F8200068B15A6803F15F
:10F120001C018A4200F1FF3014BF043203F10C02CB
:10F1300083F820005A600120704700BF7C26002021
:10F1400010B5074B93F820200446084632B15968A1
:10F15000FFF790FF10B101234470837010BD00BF12
:10F160007C26002008B5064B93F820202AB1596868
:10F17000FFF780FF08B1407808BD0120FCE700BF21
:10F180007C26002030B50A4A92F82010536882F895
:10F19000210061B1916801241C32DD78587005B9F5
:10F1A0009C7093420CBF034B04339942F5D130BDA0
:10F1B0007C2600208826002008B5044B5968FFF7FC
:10F1C00059FF003818BF012008BD00BF7C26002071
:10F1D0002DE9F3410422154E044600210DEB0200F7
:10F1E00096F8208002F044FC0025EBB2984502D846
:10F1F00002B0BDE8F0817368197821705A786270A6
:10F200009F785FB1336820469B689847FFF782FF7D
:10F2100017B901A8FFF75EFF0135E6E7DB788DF847
:10F2200004108DF805208DF80730EFE77C260020CC
:10F23000014B93F8200070477C260020034B93F885
:10F240002000042894BF0020012070477C26002065
:10F250001FB50024CDE90244C41F8DF800408DF88D
:10F2600001100C0AADF80420090C120C8DF80310E3
:10F270008DF806208DF8073002461B0A01216846EA
:10F280008DF802408DF8083002F04FFA002818BFC0
:10F290000E2004B010BD2DE9F04188B017460D4690
:10F2A0000F9A064600284DD000240121CDE90444E0
:10F2B0008DF810109DF838108DF81510ADF8163037
:10F2C000190CCDE900441B0ECDE902448DF819302C
:10F2D000ADF81A20130C120E07948DF818108DF843
:10F2E0001C308DF81D20E3B24FEA0318002D5FFAA1
:10F2F00088F803DC002008B0BDE8F081013310215C
:10F300008DF81F303A466B460DEB010002F0A3F971
:10F310000346C8B9102DAC46A8BF4FF0100CDAB2A6
:10F32000624503F1010303DB103D2DB20134DAE73E
:10F3300008EB020020326A44315C12F8202C4A406B
:10F340003254ECE70920D6E70E20D4E70138032831
:10F3500015D8DFE800F002080C100A4B1B681B6987
:10F360000B6000207047074B1B685B69F8E7054B93
:10F370001B689B69F4E7034B1B68DB69F0E705201A
:10F38000704700BFA02600202DE9F041C4B00C4614
:10F390004A9E17461D468046B8B3B1F5807F36D8E1
:10F3A0004FF488720021684602F062FB4923009303
:10F3B0004FF48073ADF804302B0C8DF80830330C0B
:10F3C000ADF80650ADF80A608DF80C3022460023E7
:10F3D000414604A82D0E360E8DF80E308DF80950DA
:10F3E0008DF80D608DF80F4002F02EFB04F1100136
:10F3F0004B9A3B4689B2684602F017F910B10128D2
:10F4000018BF0E2044B0BDE8F0810920FAE70D20B6
:10F41000F8E7000010B590B10A4C282200212060C6
:10F4200002F026FB2368084A1A6000204FF0FF32E2
:10F43000C3E90302C3E90522C3E9072210BD08207E
:10F44000FCE700BFA026002000010101024B1B6861
:10F4500018600020704700BFA026002030B1044B88
:10F460001B68DB6801330360002070470920704788
:10F47000A026002013B500230C460193D2B101A9A8
:10F48000FFF764FF18B9019B591C02D1146002B048
:10F4900010BD99B2611A002902DD0B441360F6E732
:10F4A00002D113600720F2E71B0C1B0403F5803325
:10F4B0002344F3E70920EAE728B1044B1B681C3317
:10F4C0004362002070470920704700BFA02600203B
:10F4D0001FB5044600B3002303A8039302F07CF990
:10F4E000104ABDF80C30126820469380E38200F089
:10F4F00056FA98B904F118030093216801231322E6
:10F5000002F08AF860B9204600F049FA003818BFC6
:10F510000120000104B010BD0920FBE71020F9E72D
:10F520000E20F7E7A0260020F0B5054687B01C4660
:10F530003BB32F4E3368DB68834257D894F82020C2
:10F54000002A14BF09220822834205D3204600F076
:10F550005AFA70B110200AE0002301900093A368CA
:10F5600094F82810606AFFF796FE0028EED007B0E6
:10F57000F0BD23792168B4F808C0A768043B9AB2AB
:10F5800009B90920F3E7B2F5807F2DD8ADF80EC098
:10F590008DF817304FEA174C04F12C033F0E8DF80D
:10F5A000117000932F0C08234FF0490EADF80C009A
:10F5B0008DF814708DF816002F0E0DEB0300CDF8AA
:10F5C00008E08DF810C0ADF812508DF8157002F0FB
:10F5D00023F808B10E20CAE7204600F014FA0028EC
:10F5E000B8D13368DD60C2E70D20C0E70620BEE772
:10F5F000A02600202DE9FF410A9D80460F461646B1
:10F600001C46002D5AD0002303A910460393FFF790
:10F610009DFE18B1062004B0BDE8F081039B9C421A
:10F6200001D80133F6D1284600F05EF9002847D111
:10F63000264B1A78424503D01A79424542D101201F
:10F64000AA68BA4240D103EB8002EB6A92F80180CB
:10F650002979CDE900430439927828683B4689B27C
:10F66000FFF792FE0028D6D195F820300194002BA8
:10F670004FF00103009314BF4246082295F828106A
:10F68000686A3B46FFF707FE0028C4D1013E032EFF
:10F69000C1D8DFE806F002070B0F0D4B1B681C6199
:10F6A0001C62B8E70A4B1B685C61F9E7084B1B68F2
:10F6B0009C61F5E7064B1B68DC61ACE70920AAE713
:10F6C0000F20A8E70B20A6E70220A4E7A40800204B
:10F6D000A02600201FB50A460B2A4FF00001CDE9F5
:10F6E0000011CDE9021107D00C2A13D00A2A0FD03D
:10F6F0000A2005B05DF804FB012802D120238DF813
:10F700000030684602F011F8002818BF0E20F0E71C
:10F710003023F4E70B21F4E738B5054602F000F892
:10F72000044678B97DB9094B1B680B219878FFF71F
:10F73000D1FF38B90C21FFF7CDFF18B90A21FFF727
:10F74000C9FF00B10E24204638BD00BFA02600200E
:10F750002DE9F04380468FB00C461746002A6BD047
:10F76000002969D0002529461D2206A8059505F027
:10F7700000FC8DF81350344D2B680DF114099E8850
:10F78000CDF804900DF1130302933B7900933B688D
:10F7900032462146404601F0E4FF00284ED1386849
:10F7A0003A79494602F050F9384600F04FF80028FF
:10F7B00046D13C7AFA79BB79240444EA02241C43FA
:10F7C0002B689A6894423DD99C609DF813000B21E8
:10F7D000FFF780FF034658BB0C21FFF77BFF034672
:10F7E00030BB0A21FFF776FF034608BB7B7ABA7A63
:10F7F000FF7A3F0447EA02271F433A463346214631
:10F800000920FFF725FD034690B933463A462146C5
:10F810000820FFF71DFD034650B92A689DF8131014
:10F8200091700021D1604FF0FF31C2E90411916164
:10F8300018460FB0BDE8F0830923F9E70E23F7E778
:10F840000F23F5E70323F3E7A026002010B50446B5
:10F85000002845D00168002942D011F8013B4371CE
:10F860000322063002F0F0F82046032250F8091B6C
:10F87000043102F0E9F82168CB79E3600A7A43EABF
:10F880000223E3604A7A43EA0243E3608A7A43EA66
:10F890000263E360CB7A23740B7B63742379212B9F
:10F8A0001AD110220D3104F1120002F0CDF81D2200
:10F8B0002168501C8B5C6362085C43EA0023901C47
:10F8C0006362085C033243EA004363628A5C43EA92
:10F8D00002636362002010BD112B03DC0D22E7E7F9
:10F8E0000220F8E70120F6E710B50446002854D0BE
:10F8F0000168002951D00B7843714B7883608A7876
:10F9000043EA02238360CA7843EA024383600A79A8
:10F9100043EA026383604B7903738B79C381CA79AD
:10F9200043EA0223027BC38102F00F020831103048
:10F9300002F08AF8237B002203F00F0384F82020D2
:10F9400084F82820227903F10800111A04290DDD1A
:10F9500021680933043AD21A085C84F82000D2B234
:10F96000606A84F82820194402F06EF8237922682E
:10F970001A44002012F8043CE36212F8031C43EA24
:10F980000123E36212F8021C43EA0143E36212F826
:10F99000012C43EA0263E36210BD0220FCE710B5CC
:10F9A000044660B3036853B30279162A29D9427911
:10F9B0001A700146082251F8060B013002F04EF889
:10F9C0002146082251F80E0B093002F047F823684F
:10F9D000E28A5A74E38A22681B0A93742368A26934
:10F9E000DA74A36922681B0A13752368628B5A753F
:10F9F0002368E27E9A7517232371002010BD012031
:10FA0000FCE70220FAE738B50446002863D0016815
:10FA1000002960D0037B90F8282003F00F03002A10
:10FA200057D10833207904321344984255D363796F
:10FA30000B702368A2685A70A36822681B0A93702F
:10FA400023686289DA702368E27A1A712368227B5C
:10FA50005A712368E2899A71E38922681B0A214658
:10FA6000D371227B51F8100B02F00F02083001F025
:10FA7000EBFF237B94F8282003F00F0303F1080524
:10FA80002AB1226894F82010515503F10905206825
:10FA900094F82820616A284401F0D6FF94F82830B1
:10FAA0002268E16A2B44D1545A1CE16A206892B260
:10FAB000090A81549A1C2168E08D92B28854DA1C9C
:10FAC000216894F82F0092B20433885423710020E7
:10FAD00038BD0933A6E70120FAE70220F8E7000065
:10FAE000024B1A8810431880704700BFA4260020DC
:10FAF00008B5074B1B883BB1FEF7B8F900280CBFCF
:10FB000000206FF0020008BD6FF00100FBE700BFAE
:10FB1000A426002010B5034B00241C80FEF79CF99E
:10FB2000204610BDA4260020B0FA80F0400970479E
:10FB300082B018B9084602B000F0CAB8002002B07E
:10FB4000704710B9084600F077B9704710B90846F9
:10FB500000F08EB970470346084611460BB900F015
:10FB6000E5B90020704710B9084600F071BD704734
:10FB700010B9084600F006BA0020704710B40446D9
:10FB8000084611461A46019B14B910BC00F018BA79
:10FB900010BC70470346084611460BB900F042BA44
:10FBA0000020704710B40446084611461A4614B99E
:10FBB00010BC00F0AFBA002010BC704730B405464E
:10FBC000084611461A46DDE902341DB9029430BCDC
:10FBD00000F02EBB002030BC704710B9084600F082
:10FBE000DFBB0020704710B9084600F06FBD002051
:10FBF000704710B9084600F0EEBB0020704710B9FE
:10FC0000084600F0EBBB002070470346084611464B
:10FC10000BB900F005BC0020704710B4044608463C
:10FC200011461A46019B14B910BC00F0FBBB092019
:10FC300010BC704710B40446084611461A4614B961
:10FC400010BC00F063BDC8B210BC704700487047DC
:10FC500001000102064B10B51B6A0446984730B1FB
:10FC60000448054B204498428CBF0020012010BD61
:10FC7000D078010840C220C980B92A00F0B5114BE4
:10FC800085B00C4610491F56054601F049F80F4B48
:10FC9000E4B25E6A072D4FF00103CDE9024301464D
:10FCA0000AD105220023CDE900234FF47A727A436A
:10FCB0001846B04705B0F0BD08220020CDE900206D
:10FCC0003A46F5E71B720108F4710108D078010883
:10FCD0001FB5002300930378013B372B21D8DFE8C1
:10FCE00003F01C242020201E202020204143454ECC
:10FCF0002055585B5E6164206C1E6E73787A2020FC
:10FD00007D8126202020202020202020202020202F
:10FD100083858A2020838A208C90C3780BB10223AC
:10FD20000093009805B05DF804FB8378F6E743780C
:10FD30008DF8043005238DF805308378003B18BF1B
:10FD400001235B008DF8063010238DF80730304B0F
:10FD50001B6801A803F55872CDE9022300F0C0FF2B
:10FD60000090DEE74023DBE72023D9E7827890F993
:10FD7000013012B9274AD35CD2E7274AFBE78278E1
:10FD800090F90130002AF8D1244AF4E740F6B8335C
:10FD9000C6E74FF47A73C3E74FF4FA63C0E741F262
:10FDA0008833BDE741F27073BAE71D484FF47A71AA
:10FDB00001F02EFE00F5FA60D2E71A4BB0E7144BC3
:10FDC0001B6803F55873ABE7114B1B6803F55B73B6
:10FDD000A6E71023A4E70E4B1B68A1E74FF083436F
:10FDE00000939EE7104BFBE7104B99E740F211138D
:10FDF000ADF8003095E7032392E790F901300C4A03
:10FE0000B9E70C4990F9010000F08AFFA8E700BFAC
:10FE1000AC260020A3720108AB720108B37201087E
:10FE200018FCFFFF00EA06379A99094040F70937A6
:10FE30001B720108F471010837B50B4B02781B687F
:10FE40000C2101FB02335B7A03EB4304074B1D6873
:10FE500003690093C3684278816805EBC40000F031
:10FE6000DFFC03B030BD00BFAC260020A826002078
:10FE700070B586B0027B6423ADF80030012A4FF0E4
:10FE80000003CDE90133CDE903338DF802308DF85D
:10FE9000143030D0022A39D05ABB03684BB34368C0
:10FEA0003BB31F4D80682B601E4B182269461860BB
:10FEB00001F0CAFD1C4B2C6893E807000C3384E862
:10FEC000070093E8070004F10C06032386E8070007
:10FED000A4F86C33012204F55B7104F5587000F04E
:10FEE00090FC2B684FF6B072A3F878230522C3F874
:10FEF0007C2306B070BD0A4908684360036100F5C1
:10FF00005B7100F5587000F07CFCF2E7044B1B6855
:10FF1000B3F86023B3F86C130A43A3F86023E8E74F
:10FF2000AC260020A8260020486F010808B503462B
:10FF30000A2924D8DFE801F006232323230B161B0C
:10FF400023212100BDE808400068FFF783BE90F937
:10FF500000009978052271B900F013FC003818BF31
:10FF6000012008BD052293F900000021F4E790F973
:10FF700000005978EEE70221EEE70722F3E70020C0
:10FF8000EFE7000010B504791CB1012C0BD0002064
:10FF900010BD0A4B01681B68012203F5587000F080
:10FFA00030FC0120F4E7054B01681B68224603F58D
:10FFB0005B7000F026FC2046EAE700BFAC2600207C
:10FFC000F7B50528144D1C46A8BF052058700E46ED
:10FFD0002946174600F0A4FE94F90130A070072BC3
:10FFE00013D1322000F09CFD0C4BDB6D0546984789
:10FFF00004F10C0208340346019200943A4631465B
:020000040801F1
:10000000284600F092FD03B0F0BD054A55F82310D4
:10001000D05C00F07DFDE7E7F4710108D0780108BD
:100020001B7201082DE9F04F344F90F901607B6895
:10003000D0F804908BB004468846984705460028BF
:1000400059D1E37C73B92E4A2378126803EB43033A
:10005000990002EB8303D3F80490B9F1000F01D1AA
:1000600052F80190274B484613F906B0FB689847B1
:10007000A37CD7F818A022890993072E28D1002342
:100080000121CDE90223204A0693CDE90431CDE9CF
:1000900007330521CDE900214FF47A7202FB0BF200
:1000A0004CF250311846D047637C13B3174B995D1F
:1000B0007B6D0D31C9B228469847E07C32464946EF
:1000C00000F040FE88F8006001200BB0BDE8F08F22
:1000D000002101250823CDE90013CDE90715CDE95D
:1000E0000511CDE903110292A1782B465A46284604
:1000F000D9E7074BDBE70020E7E700BFD07801082E
:10010000AC2600201B72010885450100B37201086E
:10011000A37201082DE9F04F8DB090F90130DFF89E
:10012000FCA0DFF8FC90CDE90A123E4A12F903B0B8
:100130000278DAF800300C2505FB02333A4A5B7A84
:10014000126803EB430302EBC303044693F9021066
:1001500090F9020000F0DFFD3449064694F90100F1
:1001600000F0DEFDA26861688046304600F005FDC3
:100170002178DAF80020D9F80C3069430746505846
:100180009847D9F81C309C4694F901300025072B7C
:100190004FF47A63CDE90753CDE905552DD10123FD
:1001A000CDE903530523CDE901534FF47A7303FBE3
:1001B0000BF300933946434646F2A8122846674699
:1001C000B8472378DAF800200C214B4394F901104A
:1001D000D05800F0D9FDA18994F90100FFF74EFD38
:1001E0000B9B217B1860D9F85430284698470A9B0E
:1001F00001201E700DB0BDE8F08F01200823CDE96D
:100200000350CDE901032A46CDF800B065464346C8
:100210003946A84701200546D3E700BFAC26002099
:10022000D07801081B720108A8260020F47101088B
:100230002DE9F04F8FB0002405468A469146984636
:100240000494ADF81440ADF8024007264FF0010BBE
:100250002B7AA34206D9686804A9204400F0F2FB77
:1002600000285ED102238DF8083002A86B7A8DF841
:100270000A30FFF72DFDAB7A8DF81D309DF8113057
:100280008DF81E309DF812308DF81F309DF810301B
:100290008DF82030EB7A8DF821302B7B8DF82230D1
:1002A0006B7B8DF8233010238DF81C608DF8243083
:1002B0003A4E8DF82C000DF102030A9305238DF8B8
:1002C0002D3033680C930723ADF834302B68069338
:1002D0000DF1120204AB0DF1110106A800F0CCFBE8
:1002E000072805460BD130680C22002100F5587014
:1002F00001F0BEFB3368BDF80220A3F860239DF82F
:1003000011308AF800309DF8123089F800309DF8DD
:10031000103088F80030189B28461C700FB0BDE8DC
:10032000F08F9DF81330BDF81470ADF802702044C2
:10033000C4B2F3B917B3194A002011680726024660
:100340004FF00C0C062B1BD10CFB00FE51F80EE0FD
:10035000BEF1000F04D00BFA00F23A4397B201222B
:1003600001301028EED1002A3FF472AFADF80270D0
:100370006EE75A1E042A01D9062BDCD0062667E751
:1003800047FA00FE1EF0010FEAD00CFB00FE51F808
:100390000EE0BEF1000F08BF0626E1E7AC26002004
:1003A00038B505464068FFF755FC0522841D00213D
:1003B00095F90000E4B200F0E4F908B904F0FD0496
:1003C00095F901000722002100F0DBF908B904F0DB
:1003D000FB04204638BD00207047000010B50378AC
:1003E0000F2B044618D84068FFF734FC22780B49DD
:1003F00002EB42020968831C01EB820051F82220C3
:10040000DBB21AB903F0FD0358B210BD032B06BFCF
:10041000626842600223F7E70020F6E7AC2600207E
:10042000022070472DE9F04FDFF838810446D8F8F4
:10043000000099B08946174600211E460122032379
:1004400000F55870CDE90611CDE908118DF81410AA
:100450008DF81510ADF8163000F0B5F938B9D8F8A8
:100460000020B2F8603343F00303A2F86033D8F8F9
:100470000020637A8DF8283002F55871CDE90B120F
:10048000394A94F9083012680D920DF116020F9254
:100490002268109262681192D4E90301A27A8DF861
:1004A000482001228DF8492013AA82E80300102574
:1004B000227DE18A8DF8293018468DF85420ADF858
:1004C0003850FFF7DBFB0AAB17930DF115031690BD
:1004D00000933146019705AB06AA10A800F0BCFBBB
:1004E000064698BB9DF81410204F013901F090FA90
:1004F0001F4B1B690393C4B24FF00C0B04F1600354
:100500006B44D8F8000013F848AC9DF814300BFB8E
:100510000AFC01343946B4FBF3F203FB1244D0F871
:100520007C33B0F9782350F80C00DDF80CC0E4B24D
:10053000E04728B189F800A0304619B0BDE8F08F37
:10054000013D15F0FF05D9D10D26F5E70C2801BFB7
:10055000D8F80020B2F8603343F00303A2F8603308
:10056000EAE700BFAC260020A8260020400D0300CB
:10057000D0780108F8B50679012E054601D8062085
:10058000F8BD0F2E2BD80368187A40F3030005221C
:10059000002140B200F0F5F82B680446187A40F3C9
:1005A00003100522002140B200F0EBF8A8B1B4FA24
:1005B00084F4640929680B7A086843F3030243F35F
:1005C000031352B25BB29A42C8BF0124FFF742FB49
:1005D00048B9002CD3D10420D2E70124EAE7032054
:1005E000CEE70520CCE7002CFBD10C4F29683B68F7
:1005F00006EB460003EB80000C2201F025FA3A6876
:100600000C2303FB062320465C72B2F8601301231F
:10061000B3400B43A2F86033B2E700BFAC26002022
:1006200010B4017801290ED9084B18680C234B43EC
:10063000C4180022C250C4E9012200F5587010BC51
:10064000102200F0A7B8002010BC7047AC26002094
:100650002DE9F04186B050238DF81430037A102B29
:10066000074630D14368DD7B6DBB0224A846642673
:10067000062C14D87A68535D03932A44517843EAD0
:1006800001230393927843EA02437343CDE903388D
:1006900063B968468DF80040FFF7C2FF0DE0CDF862
:1006A0000C808DF81480CDF81080F2E703AB01A820
:1006B00001938DF80840FFF75DFF0134E4B2102C80
:1006C00005F10305D4D106B0BDE8F0811FB502687D
:1006D0000379116851B901A88DF80430FFF7A0FF24
:1006E00078B9002040B205B05DF804FB02A8029280
:1006F0008DF80C30FFF73EFF0628F2D8024B185C4D
:10070000F0E70320EEE700BF14720108C90020B92A
:10071000034B0B449856C0B27047024BF9E700BF39
:100720002372010863720108F0B59A42069D03DB4B
:100730009DF914309A4220DD0020F0BD03EB430305
:1007400031F814C005EB830300264CFA06F7FF07C7
:1007500007D51F7A07F00F0E724502DBB2EB171FA9
:100760000DDD0136102E03F10C03EED10134E4B29D
:100770002301DBB29842E1D8DEE70024F8E701204C
:10078000DBE7884204DB9042CCBF002001207047A9
:100790000020704710B51409B4EB111F03464FEA4F
:1007A00011100ED391420CD202B201F00F0133F8B6
:1007B0001240012000FA01F124EA010123F812108D
:1007C00010BD0020FCE7F0B528B100EB4105012782
:1007D0000020914200D3F0BD002435F802CB23461F
:1007E00007FA04F636EA0C0608BF013304F10104E7
:1007F00008BFDBB2102CF3D118440131C0B2C9B22A
:10080000E7E710B500B149B910BD31F8134020F841
:1008100013400133DCB2A242F7D8F5E70023F9E731
:1008200082B030B5048804936AB9B3F5616F18D308
:1008300049F6AF2542F21072AB4298BF4FF47A727C
:10084000944238BF1446012C38BF01246143BDE8EF
:100850003040C3688B428CBF5B1A0023C36002B078
:1008600070476422ECE700002DE9F04F91B0154687
:10087000DDF86C8004939DF8683009930C460646B9
:1008800003F0C2FB684ADFF8A4B10590A8F5F6337F
:10089000303BB3FBF2F3534303F5F63203F5A833D1
:1008A00003F5C0730393182313FB054330320692FC
:1008B000089300254FF0FF3A089BA34207D1002D73
:1008C00014BF50464FF0FF3011B0BDE8F08FBDF9B6
:1008D0007030ADF82C300B99CDF86C804046CDF8D7
:1008E000288003F021FBB4F800906EB9B8F5616F71
:1008F0005BD349F6AF2242F21073904598BF4FF494
:100900007A73994538BF99464B46012B38BF01236E
:100910000793002E52D1B9F1640F48D1A0605F4611
:10092000A1680EA803F022FB0F9B0093DDE90A12D9
:100930000E9B0CA803F079FA049B0C9A0BB9099B47
:100940002BB12369BB4202D1394B9A420DD9394BA5
:10095000E760984509D90023ADF83430069B0D991E
:100960000C93184603F0E0FAA060606800B9E760F5
:10097000276126B103F052FBE3680344E360D4E946
:1009800003329342059B1D996360079B88BFE26019
:100990004B43E168994202D20498A8B9A6B1012359
:1009A0001D442375EDB2183486E76423A9E7B9F531
:1009B0007A7F0ABF204F214FA060B1E7049B0BB99B
:1009C000C4F80CB05F46D0E700209342207506D8EB
:1009D0005B1A9A4505F1010528BF9A46EDB2002E33
:1009E000E1D1B9F1640F164AADF8346019D049F677
:1009F000B023B9F57A7F18BF1346904584BF039A98
:100A00009B180C931C9B00930CAF97E806001B9B54
:100A1000384603F00AFA97E8030003F085FA8246A5
:100A2000C1E74FF46163E8E78051010040771B00A4
:100A30007F5101002FEC010080A81201002E9302CB
:100A400030EC01000378032B14D1437803F00F023C
:100A50001B098A704B7083788B80C27843EA02232B
:100A60008B800379C3F3021203F00F03CA700B707B
:100A700005207047002070472DE9F34798464379D9
:100A8000057990F907609146044690F906208A4658
:100A900083B190F9087075B30F2A12D194F9092027
:100AA0000F2E1ED194F90A60072D24D1002F08BF04
:100AB000012720E090F90B7090F9092090F90A6065
:100AC000E9E7A369019394F915300093216994F93A
:100AD0001430207BFFF728FE0028E1D105F0FD054A
:100AE000DEE794F91D30B3420FDC94F91C30B342B9
:100AF000DADA05F0FB0528468AF8002089F800605C
:100B000088F8007002B0BDE8F0871E46CCE7000010
:100B1000024B03FA00F0B0FBF1F0704740420F00C7
:100B20004FF4FA53B3FBF0F0704730B54FF47A75D9
:100B30000C1F6A4300FB042252001EBF00F1FF3469
:100B40001219B2FBF0F2914238BF1146039A1160BC
:100B5000820048431CBF013040084FF47A71121ADA
:100B600001FB1323002BCABF03F2E73393FBF1F120
:100B7000B3FBF1F1049B196030BD38B54000144659
:100B80000D46F1F7C7F901462846F1F711F921465C
:100B9000F1F70EF9F0F7D8FD06F02EF9F1F7DCF8D1
:100BA00040B238BD2DE9F74F019300231F469C4604
:100BB0001C01058A5FFA84FE04F0F004A54206D801
:100BC000019B82F800C01F7003B0BDE8F08F0EEBF0
:100BD0004E054FEA4309AD000024466836F8096027
:100BE0002641F60727D5866806EB050A765916B31F
:100BF000067836B9466926B136F809602641F60707
:100C000019D59AF8086090F901B046F303084FFA35
:100C100088F8D8450FDC46F3031676B25E450ADB4A
:100C20009AF8096006EB4608C66806EBC806367DEA
:100C30004EB90137FFB20134102C05F10C05CCD1AF
:100C40000133DBB2B4E70CF101060EEB040801F846
:100C50000C805FFA86FCEEE72DE9FF47044640680A
:100C6000DDE90C671D468A46914603F0D7F92368F3
:100C70001B1A3B604FF000080123337085F8008099
:100C8000636813B12368834224D8CAF80080D4F87B
:100C90001CC0A3699CF800E00393D4E9030101ABF5
:100CA00083E80300237D0093DCF80C10237A627A3A
:100CB0007046FFF7D9FD334638602A46E069494659
:100CC000FFF770FF2B782BB1C7F80080002004B02D
:100CD000BDE8F0873378002B14BF0B200C20F6E71B
:100CE00037B590F9002090F90250954204460FD094
:100CF000013A52B295420BD0A368019394F90130A6
:100D000000936168E0782B46FFF70EFD0028EFD0D6
:100D1000104603B030BD8842B8BF08467047000097
:100D200051F82000054B984205D0054BC31A584294
:100D30005841400070470120704700BF90D0030029
:100D400020A1070005281FB50ED80C4B53F8203002
:100D50000093CDE901120A4B01220021022002F08A
:100D600069FE05B05DF804FBCDE90012054B0122D8
:100D70000021022002F05EFEF3E700BF28730108A5
:100D8000BB720108DA72010807B5054BCDE9000115
:100D900001220021022002F04DFE03B05DF804FBA9
:100DA000F672010810B5102204460021F13000F05F
:100DB0005FFE0021C4F814112046F022BDE8104067
:100DC00000F056BE02460846102100F0A5B92DE9F4
:100DD000F0430446D0F8140185B00E46154604F2DF
:100DE000011988B3C0F110089045474628BF17463F
:100DF000BAB2484400F028FED4F814313B440F2B1B
:100E0000C4F814312DD9A8452BD204F1F00304F510
:100E1000807113F8012F187C8B4282EA00021A704D
:100E2000F7D104F1F10810224146684600F00CFEAB
:100E300022466946684600F0E9F9102269464046B4
:100E400000F002FE3E44ED1B04F5807804F1F1074A
:100E5000102D09D8AAB23146484600F0F5FDC4F875
:100E6000145105B0BDE8F08304F1F003711E13F8CE
:100E7000012F11F8010F434582EA00021A70F6D1E2
:100E800010223946684600F0DFFD22466946684672
:100E900000F0BCF910226946384600F0D5FD103646
:100EA000103DD5E7F0B589B00C461022002105466B
:100EB000684600F0DDFD22466946684600F0A6F966
:100EC0009DF90030002B6A464FF0000143DA137899
:100ED00012F8010F01315B0043EAD0130F2902F829
:100EE000013CF4D19DF80F305B0083F08703D4F808
:100EF0001401DBB210288DF80F303BD104F580735C
:100F0000694604F5887013F8016F11F8012B9842B7
:100F100082EA06021A70F6D104F1F00304F580713A
:100F200013F8012F187C8B4282EA00021A70F7D165
:100F300010220DEB020004F1F10100F085FD2246C4
:100F4000294604A800F062F910220021684600F04A
:100F50008FFD09B0F0BD137812F8010F01315B006D
:100F600043EAD0130F2902F8013CF4D19DF80F3069
:100F70005B00BCE79DF90030002B6A464FF0000192
:100F800037DA137812F8016F01315B0043EAD613A8
:100F90000F2902F8013CF4D19DF80F305B0083F07B
:100FA0008703471CDBB28DF80F30102F04EB0003D2
:100FB000C0F10F064FF0800288BF002600F5817057
:100FC00083F801210021324620443E4403F0D1FF42
:100FD000C4F8146104F58073694604F5887013F849
:100FE000016F11F8012B984282EA06021A70F6D1BD
:100FF00092E7137812F8016F01315B0043EAD613D0
:101000000F2902F8013CF4D19DF80F305B00C8E7CE
:101010000A780378534003704A784378534043700A
:101020008A78837853408370CA78C3785340C370FA
:101030000A790379534003714A79437953404371E4
:101040008A79837953408371CA79C3795340C371D4
:101050000A7A037A534003724A7A437A53404372BE
:101060008A7A837A53408372CA7AC37A5340C372AE
:101070000A7B037B534003734A7B437B5340437398
:101080008A7B837B53408373CA7BC37B5340C37388
:10109000704710B50B7814786340037054784B7820
:1010A0006340437094788B7863408370D478CB78B6
:1010B0006340C37014790B796340037154794B79A1
:1010C0006340437194798B7963408371D479CB7990
:1010D0006340C371147A0B7A63400372547A4B7A7B
:1010E000634043728B7A947A63408372D47ACB7A6A
:1010F0006340C372147B0B7B63400373547B4B7B55
:1011000063404373947B8B7B63408373CB7BD27B45
:101110005340C37310BD0000A1F11003DBB2102BCC
:101120002DE9F04704D8374C24FA03F3DB0705D444
:10113000002382F8F030FF20BDE8F087531E4418EA
:10114000A0424ED101F11C039B005FFA83F9C3F367
:101150000313013B2C4D82F8F03001240B46D618C6
:10116000B3FBF1F001FB103010F0FF0016F804ACF7
:1011700016F803EC16F802CC16F8017C36D115F8F7
:101180000E8015F80CE015F807C015F80A70E00994
:1011900000EB400084EA080800EBC0006400C0B225
:1011A000E4B24440C246581AC0B212F800808AEA3B
:1011B000080A02F803A01044043390F801808EEA74
:1011C000080E86F801E090F802E08CEA0E0C86F832
:1011D00002C0C078DBB247409945F770BFD8002005
:1011E000AAE710F8015B03F8015FA9E71829DAD92B
:1011F000102801BF15F80AA015F80EE015F80CC06C
:10120000EF5DD0E701010100407501082DE9F04FC5
:10121000A3B092F8F0301D911B920193002B00F0C7
:10122000538101461EA8FFF734FF1B9BA74CA84D16
:10123000A84E10330293002303939DF87C00049082
:101240009DF886000590205C06909DF87B00079035
:10125000205C089004989DF881C0205C099014F8E7
:101260000C000A909DF880000B909DF885009DF879
:1012700078809DF87DE09DF882A09DF887900C9085
:101280009DF87A00029B1C9314F80A2014F8093088
:1012900014F8081014F80E700D90205C0E909DF854
:1012A0007F000F90205C10900B98205C11900C98A0
:1012B000205C12909DF8840013909DF879001490A2
:1012C0009DF87E001590205C16909DF88300179085
:1012D000205C18901398205C19901498205C1A9048
:1012E0000398013003900298DDF804B010300290AA
:1012F0009DF80C00834536D88DF878108DF87A204B
:1013000009990E9A8DF87C108DF882201199069A11
:101310008DF880108DF87E201999169A8DF884101A
:101320008DF886200A99189A8DF87D108DF88720FF
:101330001299109A8DF87B301B9B8DF881108DF8D7
:1013400083201A99089A1D988DF885108DF87F20B2
:101350001EA903EB0B128DF87970FFF79AFE00209F
:1013600023B0BDE8F08F15F808B082EA03008BEADD
:10137000000016F80EB080EA0B008DF8780015F822
:101380000E004B40434016F80A0043408DF8793078
:1013900081EA070315F80A10594016F80930594038
:1013A00016F808308DF87A107A40534015F8092065
:1013B00053408DF87B30089A069B5340049AAA5CF0
:1013C000534016F80C2053408DF87C30DDE908328C
:1013D0005A4015F80C305340059AB25C53408DF8D2
:1013E0007D30DDE909325A40059BEB5C5340079A9A
:1013F000B25C53408DF87E30069B0A9A5340049AA3
:10140000B25C5A40079BEB5C5A408DF87F200E9BE4
:10141000109A53400B9AAA5C53400C9AB25C53400A
:101420008DF88030DDE910325A400C9BEB5C534064
:101430000D9AB25C53408DF88130DDE911325A408B
:101440000D9BEB5C53400F9AB25C53408DF8823099
:10145000129A0E9B53400B9AB25C5A400F9BEB5C66
:101460001C995A408DF88320169B189A5340139A62
:10147000AA5C5340149AB25C53408DF88430DDE985
:1014800018325A40149BEB5C5340159AB25C53409F
:101490008DF88530DDE919325A40159BEB5C5340DD
:1014A000179AB25C53408DF886301A9A169B5340B7
:1014B000139AB25C5340179AAA5C1EA853408DF849
:1014C0008730FFF7A5FDB8E6FF2049E74075010822
:1014D000407301084074010808B538B1044A054951
:1014E0001060D82200F0B0FA002008BD0220FCE70E
:1014F000B0260020DC7D01080A4B1A6870B5002375
:1015000002F1180503EB03142E5D864204D1183452
:1015100022440A60002070BD01330B2BF2D103205E
:10152000F9E700BFB02600202DE9F041CCB0064617
:10153000DDF8488117461C460D4631B3B8F1000F5F
:1015400023D006A8FFF72EFC204601A9FFF7D4FF01
:101550000446B0B9019906A80131FFF733FC26B162
:101560001022314606A8FFF732FC3A46294606A863
:10157000FFF72DFC06A902A8FFF794FC029BC8F810
:10158000003020464CB0BDE8F0810224F9E70000AD
:1015900030B595B013A90446FFF7AEFF002830D14F
:1015A0001B490C2303FB00F2555CA5422BD1139B76
:1015B000187C1090D87B0F90987B0E90587B0D90E4
:1015C000187B0C90D87A0B90987A0A90587A0990E8
:1015D000187A0890D87907909879069058790590EC
:1015E00018790490D8780390987802900A445B7830
:1015F0000193936800930022064B1146022002F0EB
:1016000019FA15B030BD01300B28CBD1F9E700BF76
:10161000B8770108407601080B2B10B402D810BC33
:10162000FFF782BF032010BC704730B50D4685B070
:101630001446014668B103AA002000922A4603908E
:10164000FFF772FF18B90398001B18BF012005B0FF
:1016500030BD0220FBE72DE9F0430D46BFB0144634
:101660009946804620B31BB311F00F0122D1F0221E
:1016700001A800F0FDF920466946FFF73DFF04464A
:1016800048B9009801AA10210130FFF745FD2E4608
:10169000AF1BFFB21EB920463FB0BDE8F08301AAE0
:1016A00009EB070108EB0700FFF7B0FD103EEFE77D
:1016B0000224F0E70524EEE7F0B5184E3468024640
:1016C00085B00846002304F1180103EB03154F5DB4
:1016D00097421ED10D2A05F1190513D10023CDE93A
:1016E0000033CDE902330C2210216B46FFF7B3FF24
:1016F0000446306810226946284400F0A5F92046C7
:1017000005B0F0BD01461022601900F09DF90024DB
:10171000F5E701330B2BD8D10324F0E7B0260020E6
:1017200009B1FFF7C9BF022070471FB51446A0B129
:101730000C2A01D10B2912D10023CDE90033CDE9C8
:1017400002330A466B461021FFF785FF18B9694638
:101750002046FFF7B1FF04B010BD0220FBE70320D5
:10176000F9E7F8B51E46DDE907479DF818505BB369
:1017700054B34FB3212D29D819462A46204600F0EC
:1017800063F90122631C691EB018FFF764FFF8B902
:10179000E37ADB093B70EBB96319204613F8012C9F
:1017A00013F8021C120642EA014213F8041C0A4311
:1017B00013F8031C012342EA0122291FFFF735FF1A
:1017C000003818BF0120F8BD0220FCE70520FAE729
:1017D0000720F8E70420F6E710B5044628B1044BCB
:1017E0005B6998472060002010BD0220FCE700BF25
:1017F000D078010808B5014630B1044B08221868BA
:1018000000F022F9002008BD0220FCE7B0260020ED
:1018100008B530B1044B0822196800F015F9002012
:1018200008BD0220FCE700BFB02600207FB5124EA5
:101830000023044602A801930D46FFF7E9FF336831
:101840005B6901936CB102AA082312F8011B41B92C
:10185000013B13F0FF03F8D102A8A04702A8FFF74D
:10186000C9FF35B1019B23B901A8A8473368019A84
:101870005A61002004B070BDB026002008B50146B2
:1018800038B1054B18680822104400F0DDF800203C
:1018900008BD0220FCE700BFB026002008B538B123
:1018A000044B19680822114400F0CEF8002008BD4E
:1018B0000220FCE7B0260020034B1B6802280CBF67
:1018C0001961596100207047B026002041B1054BD5
:1018D0001B6802280CBF1B695B690B600020704706
:1018E00002207047B026002030B58FB00024054696
:1018F0000CA80994FFF78CFF9DF8373007939DF8EB
:10190000363006939DF8353005939DF834300493B6
:101910009DF8333003939DF8323002939DF83130B7
:1019200001939DF830300093224621461E4B022041
:1019300002F080F80AA8FFF7B1FF9DF82F30079357
:101940009DF82E3006939DF82D3005939DF82C3090
:1019500004939DF82B3003939DF82A3002939DF851
:10196000293001939DF82830009322460F4B2146E1
:10197000022002F05FF809A92846FFF7A7FF9DF8AB
:10198000243003939DF8253002939DF8263001936F
:101990009DF8273000932246054B2146022002F095
:1019A00049F80FB030BD00BF9C760108DA76010817
:1019B0001877010808B50020FFF7EAFD0120FFF7BE
:1019C000E7FD0920FFF7E4FD0820FFF7E1FD002017
:1019D000FFF78AFF002008BD10B504460B20FFF773
:1019E000D7FD0C20FFF7D4FD0920FFF7D1FD08201B
:1019F000FFF7CEFD0A20FFF7CBFD2046FFF774FF6F
:101A0000002010BD014B1860704700BFAC080020DB
:101A10000B4A30B514680B4D43F2390305FB043310
:101A20001360091A6FF00042B3FBF2F2C2EBC2720C
:101A300001319B1A93FBF1F201FB1233184430BDC4
:101A4000AC0800206D4EC64101380A44914200D1D5
:101A5000704711F8013B00F8013FF7E710440A44D2
:101A6000914200D1704711F8013B00F8013DF7E7C2
:101A700003F07FBA30B530B10A4D01444FF0FF3367
:101A8000814201D1D84330BD10F8012B53400822C8
:101A900043F30004013A2C4092B284EA5303002A33
:101AA000F6D1EDE72083B8ED01207047054B4FF4E8
:101AB00000529A62044B1B6813B15B6803B118476C
:101AC000704700BF00040048B4270020054B4FF4C6
:101AD00080529A62044B1B6813B1DB6803B118474C
:101AE000704700BF00040048B42700200120704761
:101AF0000120704701F048B901F036B910B501F086
:101B000019FE0E21044640F61F1001F02DF9204663
:101B1000012101F0F9FDBDE8104001F0D7BA000045
:101B200070B50C4E01EB40030D46B3654FF6FF71E7
:101B3000002304461A46084601F05EFB96F856005C
:101B4000002101F0E1FD29462046BDE8704001F08A
:101B500095BA00BFD027002010B5044601F0AAFEB8
:101B600001281CD101F0AEFE34B11248214602F02A
:101B700017FB104802F0DAFA0F4C104B00214FF41B
:101B80008052A1659A6194F8560001F0BDFD63781A
:101B90006BB16FF07F40BDE8104001F053BA0023F5
:101BA00040F262211A46084601F026FBDCE7A068F5
:101BB0008001F0E7B8270020D0270020000400486B
:101BC000002001F0BFB9000008B501F0C7F80438E3
:101BD000C0B2032896BF024B0020185C08BD00BFAE
:101BE000CC78010808B501F0BAFD033008BD01F05A
:101BF00049B901F009B908B501F000FD00B208BD0E
:101C000038B50D46144601F05DFB284601F092FD03
